:020000040000FA
:040000006FD00400B9
:101000006F00907E00000000000000009020002093
:10101000AA220020A9BDF9F56C23002000000000E1
:10102000000000006C230020902000200000000041
:101030000000000090200020000000009020002010
:101040000000000090200020902000209020002030
:101050009020002090200020582F00209424002071
:101060000000000090200020902000201E2400207E
:1010700090200020D22300209020002090200020EB
:101080009020002090200020902000209020002020
:101090009020002001A04111B7170040985F3AC688
:1010A000945F3247E39CE6FE3245410182800111A4
:1010B00013078008F337078093F787083EC20100C3
:1010C0000100B7170040930570052380B70413068D
:1010D00080FA2380C7040100010083C6B70493F699
:1010E000F60DA385D704238007049246F3A6068055
:1010F0000100010093760502D5CEF336078093F602
:10110000860836C4010001002380B7042380C70489
:1011100001000100B70614007D89558D88C70100C4
:1011200001000100010023800704A246F3A6068007
:101130000100010073370780137787083AC6010062
:1011400001002380B7042380C704010001000100CF
:1011500001003727004093061005A303D7802380A2
:101160000704B247F3A70780010001009307800836
:10117000F3B7078093F787083ECE01000100B71749
:101180000040130770052380E704130780FA2380CB
:10119000E7040100010003C7B70413670708A3852C
:1011A000E70423800704F247F3A70780010001004A
:1011B0000561828093760504BDC6F336078093F6F9
:1011C000860836C8010001002380B7042380C704C5
:1011D00001000100B7061400938606047D89558D31
:1011E00088C7010001000100010023800704C246F6
:1011F000F3A6068001000100733707801377870884
:101200003ACA010001002380B7042380C70401000B
:1012100001003727004093062005A303D7802380D1
:101220000704D24781B773370780137787083ACC12
:10123000010001002380B7042380C70401000100DE
:1012400098471367070C98C723800704E24719BF24
:101250000111814601468145114506CE97000000E7
:10126000E780605893078008F3B7078093F78708F3
:101270003EC601000100B717004013077005238028
:10128000E704130780FA2380E7040100010003C785
:101290006704136717002383E70423800704B2471A
:1012A000F3A7078001000100F2400561828041112F
:1012B000814601468145114597000000E780A05214
:1012C00013078008F337078093F787083EC40100AF
:1012D0000100B7170040130670052380C70493066A
:1012E00080FA2380D70401000100FD552396B70240
:1012F00023800704A245F3A5058001000100733790
:101300000780137787083AC6010001002380C704CD
:101310002380D7040100010003C767041367170087
:101320002383E70423800704B247F3A70780010063
:10133000010001A0B1473305F50201007D1575FDDF
:101340008280411122C426C206C6AA8401446317C2
:101350009400B24022449244410182800504130566
:10136000803E420497000000E78000FD4180C5B741
:101370009305000273A04580824573901534924016
:101380002242B2424243D2436244F2440255925551
:101390002256B2564257D2576258F25806499649D9
:1013A000264AB64A464BD64B664CF64C065D965DD1
:1013B000265EB65E465FD65F09617300203041113C
:1013C000B7170040985F3AC6945F3247E39CE6FE49
:1013D000324541018280B71700401307000323887C
:1013E000E702854717170000232AF74873002030CB
:1013F000411122C42D6426C24AC006C637190040D6
:101400001304A4AAB704002023208900976000E0F9
:10141000E780005B9C408297976000E0E780405A3D
:10142000E5B737370040834747009146BD8B639E41
:10143000D702B73600401306F00F973500009385AA
:10144000E51F9737000083D7672F03C7A6001377E0
:10145000F70F1DE3B7E70400BC4F09468945171590
:1014600000000345A5F8829731A099466394D70000
:10147000834757007300203003C786001377F70FA8
:10148000E365F6FC13851700AE97173800002317A5
:10149000A82A2380E70075B7B787004003C7670015
:1014A000098B6309071003C77700930600031377BE
:1014B0000703630DD708173800000348F87717367D
:1014C0000000130666740547B30606012380E60094
:1014D00083C577001737000013070775429793F508
:1014E000F50F2300B70003C58700973500009385EB
:1014F000A572C2951375F50F2380A5000347070059
:1015000089451377F703630CB70C63E7E50A6306B5
:10151000071A8545630CB7129737000083C7D77148
:101520003307F600034707001377F70F19CB85073A
:1015300093F7F70F3D476363F71A17370000A30DC2
:10154000F76EB787004009472383E700B78700405D
:1015500083C77700E207E18763DE0704973700005F
:1015600083C7976D173700001307076A3E978546B4
:101570002300D700173700001307076B3E97930629
:1015800000032300D700173700001307E7683E97D2
:10159000A14685072300D70093F7F70F3D47636403
:1015A000F71417370000A309F768B7870040094709
:1015B0002383E70073002030930610026300D70EE8
:1015C000930620026305D70693060002E316D7F4BC
:1015D00003C727021377C70F13672700D5A803C7D0
:1015E00067001377070465CB03C7A702173800000D
:1015F00013080843173500001305453A1347070839
:101600002385E70203C7A7021377370F1367870005
:101610002385E702814713070004B305F5008C41D9
:10162000B306F80091078CC2E399E7FEF5B503C74E
:10163000A702134707042385E70203C7A70213770E
:10164000C70F136727002385E702F9B503C76700B3
:101650001377070449C303C767021738000013084C
:10166000E82F1735000013052527134707082383A4
:10167000E70203C767021377370F136787002383D7
:10168000E702814713070004B305F5008C41B30658
:10169000F80091078CC2E399E7FEBDBD03C767025E
:1016A000134707042383E70203C767021377C70FB3
:1016B000136727002383E70285B503C76700137705
:1016C000070411CB03C727021377370F136787006F
:1016D0002381E70291B5238006003DBD97370000C6
:1016E000A38C0754B9BD97370000A387075475BD75
:1016F0002303048015472303E48001002302A48010
:10170000828083076480E3CE07FE23030480828007
:1017100083076480E3CE07FE03454480828083070D
:101720006480E3CE07FE2302A4808280411126C498
:101730004AC24EC006C61377F50BAD47AA892E895B
:101740009544630CF700194597000000E78080FA84
:1017500097000000E78020FB8D444E859700000035
:10176000E78040F9FD59FD1463983401B240A2446A
:101770001249824941018280135509011375F50F01
:1017800097000000E780E0F92209F1BF011126CCA3
:1017900006CEB704080097000000E780C0F61545A4
:1017A00097000000E78000F597000000E78080F6D2
:1017B00097000000E78000F62AC697000000E78047
:1017C00080F432459377150089EB13651500137586
:1017D000F50FF240E24405618280FD14E9F0014515
:1017E000CDBF397126DC4ADA4ED852D656D45AD2F9
:1017F0005ED006DE62CE66CCB7E700E07D5783AAF6
:10180000070022C603AA470023A0E71823A2E7186F
:10181000B7170040130770052380E704130780FA09
:101820002380E70483C74704930B75FFB684E20760
:1018300093FBFB0F8546AA892E8B32893724004003
:10184000E187015763FA76016308D50089461307DB
:1018500000026313D5000157D98F93F7F70FB71C18
:1018600000402382FC0411472303E4801305F00F9A
:1018700097000000E78000E8094C97000000E7802F
:1018800080E863657C15B7050700DA9537870700A0
:10189000795563FEE504B3879500636AF704370B57
:1018A0000800A94733EB65016395F90881E8814495
:1018B00097000000E78020E5268515A8DA85094510
:1018C00097000000E780C0E605090345F9FFFD1415
:1018D000050B97000000E780C0E481C49377FB0FFD
:1018E000E5F797000000E780A0EA69F17D55B7179A
:1018F0000040130770052380E704130780FA238054
:10190000E70403C74704418B2382E704F250B7E79B
:1019100000E023A0571123A24711E2543244525948
:10192000C259325AA25A125B825B724CE24C21615C
:101930008280A547639BF90685691309F00FB306FA
:101940009900B3742B01B6941349F9FFB37499004D
:10195000856B33796901416B9387F9FFB3F72701F1
:1019600099E363FC340193D94900C147E3E637FFAB
:101970003DBF0569C1697D19D9B71305800D63881D
:101980006901130500026384790113051008CA85F3
:1019900097000000E780C0D997000000E78040DF93
:1019A00031D54E99B38434416DBFDA852D4597000A
:1019B0000000E780E0D7CA94E30B99EE0509970091
:1019C0000000E78020D5A30FA9FEFDB79387F9FF9C
:1019D00093F7F70F636DFC0C83C71C0413073008E3
:1019E0006315F706370708006361EB06B3079B0032
:1019F000B706100063FBD704334BEB0089476399AC
:101A0000F9068980D549E38404EADA850945970017
:101A10000000E780E0D111090327C9FF9147232087
:101A2000E48003076480E34E07FE23033481FD173F
:101A3000EDFBFD14110B81C49377FB0FE9FF9700B9
:101A40000000E780E0D461F155B5B717004003C747
:101A50005704B70708001377070219E3B787070091
:101A60007955E376FBE833079B00E3F9E7F841B5E6
:101A70008547E380F9F0DA852D4597000000E7807F
:101A800020CB9389F4FFE38404E297000000E78011
:101A900060C893F7390091EB83260480032709007F
:101AA00093074900E396E6E03E89CE84D9BFB54767
:101AB0006399F9001305900B97000000E78080C33D
:101AC000FDB3B1471305B00AE388F9FE9947639760
:101AD000F904B7050800B365BB002D459700000069
:101AE000E78000C581448D4BA14997000000E78045
:101AF00060C263967401832704802320F900850463
:101B0000E39534FF8327048013172B0163550700E7
:101B10002312F90069BB2322F90051BB9D47639F43
:101B2000F90281451305B00497000000E78040C02A
:101B3000BD442320090023220900FD59970000001D
:101B4000E78040BD93F77400CA9703C70700FD14F0
:101B5000398D2380A700E39334FF91BBA14763979E
:101B6000F90697000000E780A0C28144630D0B00D6
:101B70008D479304C0036308FB00930400056304CE
:101B80008B01930440041375C507E30295D21945F0
:101B900097000000E78000B697000000E780A0B63D
:101BA000054597000000E780E0B426859700000017
:101BB000E78020B7094597000000E78080B69700CE
:101BC0000000E780E0BCE31405CE0DB39147639FAE
:101BD000F9001305600697000000E780A0B19700A8
:101BE0000000E78040B213059009F9B5E38109CC04
:101BF000F1547DB9BD660147173600001306462132
:101C0000938606A685458347060093F7F70F91C391
:101C100082800507E3F9E6FE97370000238AB71EA6
:101C2000DDB77D166206618693178601E18763D46E
:101C3000070001458280931726003307F500AE9711
:101C400018439C4363E7E7007D16E37FF7FC7D556F
:101C5000828005458280FD15E205E18513978501A7
:101C6000618793F7F50F63480700FD15139725006B
:101C70002A97584365D713851700620561858280CE
:101C80003308B5021C4283A80600B335B502C297DB
:101C900033B50701AE98469585486367B5006394F0
:101CA000A50063E3070181480C43C6950CC388C2B5
:101CB0001CC2828081471397870161876343B70005
:101CC0008280139727002A97232007008507E5B70E
:101CD0008147014793968701E18663C5B6001335B6
:101CE0001700828093962700AA9694428507558F05
:101CF000D5B793D755408A07AA979C430545331516
:101D0000B5007D8D828017F3FFDFE702833D2A84D3
:101D100097000000E78060F405C5931725003E9406
:101D20000327C4FF814711EB7D1516053E9542053B
:101D3000418517F3FFDF6700033D05838507E5B79E
:101D40000145C5BF81471397870161876343C7007A
:101D5000828013972700B386E50094422A9785076F
:101D600014C3D5B77D1662066186014793178601B5
:101D7000E18763D50700133517008280931726008B
:101D8000B306F500AE9794429C437D16B58F5D8FE8
:101D9000F1BF8A05AA9501476363B500828083A6D7
:101DA000C5FFF11593D71600D98F9CC11397F60183
:101DB000E5B72A830148014701456343D700828084
:101DC000B387050183A80700B30706019C43C697A4
:101DD000AA976384F80033B517010507B308030118
:101DE000620723A0F80061871108C1BF2A83014759
:101DF0008147014563C3D70082803388E50083288B
:101E00000800330EE600032E0E003388A840330886
:101E1000C8416384080133B508018507B308E300AE
:101E2000E20723A00801E1871107E9B717F3FFDFF5
:101E3000E702232B0111B286B2842E86AA850A8579
:101E400097000000E780C0FA2A84A6850A859700DB
:101E50000000E78020E833348000060413351500C5
:101E6000018D056117F3FFDF6700E32917F3FFDF3B
:101E7000E702A3244111AA89AE8A328BB68402C23A
:101E800002C402C60144131C8401135C8C416349E3
:101E90009C02939B1400FD1B0549138CF4FFF15C1D
:101EA00033048901620461846340740792478E049D
:101EB000CE9423AEF4FE410117F3FFDF67006323E6
:101EC00013192400B30B2B01014A93172A00D6974C
:101ED00083A50B0088437800340050009700000071
:101EE000E78040DA050A93178A01E187F11BE35E78
:101EF000FCFC92474E9905042320F900A2473EC2FC
:101F0000B24702C63EC441B7131A8901135A8A4127
:101F1000131D240093178A01E18763CF970092472E
:101F20000A044E941CC0A24705091379F90F3EC25A
:101F3000B24702C63EC4ADB7B3079A0313152A00D1
:101F400056950841780034005000050AEA97DA9760
:101F50008C4397000000E780E0D26DBF197106C284
:101F600012C416C61AC81ECA22CC26CE2AD02ED219
:101F700032D436D63AD83EDA42DC46DECAC0CEC2C9
:101F8000D2C4D6C6DAC8DECAE2CCE6CEEAD0EED2F9
:101F9000F2D4F6D6FAD8FEDA971500009385858D2F
:101FA0008841E700050092402242B2424243D243B8
:101FB0006244F244025592552256B2564257D257C5
:101FC0006258F25806499649264AB64A464BD64BBD
:101FD000664CF64C065D965D265EB65E465FD65F45
:101FE0000961730020300000972100209381810156
:101FF000175100201301018117F5FFFF1305C500DC
:102000009705002093850500171600201306C6FDCE
:1020100063FAC5008322050023A055001105910530
:10202000E3EAC5FE17050200130585279715002072
:102030009385C5FB171600201306466763FAC50093
:102040008322050023A0550011059105E3EAC5FE92
:1020500017150020130585659745002093850527F2
:102060006377B500232005001105E36DB5FEFD4241
:10207000739002BC8D4273904280B722000093821D
:10208000828873900230970200209382A2F793E235
:102090003200739052309752000093826296739090
:1020A00012346FB0F47573002030397101436EC67D
:1020B00019A0397141536AC866CA62CC5ECE19A0B4
:1020C000397101535AD056D252D44ED64AD826DA54
:1020D00022DC06DE33016140828241114AC026C201
:1020E00022C406C68282B24D4101024D924C224C5E
:1020F000B24B4101024B924A224AB2494101024984
:1021000092442244B240410182803D432A87637356
:10211000C3029377F700BDEFADE5937606FF3D8AE6
:10212000BA960CC34CC30CC74CC74107E36BD7FE30
:1021300011E28280B306C3408A0697020000969699
:102140006780A6002307B700A306B7002306B700E1
:10215000A305B7002305B700A304B7002304B70005
:10216000A303B7002303B700A302B7002302B700FD
:10217000A301B7002301B700A300B7002300B700F5
:10218000828093F5F50F93968500D58D9396050182
:10219000D58D61B7939627009702000096968682A8
:1021A000E78086FA9680C1171D8F3E96E374C3F8C8
:1021B000A5B73367B500FD530D8B79E7B7877F7FF0
:1021C0009387F7F710419441B372F6003363F6003A
:1021D000BE92B3E262006397720C6318D606504158
:1021E000D441B372F6003363F600BE92B3E26200EC
:1021F0006398720A631BD60410459445B372F600C7
:102200003363F600BE92B3E262006391720A631E0A
:10221000D6025045D445B372F6003363F600BE9241
:10222000B3E26200639A72086311D60210499449BE
:10223000B372F6003363F600BE92B3E262006393BA
:1022400072085105D105E30FD6F6131706019397CF
:102250000601631CF7001357060193D706013305E7
:10226000F7409375F50F91E982804183C18333056F
:10227000F7409375F50F91E182801377F70F93F78D
:10228000F70F3305F74082800346050083C605003B
:10229000050585056313D60065FA3305D6408280AF
:1022A00011059105E312D6FE014582802105A105A5
:1022B000E31CD6FC014582803105B105E316D6FC4E
:1022C000014582804105C105E310D6FC01458280AD
:1022D000B717004003C777051377E70FA38BE70411
:1022E000130700F8A38DE7043D47238CE704130789
:1022F0005003A38CE70403C7A7051377D70F238DDB
:10230000E7048280B717004003C7E7020D89411137
:102310001377C70F498F93068008F3B6068093F6AC
:10232000860836C601000100930670052380D70495
:10233000930680FA2380D704010001002387E70277
:1023400023800704B247F3A7078001000100410181
:10235000828041112A83014E930E407E130F001993
:10236000930F400663E56E129308001913034006AD
:10237000B3781503854E0D4FA14F337365020D8958
:102380001335150063EFBE121308F6FF79467298F5
:102390004208135808013307C70213D61700BE07B7
:1023A00032976146B3F6C60213068070B386C60242
:1023B0003697A166F58F42075D8FB716004083C739
:1023C000F60293F70708A303F1000346710083C7E1
:1023D000F60293F70708E394C7FE83477100B71628
:1023E000004093F7F70F6388071293078008F3B74D
:1023F000078093F787083EC401000100B71700402B
:10240000930670052380D704930680FA2380D704AF
:102410000100010023AA070383C6170393E60608F9
:10242000A388D70223800704A247F3A707800100EF
:1024300001001166B71700407D16D45BC85F938515
:102440004703A98EF18EF5FA93068008F3B606804D
:1024500093F6860836C601000100930670052380B6
:10246000D704930680FA2380D7040100010098C1A5
:1024700003C7170313670704A388E7022380070431
:10248000B247F3A7078001000100410182807D135C
:102490003368E3039308E016630E08003368F30320
:1024A0009308D016630808009378330093B8180097
:1024B0009388D81633081E01131E0801135E0E01FF
:1024C00055B56393E5030548638608000148630337
:1024D00003002A8871087298FD15131E0801C205B1
:1024E000135E0E01C18179BD13F8150063F4BF00BE
:1024F0007908D5B713381800E5BF83C7F60293F7FC
:102500000708A303F1000346710083C7F60293F79F
:102510000708E394C7FE8347710093F7F70FF1DFD5
:10252000E9B531714AD966CB06DF22DD26DB4ED70D
:1025300052D556D35AD15ECF62CD6AC96EC7AA8C26
:1025400002D897100000E78020B12A8993078008FD
:10255000F3B7078093F787083EDA01000100B71749
:102560000040130770052380E704130780FA2380D7
:10257000E7040100010003C7F7021377770FA38771
:10258000E70203C7F70213678700A387E7022380E8
:102590000704D257F3A70780010001000545970003
:1025A0000000E78060D6130780C13347E902116A53
:1025B00093070AE893065002BD69930BA004814A71
:1025C000014B13048008930470057D1AB347F90288
:1025D0003307D7023EC0FD873ECC938709A69309F7
:1025E000803E3347F7023AC27D873AC43347390306
:1025F0008549B399990193D93940B306D702B30BF2
:102600007703B3C6F602B3CBFB0236C6FD8636C8E7
:1026100093D6FB4136CEB7460F0093860624334946
:10262000D9028566938606FAB3969601B389E902C4
:10263000130760553309D90293060010B389E902E4
:102640003349D902B3C9F9029316390036CA37198A
:102650000040FD8636D0930D090493D7F9413ED250
:10266000F336048093F6860836DC010001009307F8
:1026700070052380FD00930680FA2380DD000100B1
:1026800001008346390593F6860FA309D9048346D2
:10269000390593E61600A309D90423800D00E256FC
:1026A000F3A6068001000100130C80FA116DF336C9
:1026B000048093F6860836DE01000100930770055A
:1026C0002380FD0023808D01010001008346390530
:1026D000216693E60602A309D90483560905B3E6E9
:1026E000A6012318D90483560905D18E2318D904CD
:1026F00023800D00F256F3A60680010001008346F8
:10270000390593F606026381061A03463905218AC4
:102710006DDE081897100000E7800098733604807B
:1027200013768608B2C20100010023809D00238039
:102730008D0101000100B717004003C6370513766D
:10274000F60DA389C70403C6370513660602A389DD
:10275000C704835609052166B3E6A6012318D904E8
:1027600083560905D18E2318D90423800D0096467F
:10277000F3A60680010001008346390593F60602A0
:10278000638B061483463905A18AEDFE970000206D
:10279000E7806090AA8636D497000020E780A08F5B
:1027A000A256E30AD5FE835609054255B3E6A601B3
:1027B0002318D90497100000E780C08F834639059D
:1027C000A18AEDDE03560905834629058247337643
:1027D000CA00B306DA0293D5F641B296B388F64042
:1027E000E24733B8C6002E983308F840A247B3B684
:1027F00016013308D84063C70701631DF8009247EC
:1028000063FA1701C247634FF80E63950701B24799
:1028100063EAF80E894663E9660FF24693151800DD
:1028200013D3F8015E8613951800B365B30042D642
:1028300046D497C00100E78080003258050B137B17
:10284000FB0F63470001631A0838A25863870838F2
:1028500013081500B336A800B69513D6F5013298C3
:10286000B336C800AE9613581800FE06B3E606014C
:102870007336048013768608B2C6010001002380F7
:102880009D0023808D01010001000356C902B2960C
:10289000C206C1822316D90223800D00B646F3A6D4
:1028A00006800100010021B5F336048093F6860806
:1028B000B6C00100010023809D0023808D0101002E
:1028C00001008346390593E60602A309D904238053
:1028D0000D0086460DB5F336048093F68608B6C41F
:1028E0000100010023809D0023808D010100010073
:1028F0008346390593E60602A309D90423800D0017
:10290000A646BDB5E30B0BF0F336048093F68608BC
:10291000B6C801000100930680FA23809D00238041
:10292000DD00010001008346390593F5FC0F93F6A5
:10293000860FA309D90483463905CD8EA309D9048E
:1029400023800D00C646F3A6068001000100130592
:1029500080FA03463905930639051D8A631C9629BA
:102960007336048013768608B2CC0100010013068A
:1029700080FA23809D002380CD000100010003C662
:1029800006001376F60D2380C60003C60600136604
:1029900006022380C600835609051166D18E2318CE
:1029A000D904835609052166D18E2318D9042380C2
:1029B0000D00E646F3A6068001000100130680FA2A
:1029C0008346390593F60602638006268346390559
:1029D000130C3905A18AFDDA081897000000E7807A
:1029E000A06BF336048093F68608B6D00100010090
:1029F000930680FA23809D002380DD000100010002
:102A000083460C00116693F6F60D2300DC00834626
:102A10000C0093E606022300DC0083560905D18EE4
:102A20002318D904835609052166D18E2318D904A9
:102A300023800D008656F3A60680010001001306D0
:102A400080FA8346390593F60602638A0620834698
:102A50003905A18AEDFE97F0FF1FE780C0632A8C3D
:102A600097F0FF1FE7802063E30C85FF835609057D
:102A700011664255D18E2318D90497000000E780D3
:102A800060638346390513063905A18AFDDAF336FA
:102A9000048093F68608B6D401000100930680FAFC
:102AA00023809D002380DD00010001008346060095
:102AB00093F6F60D2300D60023800D00A656F3A64C
:102AC0000680010001008356090503462905D24707
:102AD000B376DA003306CA021305800C9355F6412B
:102AE0003696330DF6408257333CD6002E9C333653
:102AF000A601330CFC40330CCC40330885039256BE
:102B00004E86B335A5033305A503C29597C00100D2
:102B1000E780E0D263468001631E0C16630C0D163D
:102B2000130615003335A6002E959356F5013696FB
:102B3000B335D600AA959396F50105828585D18E89
:102B40006346B000639D051A638B061A0356C902DB
:102B500015823305D6003336C500B2956348B00000
:102B6000639105241306F00F637DA622894663F363
:102B7000561593078008F3B7078093F78708BED6EA
:102B80000100010037170040930770052300F70488
:102B9000930780FA2300F704010001008356C7025F
:102BA00089678117D58FC207C1832316F7022300D7
:102BB0000704B657F3A7078001000100FA506A54D2
:102BC000DA544A59BA592A5A9A5A0A5BFA4B6A4C49
:102BD000DA4C4A4DBA4D296182801308F5FF33352E
:102BE000A800FD152E951356F5013298B336C8008E
:102BF000AA9695B9F336048093F68608B6CA010002
:102C0000010023809D002380AD0001000100834668
:102C10003905CD8EA309D90423800D00D646F3A62D
:102C200006800100010035B3F336048093F6860870
:102C3000B6CE0100010023809D002380CD0001005D
:102C400001008346390593E60602A309D9042380CF
:102C50000D00F646F3A606800100010095B3F33699
:102C6000048093F68608B6D20100010023809D00FF
:102C70002380CD00010001008346390593E606025A
:102C8000A309D90423800D009656F3A606800100FF
:102C9000010045BB9306F5FF33B5A600FD152E9543
:102CA0009355F501AE96B3B5B600AA951396F50106
:102CB000858269B5F336048093F68608B6D801009C
:102CC0000100930680FA23809D002380DD0001002F
:102CD00001008356C9020566011693F6F60FD18EE0
:102CE000C206C1822316D90223800D00C656F3A660
:102CF000068001000100850A93FAFA0F95B233E6C7
:102D0000B60045C20356C9023305D0403338A0008F
:102D1000B305B040B385054115826345B000D1E1EC
:102D20006371A608894663F0560593078008F3B7D8
:102D3000078093F78708BEDA01000100B71700404B
:102D4000130770052380E704130780FA2380E70444
:102D50000100010003D7C7027D8B2396E702238081
:102D60000704D65781BDF336048093F68608B6DC97
:102D700001000100930680FA23809D002380DD007E
:102D8000010001008356C9020566011693F6F60F8D
:102D9000D18EC206C1822316D90223800D00E656C9
:102DA000B9B793078008F3B7078093F78708BEDEAB
:102DB0000100010037170040930770052300F70456
:102DC000930780FA2300F704010001000356C702AD
:102DD00093975600B297C207C1832316F7022300C8
:102DE0000704F657C1BB914763EEB70217D701003E
:102DF000130747428A05BA959C41BA978287B7174D
:102E0000004003A7470B1345F5FF698F23AAE70A84
:102E100003A7070B698F23A8E70A03A7070A798D81
:102E200023A0A70A8280B717004083A6470B134749
:102E3000F5FFF98E23AAD70A83A6070B558D23A881
:102E4000A70A83A6070A758F23A0E70A8280B7170F
:102E5000004003A7470B498F23AAE70A03A7070BE4
:102E60001345F5FF45BFB717004083A6470B13472F
:102E7000F5FF758F23AAE70A03A7070A598D4DB7F7
:102E8000B717004003A7470B498FEDB7914763EE93
:102E9000B70217D70100130727398A05BA959C4155
:102EA000BA978287B717004003A7470D1345F5FF70
:102EB000698F23AAE70C03A7070D698F23A8E70CE6
:102EC00003A7070C798D23A0A70C8280B7170040B9
:102ED00083A6470D1347F5FFF98E23AAD70C83A6C7
:102EE000070D558D23A8A70C83A6070C758F23A06B
:102EF000E70C8280B717004003A7470D498F23AA2C
:102F0000E70C03A7070D1345F5FF45BFB7170040B2
:102F100083A6470D1347F5FF758F23AAE70C03A778
:102F2000070C598D4DB7B717004003A7470D498FC0
:102F3000EDB7797122D43714004026D24AD0035914
:102F400024028354040206D64209C2044ECE52CC57
:102F500056CA13590901C1802DE11379F9F793F489
:102F6000F49F4209C20413590901C18093078008E4
:102F7000F3B7078093F787083EC401000100930769
:102F800070052300F404930780FA2300F404010081
:102F90000100231124032310940223000404A247F8
:102FA000F3A7078001000100B25022549254025945
:102FB000F249624AD24A45618280B7F507008146EC
:102FC0003000B105194597000020E7808081A247B5
:102FD00013972701E34A07FC1369090893E40440A7
:102FE00093098008F3B7098093F787083EC0010072
:102FF0000100930A700523005405130A80FA230088
:10300000440501000100231124032310940223002E
:1030100004048247F3A7078001000100294597F0C7
:10302000FF1FE7802031F3B9098093F989084EC268
:1030300001000100230054052300440501000100A4
:103040008357040293E707202310F40223000404AB
:103050009247B9B7B7170040884742054181937737
:10306000050491EB9377F5013755E80113050580C9
:103070003345F50282809377050C130700046397AC
:10308000E7009377F50137459C1CCDB72165130503
:1030900005D0828037E700E01C435443A183E20659
:1030A000D58F1CC1FD572320F7182322F7188280E3
:1030B00013178500B7E700E023A0E710618123A282
:1030C000A7108280B7F700E08847CC47828081470D
:1030D00037370040A14663C4C7003285828003456C
:1030E000B740E38EA6FE3385F5000345050085074E
:1030F0002304A740CDB797070020938727EF9C4371
:10310000173700201307871C3E95636EE5001737BD
:1031100000201307274F6368A70017070020232705
:10312000A7EC3E858280FD57EDBF8280411122C40D
:1031300006C62A8497000000E78000F22947B307FB
:10314000E502B2408D83B3D7870222449507B3D7F7
:10315000E70237370040C207C1832316F700410159
:103160008280411137150E0006C697000000E780E7
:1031700020FCB7370040130770F82381E7000D47A4
:10318000A381E70013070004A380E7000547238716
:10319000E700B24041018280373700408347270073
:1031A0001A0593F7F703C98F93F7F70F2301F70079
:1031B0008280B737004003C7170019C9D98DA38093
:1031C000B70003C70700136787002380E7008280EA
:1031D00093C5F5FFF98DA380B7008280AE872A875B
:1031E000B736004021463738004089E71703000012
:1031F0006700E3F383C8B600E30916FF05078348B9
:10320000F7FFFD17C20723041801C183F9BF41115D
:1032100022C406C62A8497000000E780E0E329471D
:10322000B307E502B2408D83B3D7870222449507E6
:10323000B3D7E70237370040C207C1832316F740F0
:1032400041018280716541111305052006C6970072
:103250000000E78000FCB7370040130770F82381B7
:10326000E7400D47A381E74013070004A380E74030
:1032700005472387E740B24041018280CC4141119C
:1032800006C6328503C6150083C5050022064D8E8D
:1032900042068D654186138875A2630C0611634B47
:1032A000C804138845A26300060D634AC8009385CD
:1032B00035A26301B6082390060029464DA0138865
:1032C00055A26305060D938565A2E316B6FE8D45EE
:1032D0001D4663E6E5081146198E63F3C7003E8676
:1032E000B7E704002390C600FC4797D501009385FB
:1032F000E5F59DA0138895A263030611634E060DA4
:103300001388A5A263000613938505A5E315B6FAF5
:1033100099451D4663E5E504198E63F3C7003E86B3
:10332000B7E704002390C600FC479705002093856B
:1033300025D61DA09D451D4663E3E5022146198E55
:1033400063F3C7003E86B7E70400FC472390C6003E
:103350009705002093850536BA9582970146B240BD
:10336000328541018280AD451D46E3EAE5FE3146E6
:10337000198E63F3C7003E86B7E704002390C600AA
:10338000FC4797D501009385E5EEF9B7B1451D4699
:10339000E3E7E5FC3546198E63F3C7003E86B7E7E1
:1033A00004002390C600FC4797D50100938585ED66
:1033B00065B78D451D46E3E4E5FA1146198E63F3C2
:1033C000C7003E86B7E704002390C600FC4797D5A8
:1033D0000100938565E849B78D451D46E3E1E5F8B1
:1033E0001146198E63F3C7003E86B7E704002390A9
:1033F000C600FC4797D50100938585EAB1BFA54576
:103400001D46E3EEE5F42946198E63F3C7003E86B8
:10341000B7E704002390C600FC4797D501009385C9
:1034200065E41DBFB5451D46E3EBE5F23946198E4F
:1034300063F3C7003E86B7E704002390C600FC474D
:1034400097D50100938585DF01BFB7E7040003A38B
:103450000713970600209386A6C24146A545170587
:1034600000201305E5B802832D455DE703C505007F
:103470000947631FE50803A84500411106C6034735
:10348000180032850346080022074168518F9308CF
:1034900028FE6307170563E9E800051863030703BF
:1034A00023900600294591A8130648FE630AC70425
:1034B0001518E31707FF15463E87637BF60015478F
:1034C00001A8130600023E876374F600130700028A
:1034D000B7E704002390E600FC471316070111A884
:1034E0003E8691C30546B7E70400FC472390C6001B
:1034F0004206CC45418282970145B240410182801B
:10350000130600083E87E375F6FC13070008C9B7E9
:103510002390060005458280828041677917630405
:10352000E504411122C406C685472A84639FF5003D
:10353000B7E7040022852244B24003A3871397050E
:103540000020938565314101028389476399F50025
:10355000B7E7040083A7070B8545829771D9B2406E
:103560002244410182808280797126D252CCAE847D
:103570002A8A97D501009385A5D417D50100130594
:10358000A5D606D63AC622D44AD0368432894ECE43
:1035900097B00100E780E075A28517D501001305FB
:1035A000A5D597B00100E780C074294597B0010008
:1035B000E780007983C7840093F70702F9E383C9A2
:1035C00004008947054532476396F908D44083C70C
:1035D000160083C60600A207D58FC166138616FEA5
:1035E000638CC7028D16638FD7068D6693862690EF
:1035F00029456391D706B7E70400A286225403A3A6
:103600004714B250F2494A86A6850259925452850F
:10361000624A8547456102832D450DEF93070002FD
:10362000354563E98702B7E70400FC47C844130641
:103630000002CA85829781499707002093878722D5
:103640009C43014581CB9C4391C74E852286CA8508
:1036500082970145B250225492540259F249624A6B
:10366000456182802D457DF79307700F3545E3E373
:1036700087FEB7E70400FC47C8442286CA858297C4
:1036800065BF2145C1BF411122C437E4040083272F
:10369000841326C2AA84416506C697050020938537
:1036A000A51B7D1582978327C40A17050000130503
:1036B00005E78588829795C0032304132244B2400E
:1036C000924497060020938626AE4146C5451705CD
:1036D00000201305659C41010283B24022449244BC
:1036E00001454101828019C59707002023ACA71628
:1036F00001458280454582801147636AA70A97D6B3
:1037000001009386A6BA0A0536951841411106C6EE
:103710003697AE87B2850287130700026145639D25
:10372000E700B7E70400FC47130600021705002076
:103730001305C5F882970145B240410182800547D3
:103740006145E39BE7FEB7E70400FC470546170524
:1037500000201305A5F8F9BF1307700F6145E39D1D
:10376000E7FCB7E70400FC471306700F17050020BD
:10377000130505F7C1B7130700086145E39EE7FA93
:10378000B7E70400FC4713060008170500201305DF
:10379000A5044DB715476145E390E7FAB7E7040084
:1037A000FC471546170500201305450B61B7094571
:1037B0008280411126C2B7E4040083A7C41322C447
:1037C0004AC006C62E84970500209385E5082A89FD
:1037D0008297058905C5970700209387E78B83D7D4
:1037E000A70BA28503A3440D2310F4002244B2408A
:1037F00092444A850249014641010283B240224473
:103800009244024949454101828097070020238D57
:1038100007049707002023AB0704B717004003A74E
:10382000070CB706C0FFFD16758F23A0E70C03A792
:10383000070DB7064000558F23A8E70C03A7070C18
:103840003D9B23A0E70C03A7070D1367070123A8DF
:10385000E70C8280B717004003A5470C83A7470CED
:10386000598113451500C18B058999E3136525001E
:103870009707002083C747FF6380A70297070020B0
:103880002384A7FE11C997070020938727FE03A36F
:1038900007006303030002838280114517F3FFFFD3
:1038A000670063C8011122CC06CE3714004026CA37
:1038B0004AC84EC652C483447405034AB4058349BA
:1038C00084050349940597F0FFFFE780A0A0834794
:1038D000A40593F4F40F137AFA0F93E71700230D5E
:1038E000F40493F9F90F1379F90FB717004003C7E0
:1038F000A705058B6DFF03D5C705A38D4705238C51
:103900003705A38C2705A38B9704F2406244D24469
:103910004249B249224A05618280411193970501CB
:1039200022C406C626C2C1872E8463DC0700B7E422
:103930000400FC54829719C1BC5482972165218DE3
:1039400015A893F7150013C515008DE793F725000B
:103950009DC797000000E78020F0B7E70400BC4F48
:103960001306000A8945170500200345A5F0829734
:1039700013452400B240224492444101828093972F
:10398000250163D80702B7E4040083A7C41E829709
:1039900097000000E780A0F0BC4C375607001306E4
:1039A00006308965170500200345C5EC8297096537
:1039B00079B7939715010145E3DE07FA17D50100A2
:1039C0001305859B97B00100E780804AB7E70400A4
:1039D000BC4F13060064916517050020034585E977
:1039E00082971165A9BF1D71A2CC37E404005C5C0D
:1039F000485886CE494697D50100938565938297AE
:103A000011E917D501001305E59397B00100E78090
:103A1000204601A0B7F600E0795798CAFD57DCCAE6
:103A20000567B7E700E023A0E7101306F00290C295
:103A300023A0E718010001003707002018471306EC
:103A4000000481459706002023A4E6E24157A38A9B
:103A5000E7403C4408088297970700209387877DBA
:103A60003EC8856713870740938757D1231AE10023
:103A70002312F1021307B00F97F7FFFF9387C76474
:103A80002310E1023ED81547970700009387C7E14E
:103A9000B7F50700A30FE1003EDC054797070000DC
:103AA0009387E7DF81463000E10519452301E102F4
:103AB0003EDE97F0FF1FE780C0D218088147994685
:103AC00030003E960346060085070507A30BC70096
:103AD000E398D7FEC24791C70357410185676373D7
:103AE000F70001A0B7E7040083A7470A08088297F8
:103AF000AA8511C917D501001305058697B00100E5
:103B0000E780201F01A0F6406644256182804111B4
:103B100026C2B7E4040083A7040806C622C417051A
:103B200000001305C5DF829717040020130484D416
:103B30002300A40097000000E780800297000000A7
:103B4000E780E0CC03450400224403A38405B2408F
:103B5000924413060032896541010283797106D6C9
:103B600022D413078008F337078093F787083EC2F3
:103B700001000100B7170040930570052380B704CA
:103B8000130680FA2380C7040100010083C6F702F0
:103B900093F6A60FA387D702238007049246F3A6C5
:103BA00006800100010073370780137787083AC445
:103BB000010001002380B7042380C7040100010035
:103BC00003C7F70213672700A387E70223800704D0
:103BD000A247F3A7078001000100054597E0FFFF1A
:103BE000E780807297000000E78060CB0147814644
:103BF0008147054685451305407E97E0FFFFE78036
:103C0000807537E404003C44680051468145829742
:103C1000B707C0A83EC8B787E803938707D03ECA56
:103C200097E7FF1F9387A7793EC67C586800829765
:103C3000B250225445618280411197D5010093858D
:103C4000E5D517C501001305256A06C697B0010022
:103C5000E780200A17D501001305C5EE97B00100D3
:103C6000E7802009B2402945410117B301006700F0
:103C7000230D411197D50100938585D317C5010008
:103C80001305856606C697B00100E780800617D544
:103C900001001305E5E997B00100E7808005B24017
:103CA0002945410117B3010067008309411122C46E
:103CB00006C6834705002A849DC797D501009385D2
:103CC000A5D617C501001305256297B00100E7804E
:103CD00040024C4017D50100130545FB97B0010089
:103CE000E78020013DA058410DEF97D50100938555
:103CF000A5D317C501001305255F97B00100E78024
:103D000040FF17D501001305E5F997B00100E780E2
:103D100040FE2244B2402945410117B3010067002B
:103D20002302A1679386D7036313D70297D50100B7
:103D3000938585CF17C501001305055B97B001007A
:103D4000E78020FB17D501001305C5F67DBFED0701
:103D500097D50100938545CD17C501001305C558BA
:103D6000631BF70097B00100E780A0F817D50100AA
:103D7000130585F559BF97B00100E78080F74C40E7
:103D800017D50100130545F691BF411106C622C49F
:103D9000970700209387472F054717240020130417
:103DA000C4992392A7002390B7002391E700231022
:103DB000B40017C501001305255397D5010093855D
:103DC000E5C1972700202387E78697B00100E780A9
:103DD00040F28355040017D501001305A5F797B0ED
:103DE0000100E78000F12244B2402945410117B3A8
:103DF00001006700E3F4411197D50100938585BC6C
:103E000017C501001305454E06C697B00100E780AF
:103E100040EEB2402945410117B30100670043F26B
:103E2000797122D426D24AD02E842A898145B2843F
:103E30004800714606D697E0FFFFE780402D97F7D0
:103E4000FF1F93876758DC4783D70700231421019E
:103E50002313F10097500000E78040048547A30535
:103E6000F1009307401F3EC6FD572305A100230A1A
:103E7000F10097500000E780A0162686A285480032
:103E800097500000E7806004B250225492540259C7
:103E900045618280972700202391078A9717002089
:103EA000238A0778B7E70400FC47411106C641465C
:103EB00097D501009385C5E417F5FF1F1305054E3F
:103EC000829717070020034767279307F00A6315B7
:103ED000F7029307F0F8894517050020130505261A
:103EE00017070020230CF72497070020A388072436
:103EF00097600000E78000C097600000E78060EBFB
:103F00008145370504009707002023AF0720970756
:103F10000020239907209707002023860720970772
:103F2000002023950718970700202393071697076B
:103F300000202398071E970700202399071E97301B
:103F40000000E780E048014597600000E78080C3FB
:103F500097D50100938585A917C501001305C538BC
:103F600097B00100E780E0D817D50100130505E000
:103F700097B00100E780E0D7B2402945410117B36F
:103F800001006700E3DB4111054506C6978001008B
:103F9000E78040B529E58545814617F6FF1F1306E2
:103FA000E63E97C00000E780804697D501009385E4
:103FB000A5A42DC917C501001305053397B001004D
:103FC000E78020D317D50100130545C897B001003D
:103FD000E78020D2294597B00100E78060D697F7A7
:103FE000FF1F9387673EDC47054797D50100938500
:103FF000A5A02390E70017C501001305E52E97B093
:104000000100E78000CF17D501001305A5C697B0C2
:104010000100E78000CEB2402945410117B30100FD
:10402000670003D217C501001305052C97B00100E6
:10403000E78020CC17D50100130585C241BF0111CF
:1040400022CC06CE26CA4AC84EC693F715002E8447
:10405000BDC3930710F8170700202301F70E970739
:10406000002083D767029145170500201305050D31
:1040700017070020A304F70CA183170700202300D3
:10408000F70C97070020A38C070A97600000E780D1
:1040900060A697200000E78080300545976000000B
:1040A000E78040AE13451400F2406244D2444249D6
:1040B000B2490561828093F72500E9CF17070020F8
:1040C0000357470669C7AD64B71900409384A4AA93
:1040D00023A099009706002093860605944297D75F
:1040E0000100938727CB170600200346C6038145AE
:1040F00017F5FF1F1305852A97700000E780C04F52
:1041000023A0990097F7FF1F239CA71A2A8941C172
:1041100097D501009385C59617C501001305C51CE9
:1041200097B00100E780E0BCCA8517C50100130500
:10413000653397B00100E780C0BB294597B0010007
:10414000E78000C097070020239E07FC930710F824
:10415000170700202304F7FE9707002083D7C7F234
:1041600017070020A30CF7FCA183170700202308E2
:10417000F7FC91458D4717050020130525FC17070F
:104180000020A30EF7FA97600000E780A096134581
:10419000240019BF93F7051095C3AD67371700408A
:1041A0009387A7AA17F5FF1F035525241CC3972043
:1041B0000000E780E04913450410FDB593F70520A2
:1041C00091CFAD67371700409387A7AA1CC39720EC
:1041D0000000E780C02713450420F9B593F7450098
:1041E000D1C397D501009385A58917C50100130593
:1041F000A50F97B00100E780C0AF17C501001305F8
:10420000252897B00100E780C0AE294597B001008E
:10421000E78000B3930720F8170700202300F7F288
:104220009707002083D787E817070020A308F7F037
:10423000A183170700202304F7F085471707002004
:10424000A30FF7EE97500000E78080D917050020F4
:104250001305C5EE914597600000E780A0891345DE
:10426000440099B593F78500A9C797D501009385B8
:10427000258117C501001305250797B00100E780C8
:1042800040A717C501001305E52097B00100E7809E
:1042900040A6294597B00100E78080AA9707002033
:1042A000239207E897700000E780E04413458400FC
:1042B000E5BB93F70501D1C38545170500200355DC
:1042C000E5DE97600100E780C0F797C501009385A0
:1042D000257B17C501001305250197B00100E78074
:1042E00040A117C501001305251C97B00100E78008
:1042F00040A0294597B00100E78080A4930730F8DB
:1043000017070020230CF7E29707002083D707DA6E
:1043100017070020A304F7E217050020130505E2A4
:10432000A1838D4517070020230BF7E0975000006D
:10433000E780407C1345040185BB93F70502D1C794
:1043400097C501009385C57317C501001305C5F90D
:1043500097B00100E780E09917C501001305051724
:1043600097B00100E780E098294597B00100E78009
:10437000209D930740F8170700202301F7DC9707DB
:10438000002083D7E7D017070020A309F7DAA1831D
:10439000170700202305F7DA854717070020A30039
:1043A000F7DA97070020239507CE97500000E780A3
:1043B00020C317050020130565D8914597500000CC
:1043C000E780407313450402C5B193F70504FDC3AC
:1043D00097C501009385C56A17C501001305C5F08F
:1043E00097B00100E780E09017C501001305850F25
:1043F00097B00100E780E08F294597B00100E78082
:1044000020949707002083C767D31307700A638639
:10441000E7061307800A638CE7081307600A6393B3
:10442000E704930760F8170700202309F7D09707E0
:10443000002083D707CF17070020A301F7D0A1835F
:1044400017070020230DF7CE854717070020A30C80
:10445000F7CEB14517050020130545CE9750000053
:10446000E780406997500000E78080B71345040457
:1044700097070020239707CA05B9930770F8170715
:104480000020230DF7CA9707002083D787C9170795
:104490000020A305F7CAA183170700202301F7CA4C
:1044A000854717070020A30DF7C8994565B79307FF
:1044B00080F8F1B793F705080145E38707BE97C574
:1044C00001009385E55B17C501001305E5E197B091
:1044D0000100E780008217C501001305250297B08F
:1044E0000100E7800081294597B00100E780408501
:1044F0009307A0F8170700202302F7C497070020AE
:1045000083D7C7C217070020A30AF7C2A1831707E2
:1045100000202306F7C2854717070020A301F7C232
:1045200097070020239407C097500000E78040AB16
:1045300017050020130585C0914597500000E780BE
:10454000605B134504088DB6411122C497C5010074
:104550009385C54E2A8417C501001305E5D806C604
:1045600097A00100E780E0784C4017C501001305D3
:10457000656B97A00100E780C077294597A00100EF
:10458000E780007C034704009307F00F631FF702E6
:1045900097C501009385854A17C501001305C5D449
:1045A00097A00100E780E0744C4017C50100130597
:1045B000656897A00100E780C0732244B240294596
:1045C000410117A301006700A377B24022444101D3
:1045D0008280B1C1411122C417C501001305C5D0A5
:1045E0002E8497C501009385A53E06C697A00100BD
:1045F000E7802070A28517C501001305E57497A018
:104600000100E780006F2244B2402945410117A311
:1046100001006700E3728280B7E7040003A3870507
:10462000130600149305001017F5FF1F0345052519
:104630000283B7E7040003A387051306001493055C
:10464000002017F5FF1F034565230283011126CAC9
:10465000B7E40400DC5C06CE22CC4AC8354697C5D8
:1046600001009385654F17D5010013052529829711
:1046700011E917C501001305E5CC97A00100E780FB
:10468000207F01A097F7FF1F938707203EC4B7F54F
:104690000700856793870780814617F6FF1F13067B
:1046A000261EE10519453EC697E0FF1FE78060130F
:1046B000FC44194697F5FF1F9385851C17050020BC
:1046C0001305059F8297340017F6FF1F1306461B3C
:1046D00097D501009385859E17D501001305859F09
:1046E00097700000E78040C62A8429C197C5010061
:1046F0009385053817C50100130505BF97A0010074
:10470000E780205FA28517C501001305E54597A046
:104710000100E780005E294597A00100E780406224
:10472000F2406244D24442490561828097E0000031
:10473000E780202917C501001305053A976000009E
:10474000E78040BA97A00000E780607D9760010095
:10475000E780E0E117F5FF1F130585C297600100B0
:10476000E78080CA17C5010013050538976001006E
:10477000E78060E22A8497600000E780802097103D
:104780000100E780C0B997800100E780E052977090
:104790000000E780807997700000E780809697306E
:1047A0000100E780207B97C501009385652C17C524
:1047B0000100130565B319C897A00100E780605395
:1047C000A28517C501001305653C91B797A00100AC
:1047D000E780205217C501001305853D97A0010011
:1047E000E78020512D64371900401304A4AA2945FD
:1047F00097A00100E780C054232089009730010072
:10480000E78020562320890097F00000E780A074FD
:1048100055CD85453705040097300000E78040BB43
:1048200097C501009385C52417C501001305C5ABC5
:1048300097A00100E780E04B17C501001305C538BC
:1048400097A00100E780E04A294597A00100E78092
:10485000204F97F7FF1F9387A7A583D70700171748
:104860000020231CF7EC8547171700202304F7DCF2
:1048700097200000E780A0C997F0FFFFE780E07075
:1048800097200000E780A0B1171500200355E5EA46
:1048900097500000E78060FB054597500000E780D7
:1048A000602E97C501009385A51C17C5010013054F
:1048B000A5A397A00100E780C04317C50100130519
:1048C000253597A00100E780C042B1B597500000A0
:1048D000E780402BFC44414697C501009385454342
:1048E00017F5FF1F130585AB829797F7FF1F83C747
:1048F00067F917F7FF1F0347F7F8A207A166D98FDB
:104900001386E6FF7D8E1307001001CA1387F6FF9A
:104910007D8FD1476313F700554797C501009385F5
:10492000E50E17C501001305259C97F7FF1F239B74
:10493000E77E97A00100E780C03B97F5FF1F83D576
:10494000657E17C501001305652A97A00100E78061
:10495000403A29452D6497A00100E780603E371951
:1049600000401304A4AA2320890097F6FF1F938612
:10497000A67B944297C701009387C74117F7FF1F93
:104980000357477A17F6FF1F0346E679814517F567
:10499000FF1F1305A5A097700000E780E0C5232046
:1049A000890097F7FF1F239DA790AA8421C597C56B
:1049B00001009385A50517C501001305E59297A091
:1049C0000100E7800033A68517C50100130585A9FE
:1049D00097A00100E780E031294597A00100E7801A
:1049E000203697F7FF1F239F077297200000E7806C
:1049F000009B5DB597F0FFFFE7802059FDB741119F
:104A000022C437E404008327041A06C6829797500D
:104A10000000E78040E78327040817F5FFFF130530
:104A20004562829797F7FF1F238AA7E417F5FF1FB8
:104A30001305859997500000E780208D2244B240ED
:104A40004101170300006700A3C0B7E70400FC475B
:104A50001171A2DDCAD986DFA6DBCED72E843289BA
:104A60002E86AA8517F5FF1F1305456D829717F748
:104A7000FF1F1307A76C83470700930680029387E5
:104A8000E70793F7F70FE3ECF610BA898A0717C721
:104A900001001307A78EBA979C43BA9782878D4768
:104AA00097C50100938505FF17C501001305C58350
:104AB000630FF40097A00100E780A02317C5010051
:104AC000130545BA97A00100E780A022BDA497A0D6
:104AD0000100E780002217C50100130525BA97A041
:104AE0000100E7800021294597A00100E7804025CB
:104AF000930720F8114697F5FF1F938525644A8593
:104B000017F7FF1F230CF76297F7FF1FA3890762B0
:104B100097F0FFFFE78000312A841DC997C5010087
:104B2000938545F717B501001305057C97A0010093
:104B3000E780201CA28517C501001305E5B797A0E3
:104B40000100E780001B294597A00100E780401F76
:104B500097C50100938505F417B501001305C578C5
:104B600097A00100E780E01817C50100130505B6FE
:104B700097A00100E780E017294597A00100E78092
:104B8000201C4165930730FA054697F5FF1F938572
:104B9000E55A7D1517F7FF1F2302F75A97F0FFFF1D
:104BA000E78040282A841DC997C50100938585EEBA
:104BB00017B501001305457397A00100E780601346
:104BC000A28517C50100130525AF97A00100E78056
:104BD0004012294597A00100E7808016B7E704003E
:104BE000BC4F0566130606C8A14517F5FF1F034510
:104BF000E5C88297FE506E54DE544E59BE5911617D
:104C0000828091476303F40297C50100938585E88C
:104C100017B501001305456D97A00100E780600DF1
:104C200017C501001305C5AD71BDB7E70400FC4F02
:104C3000914517F5FF1F034565C4829797C501008D
:104C4000938545E517B501001305056A97A0010096
:104C5000E780200A17C50100130545AC97A00100A5
:104C6000E7802009294597A00100E780600D974063
:104C70000000E780E036914535A485476303F402E0
:104C800097C50100938505E117B501001305C565BA
:104C900097A00100E780E00517C50100130585A96D
:104CA00015B597F7FF1F23932741B7E70400056663
:104CB000BC4F130606C8C1450DBF8D476303F40200
:104CC00097C50100938505DD17B501001305C56182
:104CD00097A00100E780E00117C50100130545A773
:104CE000D5B3930740F8114697F5FF1F9385054507
:104CF0004A8517F7FF1F2303F74497F7FF1FA38089
:104D0000074497F0FFFFE780E0112A84E30405EEF3
:104D100097C50100938505D817B501001305C55C3B
:104D200097A00100E780E0FCA28517C501001305EC
:104D3000A59897A00100E780C0FB294597A0010036
:104D4000E780000045BD9147E31CF4F6B7E7040097
:104D5000FC4F9305000217F5FF1F034525B282970C
:104D600097C50100938505D317B501001305C557F5
:104D700097A00100E780E0F717C501001305C59E65
:104D8000F1BD894763E3870297C50100938585D00C
:104D900017B501001305455597A00100E78060F5A0
:104DA00017C501001305859D31BB97F4FF1F83C410
:104DB000043997F7FF1F83C7773897C5010093859C
:104DC00065CDA20417B5010013050552DD8C97A02F
:104DD0000100E78000F2A28517C501001305459B7D
:104DE00097A00100E780E0F0C204294597A00100E8
:104DF000E78000F5C1849305D4FF93960401C18236
:104E00004A8693F5F50F17F5FF1F130555339720C5
:104E10000000E780A05FE35F90DC930750F817F78E
:104E2000FF1F230DF73083C73900228697F5FF1F38
:104E30009385C53085074A8517F7FF1FA301F73013
:104E400097F0FFFFE78000FE2A84E30505DA97C5A7
:104E50000100938525C417B501001305E54897A007
:104E60000100E78000E9A28517C501001305C5EC24
:104E7000C9B5894763E3870297C50100938585C15A
:104E800017B501001305454697A00100E78060E6CD
:104E900017C501001305859135B197400000E780E3
:104EA0002014A28517F5FF1F130545299750000010
:104EB000E78040C481B38D476303F40297C50100C6
:104EC000938545BD17B501001305054297A0010064
:104ED000E78020E217C501001305058FE5B6B76628
:104EE00002000146B7750200054597E0FF1FE78005
:104EF000408F930760F817F7FF1F2301F72497F7F8
:104F0000FF1FA38E07229307000617F7FF1F230931
:104F1000F722894717F7FF1FA304F72297F7FF1F10
:104F20002381072297F7FF1FA38D0720C14717F79B
:104F3000FF1F2309F720930720F917F7FF1FA3038B
:104F4000F720314697F7FF1FA38FA71E97F5FF1F86
:104F50009385C51E4A8597F7FF1F2386071E97F086
:104F6000FFFFE78020EC2A84E30605C897C501000F
:104F7000938545B217B501001305053797A00100C9
:104F8000E78020D7A28517C501001305658555B3B5
:104F9000B1476303F40297C501009385A5AF17B528
:104FA00001001305653497A00100E78080D417C580
:104FB00001001305A58439B6B7E70400FC4F93053B
:104FC000000417F5FF1F0345658B8297974000008B
:104FD000E7800001B145F9B5914763E3870297C5C2
:104FE0000100938525AB17B501001305E52F97A0A8
:104FF0000100E78000D017C501001305E581D9B491
:1050000097F4FF1F83C4C41397F7FF1F83C7371399
:10501000A204DD8C8E04B77702006D14BE94228644
:10502000A68517C501001305658097A00100E780DC
:1050300040CCB7E70400FC47228697F5FF1F938515
:1050400035102800829793160401C1823000A6858E
:10505000094597D0FF1FE780C0782A8409C917B592
:1050600001001305657E97A00100E78060E09307CB
:1050700070F8194697F5FF1F9385450C4A8517F779
:10508000FF1F230DF70A97F7FF1FA38B870A97F0DF
:10509000FFFFE78020D92A84E30E05B497C50100FD
:1050A0009385459F17B501001305052497A00100BE
:1050B000E78020C4A28517B501001305E57995B9ED
:1050C0009947630BF41297C501009385A59C17B50A
:1050D00001001305652197A00100E78080C117B585
:1050E00001001305E578F9BA914763E3870297C594
:1050F00001009385259A17B501001305E51E97A0B9
:105100000100E78000BF17B501001305E5775DBA20
:1051100097F4FF1F83C4C40297F7FF1F83C73702AA
:10512000A204DD8C8E04B77702006D14BE94228633
:10513000A68517B501001305657697A00100E780E5
:1051400040BBB7E70400FC47228697F5FF1F938515
:1051500035FF2800829793160401C1823000A6858E
:105160000D4597D0FF1FE780C0672A8409C917B58E
:1051700001001305657497A00100E78060CF9307D5
:1051800080F8194697F5FF1F938545FB4A8517F769
:10519000FF1F2305F7FA97F7FF1FA38387FA97F0FE
:1051A000FFFFE78020C82A84E30605A497C5010015
:1051B0009385458E17B501001305051397A00100CF
:1051C000E78020B3A28517B501001305257095B6B9
:1051D00099476303F40297C501009385A58B17B522
:1051E00001001305651097A00100E78080B017B596
:1051F00001001305256FF9B0B7E70400FC4F9305D4
:10520000000417E5FF1F034565678297974000007C
:10521000E78000DD994579B18D476303F40297C5B6
:1052200001009385258717B501001305E50B97A0AD
:105230000100E78000AC17B501001305256C59B0DB
:1052400017B501001305856C97A00100E78040C2E7
:105250001305C01297D0FF1FE780A00E014597E00D
:10526000FFFFE78060E30D4597100000E780E09FB7
:10527000294597D0FF1FE780C00C97D0FF1FE7801C
:1052800020FD8DBA99476303F40297C50100938509
:10529000658017B501001305250597A00100E7807B
:1052A00040A517B501001305256729B817F7FF1F9B
:1052B000034717E997F7FF1F83C787E822075D8F2A
:1052C0009166BA96C2061166C1821306F6EF8D4743
:1052D0006365D60297E7FF1F9387070F9C4B17F66E
:1052E000FF1F0346D6E59386C7002DC203D60700ED
:1052F00069CA8907E39CD7FE89471307A0F81146BE
:1053000097F5FF1F938585E34A8597F6FF1F23874F
:10531000E6E217F7FF1FA304F7E297F0FFFFE7802D
:1053200060B02A84E308058C97B5010093858576E3
:1053300017B50100130545FB97A00100E780609BAE
:10534000A28517B501001305655EE5B203D6070017
:10535000630EE60A8907E39BF6FE8D4779BF914706
:105360006304F40297B501009385C57217B5010077
:10537000130585F797A00100E780A09717B50100F6
:105380001305455C6FF00FF4B7E70400FC4F93057D
:10539000000817E5FF1F0345654E8297C9B897B50A
:1053A00001009385256F17B501001305E5F397A05C
:1053B0000100E780009417B501001305255A6FF02E
:1053C0006FF02390E70017E5FF1F1305E5FF973007
:1053D0000100E78080BE97B501009385A56B17B5E6
:1053E0000100130565F097A00100E780809017B5D4
:1053F00001001305A55797A00100E780808F29457C
:1054000097A00100E780C0938147C5BD23900700A6
:1054100017E5FF1F130545FB97300100E780E0B952
:1054200097B501009385056717B501001305C5EB16
:1054300097A00100E780E08B17B5010013058554A4
:105440005DBF411122C406C6834705002A849DC75B
:1054500097B501009385C55F17B501001305C5E831
:1054600097A00100E780E0884C4017C501001305B4
:10547000659397A00100E780C087E1A05841B70776
:10548000CF009387777D631DF70697B5010093855D
:10549000255C17B50100130525E597A00100E780FD
:1054A00040851C448356E4008355C40003C60700AE
:1054B00017C501001305859097A00100E780608360
:1054C000294597A00100E780A0870357E4009707CC
:1054D000002083D787266309F7008355C40008445A
:1054E00097E0FFFFE780C0CF0356E4008355C40078
:1054F00008442244B240410117F3FFFF67002355DF
:10550000B707CC009387777D6315F70497B5010043
:105510009385055417B50100130505DD979001002B
:10552000E780207D1C448356E4008355C40003C6F5
:10553000070017C501001305658897900100E780F3
:10554000407B2244B2402945410117930100670086
:10555000237FB707CE009387777D6304F70297B563
:1055600001009385E54E17B501001305E5D7979027
:105570000100E78000784C4017B501001305C5769F
:10558000CDBDB240224441018280B7E70400FC4710
:1055900041112E8606C622C426C24AC02E842A89FC
:1055A000AA8517F5FF1F130565B9829797B5010006
:1055B0009385055017B50100130505D39790010099
:1055C000E780207397F5FF1F83C545B717B5010026
:1055D000130545F497900100E780A0712945979045
:1055E0000100E780E07597F4FF1F938424B583C71B
:1055F000040041479387070693F7F70F636EF75A46
:1056000017B701001307C7E18A07BA979C43BA97F7
:1056100082879D476307F40297B50100938545494A
:1056200017B50100130545CC97900100E780606C29
:1056300017B50100130585EE97900100E780606BB8
:105640008DA497F7FF1F83C777AFDDCB17F7FF1F39
:105650000347F7AE97F7FF1F83C767AE22075D8F3B
:1056600097F7FF1F83C7C7ADC2075D8F97F7FF1F6F
:1056700083C717ADE207D98F17F7FF1F2326F7AAB5
:1056800083C7640097B501009385854217B5010073
:10569000130585C517F7FF1F2307F7A8979001008B
:1056A000E780206597F7FF1F938707A88C4317F6BD
:1056B000FF1F034646A717B501001305E5E79790BE
:1056C0000100E7800063294597900100E78040676B
:1056D00097F7FF1FA38407A62244B24092440249D1
:1056E000930700F817F7FF1F230AF7A49D4517F546
:1056F000FF1F1305A5A44101174300006700833F66
:1057000097600000E780A00E97F7FF1F2389A7A2EC
:105710009357850017F7FF1FA303F7A293570501BF
:105720002A8417F7FF1F230DF7A093578501014522
:1057300017F7FF1FA306F7A097600000E780A00CF3
:1057400097F7FF1F238FA79E97B5010093854536D6
:1057500017B50100130545B997900100E78060591E
:1057600017F6FF1F0346E69DA28517B50100130536
:1057700025DEB1B7CD476303F40297B501009385E9
:10578000253317B50100130525B697900100E78072
:10579000405617B50100130525DD79BD37E4040037
:1057A0007C44414697F5FF1F9385559917E5FF1FE8
:1057B0001305C5BE829797F7FF1F83C7479917F751
:1057C000FF1F0347B798A20703238405D98F17F754
:1057D000FF1F2319F7941306000A89452244B2409B
:1057E0009244024917E5FF1F034545094101028321
:1057F0008D476303F40297B501009385652B17B5B8
:105800000100130565AE97900100E780804E17B543
:105810000100130525E50DB517F4FF1F034424927D
:1058200097F7FF1F83C7979197B501009385452888
:10583000220417B50100130525AB5D8C979001007C
:10584000E780204BA28517B50100130565D397901B
:105850000100E780004A294597900100E780404E0B
:105860000D4697F5FF1F9385658D228597E0FFFF15
:10587000E780405BAA8421C197B501009385452349
:1058800017B50100130545A697900100E780604613
:10589000A68517B501001305E5CF97900100E780B5
:1058A00040452244B24092440249294541011793A0
:1058B00001006700E34897E7FF1F2399877EB7E75A
:1058C0000400116603A38705130606E8914539B75E
:1058D0008D476303F40297B501009385651D17B5E5
:1058E0000100130565A097900100E780804017B57F
:1058F00001001305E5E589B317F4FF1F0344248471
:1059000097F7FF1F83C7978397B501009385451AC3
:10591000220417B501001305259D5D8C97900100A9
:10592000E780203DA28517B501001305E5C79790D4
:105930000100E780003C294597900100E780404046
:105940000D4697E5FF1F9385657F228597E0FFFF52
:10595000E780404DAA841DC197B501009385451588
:1059600017B501001305459897900100E78060384E
:10597000A68517B50100130565C405B797E7FF1F96
:1059800023988770B7E70400116603A38705130601
:1059900006E89305000299B5894763E3870297B546
:1059A00001009385E51017B501001305E593979065
:1059B0000100E780003417B50100130525DCADB9FF
:1059C00097E4FF1F83C4A47797E7FF1F83C7177768
:1059D00097B501009385C50DA20417B50100130505
:1059E000A590DD8C97900100E780A030A68517B5C3
:1059F0000100130525BE97900100E780802F2945FF
:105A000097900100E780C033228697E5FF1F9385BA
:105A1000E572268597E0FFFFE780C0402A84630E89
:105A2000051A97B501009385A50817B50100130560
:105A3000A58B97900100E780C02BA28517B50100C8
:105A4000130585BA99BD854763F987188345190001
:105A50002244B24092440249B335B00097E7FF1F99
:105A60002380B76617B50100130545B941011793A7
:105A7000010067000328A2852244B24092444A856F
:105A8000024941011703000067006324994763033B
:105A9000F40297B501009385A50117B50100130520
:105AA000A58497900100E780C02417B50100130575
:105AB000A5E659B617E4FF1F0344646897E7FF1F84
:105AC00083C7D76797B50100938585FE220417B574
:105AD0000100130565815D8C97900100E7806021CE
:105AE000A28517B501001305E5B297900100E78084
:105AF0004020294597900100E7808024194697E5CA
:105B0000FF1F9385A563228597E0FFFFE780803123
:105B1000AA841DC197B50100938585F917A50100D9
:105B20001305857C97900100E780A01CA68517B51A
:105B30000100130525AF95B397E7FF1F2398875EF4
:105B4000B7E70400116603A38705130606E893056B
:105B5000000869B1854797B50100938565F517A5DC
:105B6000010013056578630BF40097900100E7804E
:105B7000401817B50100130525AC7DBC97900100B6
:105B8000E780201717B50100130585AC9790010039
:105B9000E7802016294597900100E780601A22448B
:105BA000B2409244024997E7FF1F239D07564101E7
:105BB00017630000670023B497B50100938545EF94
:105BC00017A501001305457297900100E780601248
:105BD00017B50100130585D885B4B240224492441C
:105BE000024941018280411106C622C497E0FFFFAD
:105BF000E780402321CD97E7FF1F83D7874C850798
:105C00002A8417E7FF1F231EF74A97B501009385E3
:105C1000A5EB97E7FF1F2397A74A17A501001305D8
:105C2000A56C97900100E780C00CA28517B5010014
:105C30001305851097900100E780A00B2244B24025
:105C400029454101179301006700830F97E7FF1F64
:105C500083D76747B2402244850717E7FF1F231405
:105C6000F74641018280411122C491462A8417E6F9
:105C7000FF1F1306A65A9D652D4506C697D0FF1F28
:105C8000E78020B6B7F7070003C70701A5476313EE
:105C9000F70001A09306001001469D65254597D0A9
:105CA000FF1FE78000B497E7FF1F23898756224430
:105CB000B240914617E6FF1F130646569D652945DB
:105CC000410117D3FF1F6700C3B11171CED7B7E9E8
:105CD000040083A7C904CAD917E9FF1F130909469D
:105CE000A2DD2E8686DFA6DB2E84AA854A858297D2
:105CF00097E7FF1F83C787441307700A6385E71080
:105D0000636DF7001307600A6385E704FE506E5465
:105D1000DE544E59BE59116182801307800A638593
:105D2000E7161307900AE393E7FE8D476306F41C1A
:105D300097B501009385051417A501001305C55AF1
:105D400097900100E780E0FA17B501001305C50F31
:105D500025A08D47630CF40297B50100938585114A
:105D600017A501001305455897900100E78060F8DA
:105D700017B501001305850697900100E78060F7CD
:105D8000294597900100E780A0FB49B7854717B5E3
:105D900001001305650617E7FF1F2303F7329790ED
:105DA0000100E780E00CB7750200B766020001460B
:105DB000054597D0FF1FE780C0A2930760F817E75B
:105DC000FF1F230DF73697E7FF1FA38A07369307B8
:105DD000002617E7FF1F2325F736E577938707216E
:105DE00017E7FF1F2310F736B14597E7FF1F238CF6
:105DF000073497E7FF1FA388A7344A859700000060
:105E0000E780E01621B7914763E3870297B5010069
:105E10009385450617A501001305054D97900100D0
:105E2000E78020ED17B50100130505FFB1B797E432
:105E3000FF1F83C4E43097E7FF1F83C75730A204D6
:105E4000DD8C83A7C9046D14228697E5FF1F938517
:105E5000352F280082978E0493160401B77502002F
:105E6000C1823000A695094597D0FF1FE780609753
:105E7000930770F817E7FF1F2302F72C994597E760
:105E8000FF1FA38FA72A95BF914763E3870297B5AA
:105E90000100938525FE17A501001305E5449790A1
:105EA0000100E78000E517B50100130565F8E9B5C5
:105EB00097E4FF1F83C4C42897E7FF1F83C73728D1
:105EC000A204DD8C83A7C9046D14228697E5FF1F09
:105ED00093851527280082978E0493160401B775C1
:105EE0000200C1823000A6950D4597D0FF1FE780C4
:105EF000408F930780F8BDBF17B50100130505F665
:105F000097900100E780C0F6930790F82304F10012
:105F1000834719008D452800A304F1008347290019
:105F20002305F10097000000E78060041305C0120C
:105F300097C0FF1FE780E040014597D0FFFFE78053
:105F4000A0150D4597000000E78020D2294597C095
:105F5000FF1FE780003F97C0FF1FE780602F7DB3E2
:105F600097E7FF1F23A4A72C828097E7FF1F938743
:105F7000E72B03A30700630303000283174300001A
:105F8000670043B741114AC097F6FF1F83D6E67AF0
:105F9000328917D6FF1F0356464522C426C206C6BD
:105FA0002A84AE8497000000E780A06135C12DC02F
:105FB000994763FF97048347140003470400A2072F
:105FC000D98F13978700A183D98FC2073167C18307
:105FD0001307C755639EE70297D7FF1F83D7E74094
:105FE000A301F400A1832302F40097F7FF1F83D7D6
:105FF000C77491C7A302F400A1832303F400A6850C
:1060000017B50100130505EB97900100E78060CEFE
:1060100097F7FF1F83C70762A5C797D5FF1F83D5D3
:10602000C53C17B501001305A5EA97900100E7806C
:1060300040CC2686A28517D5FF1F0355053B970048
:106040000000E78080BA6306090497F7FF1F83C743
:10605000675EA1E397E7FF1F83C7871D9DCB95C8A8
:1060600097E7FF1F83C7C7058DE722852244B2400B
:106070000249A6859244410117430000670083A7A7
:1060800017B501001305C5E597900100E78040DED4
:106090005DBFB2402244924402494101828083475D
:1060A00055008345450017B50100130565DFA207BC
:1060B000DD8D179301006700C3C317B501001305F9
:1060C00025DD179301006700A3DA8D4763FBB70A4C
:1060D000011126CA06CE22CC0344350097E4FF1FE7
:1060E00083C4141597B50100938545E0B33780004C
:1060F00017E7FF1FA30EF71209C497B50100938598
:10610000A5DF17B501001305A5DF97900100E78013
:1061100040BE97E7FF1F83C7B7116386970097E0DC
:10612000FFFFE780405197E7FF1F83C777108DC7B8
:1061300085472306F100B7E7040083A747177000DF
:10614000854513055030829717B50100130545DCCE
:1061500097900100E780C0D19967938757EE231687
:10616000F100680085479145A30781002307F100EE
:1061700097000000E780A0DFF2406244D24405614E
:1061800082808280894763FCB708011122CC06CE49
:106190008347250005472A846393E706914763FCFC
:1061A000B7048347450003473500A207D98F17D7A7
:1061B000FF1F03578723630AF70017D7FF1F231614
:1061C000F72297E0FFFFE78060459967938767EEC6
:1061D0002314F10085472305F10083473400A3050C
:1061E000F10083474400954528002306F1009700FD
:1061F0000000E780C0D7F240624405618280E5FF7D
:106200009967938767EE2314F10097D7FF1F83D711
:10621000C71DA305F10023050100A183E9B7828012
:106220000111996722CCD51717F4FF1F130484407E
:106230002314F1008347040026CA97F4FF1F9384B8
:10624000C44F2305F10083D7040028009545A3051A
:10625000F100A18306CE2306F10097000000E7803D
:1062600000D103D604008345040017B501001305CF
:10627000A5CB97900100E780C0A7F2406244D244CA
:10628000056182809D677971D9172316F10097F710
:10629000FF1F83C7273A06D62307F100A9C3B7E734
:1062A0000400FC47414697D5FF1F9385250F130532
:1062B000F10082976800CD4597000000E78020CB71
:1062C00097F5FF1F83C5053717B501001305C5C82E
:1062D00097900100E780E0A1B25045618280B7E766
:1062E0000400BC47414681451305F1008297D9B7A8
:1062F00045C5411106C622C4930750FA2300F50094
:106300009307A005A300F50089472301F5009147F5
:10631000A301F50093072004A302F50097F7FF1FE0
:106320009387473183C70700230205002A8423038C
:10633000F50097E7FF1F9387B7EF83C70700414634
:1063400097D5FF1F93858505A303F50097F7FF1FDA
:1063500083D7A73E2304F500A183A304F50097D7B4
:10636000FF1F83D787082305F500A183A305F50048
:10637000B7E70400FC47310582972285F145970075
:106380000000E7800020230EA4002181A30EA400BA
:10639000B24022444101828082805D710A8586C6B6
:1063A000A2C497000000E780E0F437E404007C44D6
:1063B0008A850810794682973C441305E103094613
:1063C00081458297101093050002014597D0FFFF89
:1063D000E780C032B640264461618280011122CC40
:1063E0002D6426CA4AC84EC652C456C25AC006CEEA
:1063F000B71400401304A4AA80C037E900E0B7092D
:1064000040002A8AAE8A328B23203919010001000C
:106410008566AA850146254597C0FF1FE780603C39
:10642000DA865686D285294597C0FF1FE780603BF4
:106430002320391180C0F2406244D2444249B2491B
:10644000224A924A024B056182800111B7C7A55AC0
:1064500022CC9387C73317E4FF1F130474DD3EC4B7
:10646000834704002C002146196506CE3EC69700DE
:106470000000E780E0F68345040017B5010013052E
:10648000A5BC97900100E780C086F2406244056198
:1064900082800111A146300099652D4522CC06CE9F
:1064A00097C0FF1FE780E033A24737C4A55A130403
:1064B000C43363958702B24517B50100130505ACD7
:1064C000B335B00097E7FF1FA384B7D697900100BC
:1064D000E7802082F2406244056182809165A14696
:1064E0003000938505F02D4597C0FF1FE780602F92
:1064F000A247E38287FC97E7FF1FA38B07D2814562
:1065000017B501001305C5A9D1B77971D14670003F
:1065100091652D4522D406D697C0FF1FE780602CD9
:10652000B24737C4A55A1304F43563988702B7E716
:106530000400FC4717D5FF1F130545E641460C082C
:10654000829717B501001305A5AB97900100E7806E
:106550002092B2502254456182809165D1467000EC
:10656000938505E82D4597C0FF1FE7808027B24738
:10657000E38F87FA17B50100130585AAF9B7C1673C
:1065800069768146FD17050613970601418363640A
:10659000B7003E8582803307D50003470700B98FD7
:1065A000214713F81700858363050800B18FC207E0
:1065B000C1837D171377F70F6DF78506F1B741C5D6
:1065C000A547054763F2B708834715000347050051
:1065D0003168A207D98F13978700A183D98FC2078B
:1065E000C1831308C855054763900707411106C6C4
:1065F00022C426C203442500914763F08704930711
:10660000540063ECF502A301C50021822302C500FA
:106610009304340091C6A302D500A1822303D500C0
:106620002A84A68597000000E780A0F52694230021
:10663000A4002181A300A4000147B2402244924457
:106640003A854101828005473A8582800111B7C7AA
:10665000A55A22CC9387E7342A842AC621462C00E7
:10666000156506CE3EC497000000E78060D7A2857E
:1066700017B501001305459F97800100E78060670B
:1066800097000000E780A0D1F2406244056182805B
:106690000111A146300095652D4522CC06CE97C04C
:1066A000FF1FE7800014A24737C4A55A1304E4343F
:1066B00063958702B24517B501001305659097D71A
:1066C000FF1F2394B7D2C205C18197800100E780E4
:1066D0004062F2406244056182809165A1463000CB
:1066E000938505EE2D4597C0FF1FE780800FA247D9
:1066F000E38287FCD14717D7FF1F2318F7CED14578
:1067000017B501001305C58DC9B721C1411126C2B6
:1067100006C622C4AE848DC52A8497000000E78097
:10672000E06697E7FF1F83C7A7B099CB2285224475
:10673000B240A68592444101173300006700833BB5
:10674000B2402244924441018280828001114AC8B1
:1067500006CE22CC26CA4EC693F715002E899DCBB5
:10676000AD67371700409387A7AA1CC3B7E704009B
:10677000BC4F13060019854517D5FF1F0345C5C635
:10678000829713451900F2406244D2444249B2490B
:106790000561828093F72500638A071C17F7FF1FA6
:1067A000035787F9954763F9E70C014417F6FF1F74
:1067B000130686E8930630051305500413081004E9
:1067C0009308B00413039005930764006374F704FF
:1067D0003A84FD5997F4FF1F83C404E697F7FF1F1F
:1067E00083C797E5A204DD8CAD679387B755638BAC
:1067F000F41463E3970AA9679387A755638EF4148B
:10680000A28517F5FF1F130525E397000000E78019
:1068100000F031A2B307860083C50700639AD50450
:1068200083C517006396A50483C5270063920505F9
:1068300083C53700639ED50283C54700639A15035D
:1068400083C7570063966702A2890DE897F5FF1F7B
:1068500083D585EEB3853541C20517F5FF1F1305B6
:10686000A5DDC1814E9597000000E78040EAE1A0D8
:1068700005044204418089BF3A84FD598547E3EB12
:1068800087F45DC4854517F5FF1F1305E5DA97000A
:106890000000E780C0E769A8B1679387C7556380A8
:1068A000F404B5679387D755E39CF4F4A28517F5F4
:1068B000FF1F130565D897300000E780A0238947A4
:1068C000630FF4049305E4FFC205C18117F5FF1FB0
:1068D0001305A5D697000000E780404B89A09720BC
:1068E0000000E780A00D97000000E780804911C9F3
:1068F000A28517F5FF1F130525D497000000E78038
:10690000E0480546A28517F5FF1F1305E5D297F06D
:10691000FFFFE780606797200000E780200AA685D8
:1069200017A501001305057697800100E780603CFC
:10693000FD57E39DF9F097F7FF1F239F07DE1345EF
:10694000290091B5A28517F5FF1F1305E5CE97F035
:10695000FFFFE7800075E1B7A28517F5FF1F13055C
:10696000A5CD97F0FFFFE780807555BF93F74500F1
:106970000145E38A07E017A501001305E57197803B
:106980000100E780E04E97300000E7804044134567
:106990004900D5BB411122C437E404005C5C06C643
:1069A000354697A501009385251B17B501001305F2
:1069B000E5F4829711E917A501001305A56E9780EC
:1069C0000100E780E04A01A08327041C82972A8403
:1069D000054597C00000E78020FE97700100E78022
:1069E000408397600100E780405897B00000E7803F
:1069F000A00F2285B2402244410182804111054509
:106A000006C622C426C297C0FFFFE780C052130506
:106A1000A00497B0FF1FE7808069757585457D15D7
:106A200097C0FFFFE780603C7D7585451305F5360F
:106A300097C0FFFFE780C045371400408327840AD2
:106A40008D451305002093E707202324F40A97C0FF
:106A5000FFFFE7808039B7E4040097C0FFFFE780BD
:106A6000A07EC85897800100E780804017B50100DC
:106A70001305C5E897800100E780803F8327840CD9
:106A80008545414593E707082324F40C97C0FFFF91
:106A9000E78000408D451305000897C0FFFFE780A1
:106AA000203F97C0FFFFE780006C37A50700130564
:106AB000051297C0FFFFE780A067014597C0FFFF61
:106AC000E780C06D95450545894717F7FF1F2307E8
:106AD000F7C697C0FFFFE780006EB7E700E0130737
:106AE0000006238DE7403707000423A0E71097D066
:106AF000FFFFE78080EF97D0FFFFE78080019700DE
:106B00000000E78060E997000000E780C0989700E8
:106B10000000E78020B897E0FFFFE78080EE970055
:106B20000000E780E02797000000E780E01083A7DF
:106B30000408170500001305A5C1829797D7FF1F0A
:106B40002384A78ABC4C130600648545829797C0AE
:106B5000FF1FE780E089014582807D77B377E500FC
:106B6000AA9563E9F5048566FD16AE9641119D8EE2
:106B700006C622C426C2F98E91E285662D673716B5
:106B800000401307A7AA18C237E400E0B70440008A
:106B900023209418010001000146BE85254597C0B9
:106BA000FF1FE78000C4B240232094102244924487
:106BB000410182807D5582804111B2862E86AA8550
:106BC0002D4506C697C0FF1FE780A0C1B240014512
:106BD000410182809307000463ECC7041D71A2CCBD
:106BE0002A840808A6CACAC886CE32C69780010081
:106BF000E780C004AD67371700409387A7AA1CC37E
:106C0000B7E400E03709400023A024190100010087
:106C1000B2461008A285294597C0FF1FE78060BCD7
:106C2000F640664423A02411D6444649256182805B
:106C30003955828041110D658D4506C697C0FFFF0D
:106C4000E780A01AB71700408D6623A6D70A17F56C
:106C5000FF1F1305E5AE1387C70A9387870A1CC178
:106C60005CC5856689675CC958C114C518C9B7E792
:106C70000400B24003A3871E410102838145B3078C
:106C8000B5008387070089E7172300006700A3D9B1
:106C90008505C205C181E5B797A701009387076104
:106CA0001357C5003E9703470700011106CE230482
:106CB000E100135785003D8B3E97034707002306ED
:106CC0000100A304E100135745003D8B3D893E9729
:106CD000AA970347070083C7070028002305E100A0
:106CE000A305F10097000000E78080F9F2400561FC
:106CF0008280411126C2E97797F4FF1F9384C4B4C0
:106D000022C49387A7552E842381B4002E86AA859A
:106D100017F5FF1F130585B306C62390F400A38162
:106D2000040097800100E78060F193052400C2050C
:106D3000C18117F5FF1F130545B197000000E780DB
:106D40004084B38784002382A7002181A382A70007
:106D5000930564002244B24026859244C205C18155
:106D6000410117230000670003CC09C99307800283
:106D700063E6B700170300006700E3F7828017F5AA
:106D8000FF1F0345659D828097F7FF1F83C787AB71
:106D900089E717230000670003C9828097F7FF1F68
:106DA00083C767AD99EF411106C697200000E780C1
:106DB00060BFB240854717F7FF1F230EF7AA4101B6
:106DC0008280828063030560638105605D71A2C477
:106DD000A6C286C6CAC04EDE52DC56DA5AD85ED685
:106DE00062D466D26AD0B9472A84AE8463F9B70602
:106DF000394697A501009385A53397800100E78068
:106E000080E131ED8347E400130710036394E70248
:106E1000854717F7FF1F2307F7A217A501001305E2
:106E2000253297F7FF1F239E07A097000000E780F9
:106E300020E571A01307000317A5010013054533D2
:106E4000E395E7FE97F7FF1F238E079E97F7FF1F37
:106E50002399079E17A5010013050530F9B797F789
:106E6000FF1F83C7279E63890722BD6AB96B938C76
:106E7000FA55014A17FBFF1F130B4B8E138CEB6562
:106E8000938AFA6605A8B307440183C6070097F7FB
:106E9000FF1F83D7079BB1E39307A005639BF60011
:106EA000854717F7FF1F231EF79897F7FF1F2387C4
:106EB000D78A050A93170A01C183E3E697FCB64017
:106EC000264496440649F259625AD25A425BB25B52
:106ED000225C925C025D61618280054D639BA70329
:106EE0009307500A639EF600894717F7FF1F231A7E
:106EF000F794930750FA17F7FF1FA301F78655BFC2
:106F00009307A005E387F6FA97F7FF1F239B0792E5
:106F10004DB7138717004207DA9741832380D700C4
:106F200017F6FF1F231FE6908D47E3F4E7F817F9E4
:106F3000FF1F0349D98297F7FF1F83C747822209A2
:106F40003369F9009307F9FFC207C1839306F00D77
:106F5000E3ECF6FA93076900C207C183E31BF7F479
:106F600093052900C205C18117E5FF1F1305257F81
:106F700097F0FFFFE780E06033072B01834757005E
:106F800003474700A207D98F17F7FF1F231B078A64
:106F90006319F50E8149630DA90197E9FF1F83C9A4
:106FA000297CA20997E7FF1F83C7977BB3E9F90004
:106FB000170500001305A5DB97F0FFFFE78080FAB7
:106FC00063878907636D3C039387EB556382F904FC
:106FD00097E7FF1F83C7C77805476389E70681CB1B
:106FE0001387A7051377F70F8D4663F2E60813079B
:106FF000F0072300E100A300F10089459DA0638212
:107000009905E39759FD97F0FFFFE780E02711A866
:10701000CA8517E5FF1F1305A57497F0FFFFE780EA
:10702000000B014597F0FFFFE780C0F359B5CA8513
:1070300017E5FF1F1305C57297F0FFFFE780C01427
:10704000CDB797F0FFFFE780E01DE1BF930710F891
:10705000130511002300F10097F0FFFFE78080295E
:10706000FD450A8597000000E780E0C85DBFCA853E
:1070700017E5FF1F1305C56E97F0FFFFE78020C5DA
:107080004DB79307F00789450A852310F100970053
:107090000000E78040C631BDBD4763F197204146FF
:1070A00097A501009385050F228597800100E78051
:1070B00080B66317051E17A501001305E50E97009E
:1070C0000000E780E0BB17E5FF1F03550567970049
:1070D0000000E780A0BC97E7FF1F83C7A75517A54F
:1070E00001001305E50289E717A501001305C50294
:1070F00097000000E780C0B817A501001305450CF4
:1071000097000000E780C0B717C5FF1F0355852B08
:1071100097000000E78080B8054597500100E780A0
:10712000609C97A701009387A7FF09E597A7010037
:10713000938787FF3E8597000000E78060B417A51E
:1071400001001305250897000000E78060B317C50C
:10715000FF1F0355852997000000E78020B417A57D
:1071600001001305A50697000000E78060B117D560
:10717000FF1F035545F597000000E78020B217A5D3
:1071800001001305250597000000E78060AF17D5C3
:10719000FF1F035505F397000000E78020B017A5F7
:1071A00001001305A50397000000E78060AD17D527
:1071B000FF1F035525F197000000E78020AE17A5BB
:1071C00001001305E50197000000E78060AB9740E0
:1071D0000000E780C061418197000000E78000ACBB
:1071E00097400000E780A0604205418197000000C1
:1071F000E780C0AA17A50100130505FF970000004E
:10720000E78000A897400000E780205F4181970059
:107210000000E780A0A897400000E780005E4205DC
:10722000418197000000E78060A717A501001305C2
:1072300025FC97000000E780A0A417C5FF1F035599
:10724000250897000000E78060A517A50100130539
:10725000A5FA97000000E780A0A297C7FF1F83C789
:10726000E713A20717C5FF1F034555135D8D970050
:107270000000E780A0A297C7FF1F83C74712A2079D
:1072800017C5FF1F0345B5115D8D97000000E7800E
:10729000E0A0179501001305E56141BE6390F4126B
:1072A0003D4697A50100938565F5228597800100ED
:1072B000E78060964DE5C514C2041306F400C18052
:1072C0004D0481470D452548954563799500631C1C
:1072D00086001397070141876348E00417A5010062
:1072E0001305C5F299B603470600930607FD93F60A
:1072F000F60F637CD8009306F7FB93F6F60F63EC6A
:10730000D500130797FC9376F70F9207D58FC20726
:10731000C18305065DBF9306F7F993F6F60FE3EF19
:10732000D5FA130797FAC5B717C7FF1F0357E70B1F
:10733000630AF70017C7FF1F2319F70A97D0FFFF4B
:10734000E780C02D17A50100130585EE970000000A
:10735000E780009317C5FF1F035525093DB7C147B7
:1073600063FE9704414697A501009385A5ED22850C
:1073700097800100E780208A31E1834704011307E9
:107380001003639CE700854717E7FF1F2306F73CC0
:1073900017A50100130545EC49BC1307000317A509
:1073A0000100130565EEE392E7A897E7FF1F238529
:1073B000073A17A501001305A5EB85BCA685228514
:1073C00097C0FFFFE780C0E1DDBC8280411126C28B
:1073D000AE848D4522C406C62A8497C0FFFFE7808D
:1073E00020ABB717004099C803A5C70C418D23A651
:1073F000A70CB240224492444101828003A5870C2D
:10740000418D23A4A70CF5B783470500034715005A
:10741000A207D98FC2076177C18713072720639A14
:10742000E7008345250037050400170300006700C7
:1074300023FA828017E6FF1F130646448147B2866F
:107440001303F00FA9483308F6000348080013F7A8
:10745000F70F6307A80C630668008507E39517FF1D
:107460002947B387E6002380A70097E7FF1F93878C
:10747000A7415DA8411113D765001347170006C641
:1074800093F63500058B954791CA05469947638762
:10749000C60009469D476383C600A14713F6450011
:1074A0003336C00093F68503050685C2A145638B7C
:1074B000B604E145638AB604930580026388B60486
:1074C000930580036393B600914697E5FF1F2382DF
:1074D000F56297E5FF1F238DC56097E5FF1FA38920
:1074E000D560BE8517A50100130545E09780010012
:1074F000E7802080B240854717E7FF1FA30BF75EA8
:10750000410182808546D1B78946C1B78D4675BF96
:1075100017A50100130505E0177301006700637DDF
:1075200017E7FF1F13074736BA972380B700E147D5
:10753000E302F5F493077002E30CF5FC82802A87DE
:1075400023800500814717E5FF1F13052533130826
:10755000F00F2946B306F50083C606006396E602DF
:1075600097E6FF1F93864632B69783C70700054507
:107570002380F5009947636EF7029D4763FDE7009E
:10758000E147630DF7008280638506018507E39379
:10759000C7FC0145C5B7238005008280B73700408E
:1075A00003C7370083C7050093F70704D98F2380EB
:1075B000F50082805D7152DC56DA5ED6716A97EB17
:1075C000FF1F938B2B648D6AA6C24EDE62D486C6E3
:1075D000A2C4CAC05AD866D26AD06ECEC1495E8CE7
:1075E00097E4FF1F9384042B130A0A20938A7ADC02
:1075F00017E9FF1F03490964B3872B0183C70700FD
:1076000093F7F70FC9EFB787004003C76700058BF3
:10761000E310077C03C76700118BE30D077E83C768
:107620005700918B99E36F10200317E7FF1F034763
:10763000876085476304F7006F10400197E7FF1FDD
:10764000A389E74A97E7FF1F2386073097E7FF1FC5
:107650002384073C97E7FF1F2382074897E7FF1F14
:10766000238F074697E7FF1FA386072E97E7FF1F85
:10767000A384073A97E7FF1FA382074697E7FF1FF8
:10768000A38F074497E7FF1FA386074697E7FF1FCF
:10769000A383075AB787004011476F00707793079D
:1076A000190093F7F70F3D476364F70617E7FF1FCD
:1076B0002302F75897E7FF1F9387C756CA9783C7D8
:1076C00007001307100293F7F703638EE71E636644
:1076D000F70405446385871CE38C07620947638EC2
:1076E000E71013070002E384E74EB7E700E037072F
:1076F000400023A0E718010001006299230009005F
:10770000FD1923A0E71093F9F90FE39309EEE5BD06
:1077100097E7FF1F2380075271BF1307300263886A
:10772000E70C63E8E71613074002638CE70A1307C8
:107730000003E39CE7FA97E7FF1F9387A74DCA97DB
:1077400003C70700A1471377F70FE31BF71483C79D
:10775000640097E6FF1F2385F63897E7FF1F83C76E
:10776000D71391C7FD5797E6FF1F238BF63697E592
:10777000FF1F83C5351297E7FF1FA383B73697E72F
:10778000FF1F83C7271113FB07089306000493F715
:107790000706639FD74C9307A009638DF51663EA2C
:1077A000B7129307F0056386F54A9307500963847F
:1077B000F52A014497E7FF1F83C797321547E392E5
:1077C000E736B7E700E03707400023A0E7180100DD
:1077D0000100B786004023808602130680FC6F00FC
:1077E000500EFD5717E7FF1F230BF72EFDBDFD576A
:1077F00017E7FF1F2304F72ECDBD17A501001305C2
:10780000E5C297700100E780A06697E7FF1F9387A6
:107810006740CA9703C40700014B97ECFF1F938C86
:10782000EC1F1374F40F17AD0100130DADC06347C7
:107830008B04294597700100E7808050854717E742
:10784000FF1FA30BF71C17E7FF1F2308871C17E771
:10785000FF1F2301F72A37E700E0B7064000232087
:10786000D71801000100378600408347A60293F72E
:10787000370F2305F6022320D71085BDB3876C018F
:1078800083C507006A85050B97700100E780604695
:1078900079BF854717E7FF1F2300F718B9B517E72A
:1078A000FF1F130727374A970347070097E6FF1F75
:1078B000A382F60A97E6FF1F238FE60817E7FF1F4C
:1078C000230AF7221DB5854717E7FF1F2304F70892
:1078D00029BD9307400A6389F5349307200B63841D
:1078E000F5369307100AE396F5EC838724000144EC
:1078F000E3D207EC97E7FF1F83C7F7F993F637004A
:10790000638A061A0546638AC62209466395C61A23
:107910001D4755A217E5FF1F0345E5F7C94797EC3B
:10792000FF1F83CC5CF797E5FF1F83C5E5F617E4DF
:10793000FF1F034474F66315F510CD476392FC10E6
:1079400093077008639CF5021307300FB7170E00FA
:107950006308E4001307900DB7B704006314E4084C
:1079600017E7FF1F2324F718BE8517A5010013058D
:10797000E5AC97700100E780C03725BD930780080C
:10798000639DF500B307804013F4F70FB777460007
:10799000938787CDB3D78702E1B793079008639A9F
:1079A000F500B307804013F4F70F91679387C7661C
:1079B000D5B79307A008639BF500B307804013F485
:1079C000F70FB7173D0093870790E9B79307B00803
:1079D000639AF500B307804013F4F70F916793871C
:1079E00097D04DBF93F5F5078D47639BF500B3071F
:1079F000804013F4F70FB7975B00938707D859BF00
:107A00008947639BF500B307804013F4F70FB777FE
:107A10000B009387071BBDBF8547639AF500B3072B
:107A2000804013F4F70FDD67938767E3A5B7D2872C
:107A300085F9B307804093F7F70FB3D7FA020DB774
:107A400097000000E780409FA285668597000000B0
:107A5000E780809EB9BB9305610017E5FF1F0345D2
:107A600085E317E4FF1F034414E397000000E78059
:107A700040AD93057100228597000000E78060AC5F
:107A80003C0017E7FF1F232DF716834761002304EF
:107A9000F10083477100A304F100894717E7FF1F36
:107AA0002300F7048357810017E7FF1F2314F7DE35
:107AB000094409B3154793F64700B336D00093F74E
:107AC0008703850685C32146638BC7066146638AA3
:107AD000C706130680026388C706130680036393F4
:107AE000C700914717E6FF1F2304D60097E6FF1F44
:107AF000A380F60097E7FF1F238DE7FE17E7FF1F20
:107B0000034787D99376070497E7FF1F83C7D7D822
:107B10008DEE1377770C93067008630CD7021377FA
:107B2000F7078D466312D70CB307F040B7955B009B
:107B300093F7F70F938505D849A81947ADBF854737
:107B400055B7894745B78D4771BF930670086311D4
:107B5000D7021307300FB7150E006389E70213072A
:107B6000900DB7B504006383E7021307700845BFA3
:107B70009306800C6311D702B307F040B775460037
:107B800013F7F70F938785CDB3D5E70297E7FF1F6C
:107B900023AEB7F4D9BB9306900C631CD700B30790
:107BA000F04093F5F70F91679387C766B3D5B70297
:107BB000F1BF9306A00C631DD700B307F040B715C3
:107BC0003D0093F7F70F93850590B3D5F5027DBF80
:107BD0009306B00CE315D7F4B307F04093F5F70F15
:107BE0009167938797D0D9B78946631BD700B307AE
:107BF000F040B7750B0093F7F70F9385051BF1B7AE
:107C00008546631AD700B307F040DD6593F7F70F99
:107C1000938565E35DBFD28535FBB305F04093F5F1
:107C2000F50FB3D5BA029DB783C72400C18B99C79E
:107C3000854717E7FF1F2308F7EAA5BE97E7FF1F51
:107C4000238307EABDB6854717E7FF1FA303F7EABB
:107C50008DB63C0017E7FF1F2324F7FA0947930767
:107C600000032314F10097E6FF1F238BE6E62DBDEA
:107C700063940756A94763E5B742179701001307B6
:107C800027648A05BA959C41BA97828717E4FF1F3B
:107C9000034474C0894C6306940D63E68C068547E3
:107CA0006303F4089307F00F17E7FF1F034747E349
:107CB00063F6E70017E7FF1F2304F7E297ECFF1FC7
:107CC00083CC0CE29307000413F4FC0F63F49701D8
:107CD0001304000497E7FF1F938787F203AD0700A3
:107CE00022862685EA85B38C8C40229D9770010000
:107CF000E780C0F497E7FF1F238497DF97E7FF1F14
:107D000023A0A7F145BC8D47630CF40A9947E31BF8
:107D1000F4F8979701009387276117E7FF1F232146
:107D2000F7EEA94751B717E7FF1F0347C7F097E7DB
:107D3000FF1F9387E7DC4946979501009385C56748
:107D40006306870097950100938505633E859770CC
:107D50000100E780A0EE17E7FF1F2323A7EAC9472A
:107D6000A1B797E6FF1F83C606ED054797E7FF1FFC
:107D7000938707D96394E6023E85130670029795B0
:107D800001009385E56097700100E78020EB17E71D
:107D9000FF1F2327A7E69307700239B73E85130616
:107DA0003004979501009385E55897700100E780AE
:107DB000E0E817E7FF1F2325A7E493073004EDB59C
:107DC00097E5FF1F83C525AD17950100130545688D
:107DD00097700100E780E0F1054D97EDFF1F83CD1F
:107DE0008DE597E5FF1F83C505AB179501001305CA
:107DF00025666398AD0B97700100E78080EF97E7E9
:107E0000FF1F83C747A9B5CBE36EF4E817940100C1
:107E10001304C45E638CB701179401001304845EDD
:107E200063869701179401001304445F22859770BD
:107E30000100E78020051375F50F930715008607ED
:107E400017E7FF1F230EF7CA8D4717E7FF1FA30988
:107E5000F7CA97E7FF1F9387A7CA0147BE86137625
:107E6000F70F89076365A60297E7FF1F23AAD7D8F4
:107E700097E7FF1F83C7C7C805BD97970100938782
:107E8000E75017E7FF1F232DF7D6914731BD330683
:107E9000E40003460600A380070005072380C7000F
:107EA0007DBF97700100E780C0E497E7FF1F83C79D
:107EB000879EE1D7E368F4DE1794010013040451B0
:107EC000638CA701179401001304C45063869701C3
:107ED0001794010013048451228597700100E780F4
:107EE00060FA1375F50F93071500860717E7FF1F54
:107EF0002308F7C08D4717E7FF1FA303F7C097E7D5
:107F0000FF1F9387E7BF0147BE861376F70F8907E8
:107F1000E37CA6F43306E40003460600A3800700D2
:107F200005072380C700D5B797E5FF1F83C5A59632
:107F3000179501001305855297700100E78060DBFB
:107F400097E7FF1F83C797BB93E7470017E7FF1F1C
:107F5000A306F7BA83C7240017E7FF1FA30EF7B8DD
:107F600089B8179501001305A55097700100E780A7
:107F700020F097E7FF1F938727B883C7070017E70D
:107F8000FF1F2309F79017E4FF1F034464B5333440
:107F900080000DB0179501001305C54E97700100C4
:107FA000E78000ED97E7FF1F83C757B593E7070109
:107FB00017E7FF1FA304F7B483C7240017E7FF1FC9
:107FC000230CF7B26FF0EFFE179501001305C54CB7
:107FD00097700100E780C0E903C704007D8B51EF73
:107FE000B787004003C767021377C70B13672700E3
:107FF0002383E70203C7A7021377C70B1367270082
:108000002385E70203C7E7021377C70B136727002F
:108010002387E70203C727031377C70B13672700DC
:108020002389E702854717E7FF1F2305F79217E724
:10803000FF1F2303F79E17E7FF1F2301F7AA17E788
:10804000FF1F230EF7A897E7FF1FA385079097E769
:10805000FF1FA383079C97E7FF1FA38107A897E74C
:10806000FF1FA38E07A697E7FF1FA38507A897E723
:10807000FF1FA38207BC6FF0CFF389476312F7029B
:1080800097E7FF1F83C747819146638CD70863E05A
:10809000F604638EE70C6369F70A05476380E70E11
:1080A000FD5717E7FF1FA30DF7A237074000B7E7FB
:1080B00000E023A0E71801000100B7860040130686
:1080C000F0FC2381C60223A0E7106FF00FE2130734
:1080D00020086382E7086362F70213071008E39140
:1080E000E7FC378700408347670293F7C70B93E7A6
:1080F00027002303F7026FF0CFEB130730086389E3
:10810000E70213074008E39DE7F8378700408347FD
:10811000270393F7C70B93E727002309F7026FF0B4
:108120004FE9378700408347270393F73707F5B7B1
:10813000378700408347E70293F7C70B93E7270091
:108140002307F7026FF0EFE6378700408347E70227
:1081500093F73707F5B7378700408347A70293F7B0
:10816000C70B93E727002305F7026FF08FE43787EB
:1081700000408347A70293F73707F5B737870040DA
:108180008347670293F73707ADB7179501001305CB
:10819000A53197700100E780A0CD97D7FF1F238BF3
:1081A000076ED5B3179501001305053197700100CF
:1081B000E78000CC97D7FF1F239E076C97E7FF1F30
:1081C0009387079203C40700894763F38700094434
:1081D0001374F40F6FF00FDE13070002E392E7EC65
:1081E000631B0B0A638FF500930720026383F50876
:1081F000179501001305C52F97700100E78060AF48
:1082000045B5179501001305E52B97700100E78030
:1082100020C60144179D0100130D0D2CA14CB387FE
:10822000840083C507006A85050497700100E78014
:1082300040ACE31694FF178501001305A56D9770F8
:108240000100E780E0C217D4FF1F0344E46401E8A3
:1082500097D7FF1F23820762014B6FF0AFD5894785
:10826000E310F4E4854717D7FF1F2307F7606FF08B
:108270004FD417D6FF1F0346166297D5FF1F83C53D
:108280008561179501001305A52597700100E7800A
:1082900040A66FF00FD26380F50693071002E399B2
:1082A000F5F497D5FF1F83C5255F179501001305CA
:1082B000252597700100E780C0A397E7FF1F23A142
:1082C000979497E7FF1F93876782944383D747006C
:1082D00017E7FF1F0347E78117D6FF1F232CD65A46
:1082E0001D4497D6FF1F2399F65A97D7FF1F238661
:1082F000E75A6FF02FCC97D5FF1F83C5E559179527
:1083000001001305652197700100E780809E97D7D3
:10831000FF1F2383075697D7FF1F239D07566FF034
:108320002FF92547638FE7C8994637870040639444
:10833000D70223008702B7E700E0B706400023A07A
:10834000D71801000100130600FC2301C70223A077
:10835000D7106FF08FB99306100A639FD7002300E0
:108360008702B7E700E0B706400023A0D718010056
:108370000100130680FCD1BF9306A009E381D7FE5C
:108380009306400AE38DD7FC93062002639DD70035
:10839000B7E700E0B706400023A0D71801000100AE
:1083A00023008702F9B78546E384D7FE93070008C8
:1083B000E300FBFEB7E700E0B706400023A0D718B4
:1083C00001000100130620FC23008702BDBF17D760
:1083D000FF1F0347F7706302F71E63E7E702954745
:1083E0006300F7109947630AF704B78600402380BB
:1083F0000602B7E700E03707400023A0E7180100B6
:1084000001001306A0FC75B99307F005630AF70095
:10841000930750096306F70093071002E317F7FC70
:10842000B7E700E03707400023A0E718010001008C
:10843000B7860040130620FC69B117DBFF1F034B12
:108440002B6A930700045A8D63F46701130D00042F
:1084500097D7FF1F9387C77A83AC07001374FD0F6C
:108460002286E685268597600100E780207DB30798
:108470008B40669417D7FF1F2304F76697D7FF1F1B
:1084800023A08778B7870040630C0B022380A703E3
:10849000B7E600E03706400023A0C618010001003F
:1084A00003C72702134707042381E70203C72702F4
:1084B0001377C70F2381E70223A0C6106FF0EFA246
:1084C0002380070237E700E0B70640002320D718D3
:1084D00001000100130620FC2381C7026FF0AFB931
:1084E000378700408347370097D6FF1F83C6D66083
:1084F00093F70708D58FA301F700B7064000B7E749
:1085000000E023A0D718010001001306A0FC35BD30
:1085100097D7FF1F93870770CA9783C7070093F702
:10852000F70FC1CF97D7FF1F83C7E770D9E717D7DA
:10853000FF1F0347F75A930700026310F70883AD44
:10854000040017DDFF1F034D2D3597DCFF1F83CC83
:10855000BC3417DBFF1F034B4B34E6876A87DA8690
:108560006E8697D5FF1F83C525311795010013052A
:1085700025FC97600100E780C07797D7FF1F23A7EE
:10858000B75797D7FF1F2385A75797D7FF1FA381FB
:10859000975797D7FF1F238E675597D7FF1FA38C39
:1085A000872CB7E700E03707400023A0E718010059
:1085B0000100B78600406FF04FA2B7E700E0370731
:1085C000400023A0E71801000100B786004015BD58
:1085D00097D6FF1F83C626660547639CE604294796
:1085E0002381E70209472383E7022385E70297D720
:1085F000FF1FA381075097D7FF1FA38E0762B7877E
:108600000040A381070017D7FF1FA307074E0547A8
:108610002383E700B640264496440649F259625A3D
:10862000D25A425BB25B225C925C025DF24D6161A8
:10863000828029472381E70209472383E7022385B4
:10864000E7022387E7022389E70255B717D7FF1F01
:10865000A303F7226FE01FFF854717D7FF1F230BE8
:10866000F72E17D7FF1F2309F73A17D7FF1F230746
:10867000F74617D7FF1F2304F7466FE0BFFE854775
:1086800017D7FF1F2308F72C17D7FF1F2306F7382C
:1086900017D7FF1F2304F74417D7FF1F2301F74401
:1086A00017D7FF1FA308072A17D7FF1FA3060736F0
:1086B00017D7FF1FA304074297D7FF1FA3810742C5
:1086C0008280411106C697000000E78080FBB787D3
:1086D000004023800700130740FC2386E7001307B0
:1086E000C004A386E70017D7FF1F1307A71A239814
:1086F000E70017D7FF1F1307E71D239AE70017D7D7
:10870000FF1F13076729239CE70017D7FF1F1307D5
:10871000E734239EE70029472381E70209472383A3
:10872000E7022385E7022387E7022389E702A38183
:108730000700930600F8A380D700930690022380D9
:10874000D700FD562383D7002381E7009306000559
:1087500037E700E0230BD740B70640002320D710AF
:1087600003C7170013671700A380E700B24097D72D
:10877000FF1F2393073841018280411106C69700ED
:108780000000E78000F0B787004023800700130750
:1087900000FC2386E7003147A386E70017D7FF1FB9
:1087A0001307470F2398E70017D7FF1F13078712F8
:1087B000239AE70017D7FF1F1307071E239CE70024
:1087C00029472381E70209472383E7022385E7023C
:1087D000A3810700930600F8A380D70093069002B8
:1087E0002380D700FD562383D7002381E70093061B
:1087F000000537E700E0230BD740B70640002320F1
:10880000D71003C7170013671700A380E700B24013
:1088100097D7FF1F2392072E41018280F16793872C
:10882000072017D7FF1F2323F72C854717D7FF1FD4
:108830002310F72CA14717D7FF1F230CF72A97D730
:10884000FF1FA388072A97D7FF1F2385072A97D7DB
:10885000FF1F2383070297D7FF1FA38E07008147BF
:1088600017D5FF1F13058501FD5517D6FF1F1306EA
:10887000A6012947B306F5002380B600B306F6002B
:10888000238006008507E397E7FE97D7FF1FA38A9B
:10889000072497D7FF1FA388072497D7FF1F238399
:1088A000072497D7FF1F238E072297D7FF1F238DFB
:1088B000072297D7FF1FA387072297D7FF1F23847D
:1088C0000722814717D6FF1F1306C6334147B30659
:1088D000F600238006008507E39BE7FE828017D71A
:1088E000FF1F0347473585476316F700170300004E
:1088F0006700E3E8170300006700E3DC411122C4CE
:1089000006C617D7FF1F0347073385472E8613F484
:10891000F50FAA856317F70417D5FF1F1305C50BBD
:1089200097600100E780803197D7FF1F2386070EED
:10893000B787004023848702B7E600E0370640008F
:1089400023A0C6180100010003C7A7021377C70FB1
:108950002385E702B240224423A0C610014541010D
:10896000828017D5FF1F1305E5FA97600100E780A5
:10897000E02C97D7FF1F238F07FCB7870040238287
:108980008702B7E600E03706400023A0C6180100C2
:10899000010003C767021377C70F2383E7025DBF98
:1089A000411106C697000000E78080E7B240410110
:1089B000170300006700E3F2411106C697F0FFFFBE
:1089C000E78080BF97D7FF1F83C7D7F8A1CB97D584
:1089D000FF1F83C545F889C917D5FF1F1305C5F7C4
:1089E00097E0FFFFE780403E97D7FF1FA38407F67D
:1089F00097D7FF1F2380071037E700E0B706400036
:108A00002320D71801000100378600408347660203
:108A100093F7370F2303F6022320D710B24041010A
:108A2000828041C9D9C597D7FF1F83C7E70CD1C33F
:108A3000011122CC4AC84EC656C25AC006CE26CA1A
:108A400052C42E89AA890144930A0004371B0300EB
:108A500063772403B3078940C207C183BE8463F4EC
:108A6000FA0093040004C204C180130A1BD497D7F0
:108A7000FF1F83C727EE9DE37D1A631C0A00F240A7
:108A80006244D2444249B249224A924A024B0561A9
:108A9000828097F0FFFFE78020B2D1BF3385890045
:108AA0002694A685420497000000E78060E5418097
:108AB00045B7828097D7FF1F9387871B18429C4337
:108AC00083D645000345070083C5C700035646000B
:108AD0006396A50083D5E700638DD502011106CE0C
:108AE0002386A7002397D700B705CF00DC4B9385DB
:108AF000757D05077D162EC2230001003AC423169A
:108B0000C1002317D10099C30A858297F2400561FD
:108B100082808280DC4DDC4B81CFB7E7040090453A
:108B200003A38705914517D5FF1F0345A5140283AD
:108B300082806D713C083EC6B707E5002322911084
:108B40003EC8AA843C083285232611103ECA23243D
:108B50008110232021112E8997300000E780C06307
:108B60002A8497950100938525A0177501001305A8
:108B7000A57797600100E780C017A28517950100CF
:108B8000130505AF97600100E780A016294597609F
:108B90000100E780E01AB705CB009385757D68007A
:108BA00097100000E780206CA285680097300000D5
:108BB000E780E050014781467000CA8526859720EE
:108BC0000000E780A08F05CD2A849795010093854A
:108BD000A599177501001305257197600100E780BD
:108BE0004011A28517950100130545A99760010062
:108BF000E7802010294597600100E78060148320FA
:108C0000C1100324811083244110032901105161F4
:108C1000828097D7FF1F9387A70518429C437971DD
:108C200022D406D60348070083C807012A8483D6C6
:108C30004500035546006396080183D82701638DDC
:108C4000D8022388070105072399D7003708CC00ED
:108C5000DC4B1308787D3ACC1307F5FF42CA230892
:108C60000100231EE100231FD10099C7080832C666
:108C70002EC482973246A245228597000000E780E5
:108C800080EBB2502254456182806D713C083EC039
:108C9000B707E5003EC23C083EC42326111023243A
:108CA000811023229110231701002318010023199A
:108CB0000100231A0100231B010097A7FF1F83D780
:108CC000277599E3C167FD172316F10097A7FF1FCA
:108CD00083D7277491EB97D7FF1F938767F99C433E
:108CE0009C43DC4783D7070017A4FF1F130444727B
:108CF000584C2317F10083574400484B2318F100C8
:108D000031E1979501009385258D177501001305B5
:108D1000A55D97600100E780C0FD17950100130570
:108D2000E58C97600100E780C0FC29459760010051
:108D3000E78000018320C1100324811083244110A7
:108D40005161828097A7FF1F83C7F76C89EBB7E754
:108D50000400BC5782975C4C23AA0700E1BFFD17B3
:108D600097A6FF1FA389F66A0356070183470401EC
:108D70004C470A85230BF10097300000E780403113
:108D800097D7FF1F9387C7EE9C43014781468843CF
:108D90000A866C0097100000E7804072AA8429C1FF
:108DA0009795010093854583177501001305C553F9
:108DB00097600100E780E0F3A68517950100130591
:108DC000A58397600100E780C0F229459760010004
:108DD000E78000F7584CB7E70400BC57484B9DBFED
:108DE00097A7FF1F83C73763F5D7B7E70400BC4FCA
:108DF0001044854517D5FF1F0345C5E782971DBF62
:108E00005C4EDC4BB9CFB1CD411122C417750100C6
:108E10001305854D2E84978501009385257A06C616
:108E200097600100E780E0ECA2851785010013053B
:108E3000657F97600100E780C0EB294597600100DE
:108E4000E78000F0B7E704002244B24003A387059F
:108E500017D5FF1F034505E2130640069145410162
:108E600002838280411122C417A4FF1F13040458F7
:108E70001C4C06C689C7DC4399C34C488297584CA2
:108E8000B7E70400BC57484B82975C4CB240224481
:108E900023AA07004101828017A7FF1F1307075766
:108EA000834707009306F00B850793F7F70F63E9F5
:108EB000F60097A6FF1F238BF65403450700828018
:108EC000930700F8FDB7835745006386071001112B
:108ED0004AC817A9FF1F1309A95352C4032AC9017D
:108EE00006CE22CC03274A0126CA4EC656C2F157E7
:108EF00035E31307D00DFD57636EC704B7E90400CF
:108F000083A709072A841305860042054181B2849C
:108F1000AE8A8297232AAA000325C9015C49A9E7E2
:108F20009785010093858567177501001305C53B7B
:108F300097600100E780E0DB178501001305C57627
:108F400097600100E780E0DA294597600100E7803B
:108F500020DFDD57F2406244D2444249B249224AFE
:108F6000924A3E850561828093874400B705CF0011
:108F70002319F5009385757D310597100000E78072
:108F8000802E0325C9018345640031059730000018
:108F9000E780E0120325C9012686D6853105973082
:108FA0000000E780E00E7146A2854A8597600100C7
:108FB000E780C0C8504419CA83A78905854517D5DD
:108FC000FF1F034525CB8297814769B797000000B3
:108FD000E780E0CBD5BFFD573E858280411126C298
:108FE00097A4FF1F9384C442D84C22C437E40400E2
:108FF0003C54484B06C68297DC4C0323C4052244EC
:10900000B240924423AA070017D5FF1F034585C627
:10901000854541010283411126C297D4FF1F9384E5
:1090200024C59C4006C622C44AC0D5C3DC43C5C380
:109030005CC12300B5002A849785010093854551C2
:10904000177501001305452A97600100E78060CA83
:10905000294597600100E780A0CE9C4023A407002B
:1090600023A2070097A7FF1F93874738DC4FDC4BED
:1090700091C7295597000000E78000DF97A7FF1FE1
:1090800093870739DC4FDC4B89C797000000E780E6
:1090900020F537E904008327C905894517D5FF1F47
:1090A000034545BD82978327C905914517D5FF1F05
:1090B000034545BC82979C4003A347016309030015
:1090C00022852244B2409244024941010283B240C7
:1090D000224492440249410182800111328506CE28
:1090E00022CC26CA2E8497300000E780E00AAA84AA
:1090F0009785010093850549177501001305C51E65
:1091000097600100E780E0BE030784000356640017
:1091100083554400A686178501001305A552976064
:109120000100E78000BD294597600100E78040C14C
:1091300097A7FF1F83C7E72B639D97000145970003
:109140000000E78060D281450A8597000000E78033
:10915000C0ECF2406244D244056182806D712324E8
:109160008110232611102322911093F745002E849D
:10917000638707143C083EC0B707E5003EC23C08C1
:109180003EC4231701002318010023190100231AEC
:109190000100231B010097A7FF1F83D7272599E311
:1091A000C167FD172316F10097A7FF1F83D7272458
:1091B00091EB97D7FF1F9387A7AB9C439C43DC475A
:1091C00083D7070017A7FF1F130747222317F100B4
:1091D000544F835747002318F100DC4AA1E79785D5
:1091E00001009385653E177501001305E50F976033
:1091F0000100E78000B0178501001305253F976047
:109200000100E78000AF294597600100E78040B387
:10921000134544008320C11003248110832441108E
:109220005161828097A7FF1F83C7B71C2555D9C3FB
:10923000FD1717A6FF1FA30EF61A03D606018347D4
:109240000701CC460A85230BF10097300000E78028
:1092500020E497D7FF1F9387A7A19C4317A7FF1F61
:109260001307C718978601009386463B88430A86F2
:109270006C0097100000E7806024AA8451D997857C
:10928000010093856534177501001305E5059760A6
:109290000100E78000A6A685178501001305C535E6
:1092A00097600100E780E0A4294597600100E7800E
:1092B00020A9268597000000E78000BB91BF93F7A7
:1092C00025009DC7B7E70400BC47414681452808F3
:1092D0008297255597000000E78000B9280893057C
:1092E000F00F97000000E78040D3134524001DB71E
:1092F00093F71500014599DF97000000E78020995A
:109300001345140001BF5C4D411106C688C317D731
:10931000FF1F232FF794B7E7040083A7070817055B
:1093200000001305E5E38297B24097D7FF1F238320
:10933000A79401454101828001113335A000A307A4
:10934000A100B7E7040083A7471706CE1306F10074
:109350008545130550308297F240056182808280F6
:10936000411122C406C697D7FF1F83C72792014425
:1093700089EF97B7FF1F83C7B7EB054499E717B489
:10938000FF1F0344E4EA1344140022859700000001
:10939000E780C0FA178501001305053C09E417852D
:1093A00001001305653C2244B240410117630100EE
:1093B00067002394797122D4A30F010037E40400DD
:1093C0008327841726D24AD006D6AA842E8913056D
:1093D00050309305F10132C6829732468347F1013E
:1093E00093150601C18185CB01452EC6970000006B
:1093F000E780C0F483274417B2454A8626858297C2
:10940000054597000000E78060F3B2502254925463
:10941000025945618280832744174A8626858297B0
:10942000EDB741119397050122C406C626C2C18734
:109430002E8463D40702B7E40400FC5417A5FF1F71
:1094400003450500829719C1BC5482972165218D7F
:10945000B240224492444101828093F715008DC7A7
:10946000B7E7040083A7471A17A6FF1F130646FC99
:1094700097D5FF1F9385C58017A5FF1F034545FCA2
:10948000829713451400E9B793F7250099CFB7E702
:109490000400BC4F13060064894517A5FF1F034550
:1094A00025FA82971345240065B793F7850085CF89
:1094B00097C7FF1F83C7477E85E7B7E7040003A868
:1094C000871A1307401F97A7FF1F83C767F78146B7
:1094D00013064006994517C5FF1F0355657B029883
:1094E00013458400B5B793F745000145B5D3B7E4FC
:1094F000040083A7041817C5FF1F035565798297D9
:10950000BC4C13060064914517A5FF1F034545F3A6
:109510008297134544002DBF97C7FF1F83D7477716
:109520006398A70217C7FF1F2315B77617C7FF1F3A
:109530002312C77617C7FF1F231FD7742E861785E0
:1095400001001305E528BE85175301006700637A03
:109550001785010013054529176301006700439132
:109560000357450097C7FF1F83D78772631EF70411
:10957000C1674111F91722C417C7FF1F232AF770CB
:1095800037E4040097C7FF1F23A6077097C7FF1F84
:10959000A38E076E97C7FF1F238007707C4C06C6FB
:1095A000894517A5FF1F0345A5E982977C4C914586
:1095B00017A5FF1F0345C5E882972244B240410129
:1095C00017030000670003DA178501001305C521A2
:1095D000176301006700C3897D15954763E2A71CE7
:1095E000178701001307C7150A053A951C41011199
:1095F00022CC06CEBA972E848287178501001305E8
:10960000251F97600100E780A086A1A203C725005F
:1096100099476311F7022E8597000000E78080F4D8
:1096200083456400178501001305851D97500100CF
:10963000E780206C97B7FF1F238C07BE17850100BA
:109640001305C51D7DBF03C7250095476319F702A4
:10965000C16717C7FF1F0357A763F91703D5A500F5
:109660006309F702B7E7040083A7C7178297178536
:1096700001001305A51B97500100E780607F854717
:1096800017B7FF1F2306F7BA178501001305851CBE
:109690008DBF97C7FF1F239DA75E83D7E50097C6A1
:1096A000FF1F2398F65E83D7050197C6FF1F2393FC
:1096B000F65E83D7250197C6FF1F239EF65C97C7EA
:1096C000FF1FA385075C631BE502B7E70400BC4FDF
:1096D000096613060690A14517A5FF1F034545D649
:1096E00082970356E4008355A400178501001305F3
:1096F000251597500100E780C05F51B79307700FA1
:109700002316F100B7E7040083A7870D17A6FF1FF4
:10971000034606D36C0082974DF9854717C7FF1F94
:10972000A306F7565DB71785010013056513D1BD74
:1097300083C5250091476392F50217850100130543
:10974000A51397500100E780A07297000000E78002
:1097500060C1F24062440561828099476392F502DC
:10976000228597000000E780E0DF834564001785CD
:1097700001001305E50897500100E7808057D1BF2D
:109780009547639AF50083471400E1F317850100BC
:109790001305C510BDB5178501001305A510E1BF60
:1097A00082800111B7F5070030008146E1051945B7
:1097B00006CE9790FF1FE780C0028347C100034792
:1097C000D100B7562D47A207D98F938676D517A714
:1097D000FF1F130727C814C3B736302D93863603EF
:1097E00054C313D6C70097860100938626FB36968E
:1097F0000345060013D687003D8A3696834506004A
:1098000013D647003D8ABD8B3696B69783C60700B0
:109810000346060097A7FF1F938747C52304A700A9
:10982000A304B7002305C700A305D700230607003C
:109830002385A700A385B7002386C700A386D7008A
:10984000F24005618280411106C697000000E78062
:1098500080F5B7E7040083A7871417A6FF1F130638
:1098600066BFD54501458297B2405D4697A5FF1F6B
:109870009385C5BF130570304101170300006700D1
:10988000A3B361712324811A37E4040083270408F9
:109890002326111A2322911A2320211B232E31194A
:1098A00017050000130525B8829717A9FF1F130994
:1098B00029B9994785442300A900231CF100978505
:1098C00001009385A5EC9307400617750100130569
:1098D000A5A1231CF1082308910097C9FF1F9389B4
:1098E000C9E597500100E780C04083D5090017857E
:1098F00001001305A5E897500100E780803F294546
:1099000097500100E780C04303D50900896997009B
:109910000000E78040E983274417100885451305B8
:10992000503082978327441717A6FF1F130606B4EB
:10993000DD451305703082978327441717A6FF1F54
:10994000130646B0B5451305603082978327441748
:109950003008894513051031829783274417300951
:1099600089451305203182978327441593850990F3
:109970000D45829783274415938509901145829759
:10998000A30591002306910002CD23080100230CBA
:109990000100832784163009914513057040829792
:1099A000832784161306B10085451305004082976E
:1099B00083278416700085451305104082978327FE
:1099C0008416300885451305204082978327841626
:1099D00010088545130550408297832704157D554F
:1099E0008297832744137D5582977D5597A0FFFF6B
:1099F000E780A0C98327440C829797A0FFFFE780E8
:109A000000A58327841417A6FF1F1306A6A4D54517
:109A10000145829789471306700F8145280923065F
:109A2000F1009780FFFFE780806E8D4713060008E6
:109A300081452808230CF1089780FFFFE780206DFF
:109A40009147230CF100976701009387677B984348
:109A500083C747003AC8230AF10097D0FFFFE78089
:109A6000009470008545054597A0FFFFE78000C979
:109A700030099305700F094597A0FFFFE78000C8E4
:109A80003008930500080D4597A0FFFFE78000C749
:109A900010089545114597A0FFFFE78020C6C167D4
:109AA00017C7FF1F1307C71EF9171CC32322070080
:109AB00017A5FF1F1305859897A0FFFFE780E0C259
:109AC0008327C41D17C5FF1F1305051B82973C483C
:109AD00003450900854582978320C11A0324811A12
:109AE0008324411A0329011A8329C1195D618280E7
:109AF000C16717C8FF1F0358A819F9176301F808B1
:109B00003DCDB5CD011126CAB7E4040083A7841268
:109B100022CC2E862315B10006CE2A840147814629
:109B2000ED45428582972AC611ED17850100130580
:109B300025C897500100E780A033F2406244D24428
:109B400005618280FC440356A100A28582972C0007
:109B500017C5FF1F0355C51397A0FFFFE780A0C5DA
:109B600069DD178501001305E5C597500100E78001
:109B7000203083A7C412ED45280082977DBF8280E4
:109B80000DC5854717A7FF1FA303F78C97A7FF1FD6
:109B90002380078C354697A5FF1F9385A58A13055B
:109BA0006030170300006700238197A7FF1FA38081
:109BB000078AE9BF97C7FF1F83C7070EA9EFC167D1
:109BC00017C7FF1F0357C70CF9176306F7044111A6
:109BD000854722C417C7FF1F2300F70C37E4040092
:109BE0007C4C06C6A14517A5FF1F034565858297D6
:109BF0000323841A2244B24097A7FF1F83C74784D8
:109C000017C5FF1F0355C5081307401F814631467E
:109C100099454101028382806D712324811023269E
:109C2000111023229110328401CD8947630AF50275
:109C30008320C1100324811083244110516182804C
:109C4000178501001305C5C6AE8497500100E78053
:109C50002022A285268597C0FFFFE7804093C9BFD9
:109C6000B7E70400FC472800829717850100130519
:109C7000E5C497500100E780A01F8347810039C4E5
:109C80001307000B6380E7021387A7051377F70F0D
:109C90008D4663EDE602A285280097C0FFFFE780AE
:109CA000000379B78547E3F587F883459100177579
:109CB00001001305A594B335B00097A7FF1F2381BA
:109CC000B74097500100E780C0029DB7034791005D
:109CD000A207D98F35671307D7556385E7086368EF
:109CE000F7022D671307B7556387E7063167130738
:109CF000C755638AE70429671307A7556394E702EA
:109D0000A285280097C0FFFFE780603B15B7396741
:109D10009306E7656381D70863E9F6001307E75503
:109D20006384E706A28528003DB73D679306F75593
:109D3000638AD7061307F766E396E7FE97C0FFFF2F
:109D4000E7808054F5B50146A285280097C0FFFF43
:109D5000E7808023F1BDA285280097C0FFFFE78040
:109D60004034F9B58947E3F587EC97000000E780B8
:109D7000A0E49305E4FFC205C1811305A1009790FB
:109D8000FFFFE780E0456DB5A285280097C0FFFF83
:109D9000E780E03371BDA285280097C0FFFFE78010
:109DA000A03E79B597C0FFFFE780C04751B5C167B6
:109DB00017C5FF1F0355C5EDF9176307F500B7E792
:109DC000040003A3C71702838280854717C7FF1FBC
:109DD000230EF7EA014517F3FFFF670023561783A9
:109DE000FFFFE702232E2A8408452E89B28919C96C
:109DF00000C1971500009385A58661059730010085
:109E0000E780400281447D5A97100000E780E039E6
:109E100063C7A404814497100000E780003A63C838
:109E2000A40497C7FF1F938767E79C43DC47B307EA
:109E3000F94091872302F400638309048327C90052
:109E4000B307F4409587A302F4001C4C89C79C47D4
:109E500099C3228582971783FFFF6700E3295C443B
:109E6000139714008504BA972390470171BF1C48CB
:109E7000139714008504BA972390070069BF8327BE
:109E800089000547B307F4409587A302F400835780
:109E90000400638EE7028DC309476384E7040D471E
:109EA000E395E7FA97870100938707F41CCC97871F
:109EB0000100938767F411A897870100938747BA39
:109EC0001CCC978701009387A7BA5CC8BDBF978752
:109ED00001009387E7A51CCC97870100938747A6CD
:109EE000EDB7978701009387E7F41CCC97870100B3
:109EF000938747F5D9BF95E51783FFFFE702231E38
:109F0000004618448347940075839D8B6317F700C0
:109F100097100000E78060B448C41783FFFF670014
:109F2000431E82801783FFFFE702C31913893500A0
:109F3000C16442094111AA890144F114135909016C
:109F4000054A2EC697100000E7802026B2456348D8
:109F5000A400014541011783FFFF6700E31983A7B0
:109F6000090013171400BA9783D707006388B70056
:109F70006394970063742A010504E1B70545D9BFCE
:109F80001783FFFFE7022313AA892E89328BB68439
:109F90003A8ABE8A97A00000E780E0FB71C9268557
:109FA00097200000E780E0098D4763E7A7007D5513
:109FB0001783FFFF6700A31383DB440097100000A3
:109FC000E780A0242A8497100000E78040259307AB
:109FD000740031443305850263CDA7029710000059
:109FE000E780A02297100000E78020222A849710A3
:109FF0000000E780C02293077400314433058502D6
:10A0000063C3A70497100000E78020209307450052
:10A0100029A897100000E7808020330585021307E8
:10A02000F0179307C017E35FA7FA2D55E3C277F93E
:10A0300063040B02D6865286A6854A8597200100C6
:10A04000E780E0BAB5B797100000E780401D330500
:10A0500085029307C5FFD1BF832749001385C90037
:10A0600083D5270097000000E78000EC61F581B7F9
:10A0700069553DBF97C7FF1F2394A7C297C7FF1F0E
:10A080009387C7C1904381470C463307F5004207C9
:10A0900041836393B7008280544613984700850735
:10A0A000C2962390E600D5B797C7FF1F938707BFD7
:10A0B0009C4303C58700828017C5FF1F035545BE1B
:10A0C00082801783FFFFE7028301C1671387D7FFF1
:10A0D000630BE502636AA700F1176300F50201450F
:10A0E0001783FFFF6700E3011387E7FF6302E502C1
:10A0F000FD171D8D13351500E5B797500000E7805B
:10A1000080277D15C5BF97500000E78000FCD5BFB4
:10A1100097500000E78020FAEDB71783FFFFE702B2
:10A1200003FC4111AA8401442EC697100000E78069
:10A13000C008B2456348A400014541011783FFFFF1
:10A14000670023FC9C48131514003E9583570500B7
:10A15000E385B7FE0504C9BF03485500814693F760
:10A16000F60F63E5070181473E8582805845939746
:10A170005600BA9703D727006316B70003D7070026
:10A18000E304C7FE8506E1BF834645000147937798
:10A19000F70F63E4D700814711A81C451316570039
:10A1A0000507B29703D60700E313B6FE3E8582800B
:10A1B0001783FFFFE70203F193170501C18797CAD1
:10A1C000FF1F938AAAAD635BF00883A70A00C0470C
:10A1D0009C4703570400198D420541816368F500CF
:10A1E000014422851783FFFF670003F112052A94BB
:10A1F000CDBFDC4713944900014A3E948347440095
:10A200006341FA02014A834754006349FA0285090F
:10A21000C20993D9090183A70A009847E3EBE9FC37
:10A22000C1B71C4413195A00A6853E994A85970068
:10A230000000E780C0EE05E1050AC9B75C441319C8
:10A240005A00A6853E994A8597000000E78020EDD8
:10A2500019E1050A4DBFE30C09FA61B7AA848149E7
:10A260005DBF1783FFFFE70283E71C452A8481E770
:10A270009307C5001CC51C44231204001CC093078F
:10A28000F00F63EDB70093F5F50F228597200000DE
:10A29000E780E0E21783FFFF6700A3E693940501E0
:10A2A000C167C18063F9F500A6852285972000006B
:10A2B000E78000E6C5B7C18193F5F50F22859720A9
:10A2C0000000E780C0DFA685228597200000E78098
:10A2D00000E1C9B797C7FF1F9387479C88438280D7
:10A2E0001C4599C797C7FF1F23AAA79A01458280DB
:10A2F0007D55828097C7FF1F9387479A984383476E
:10A300004500484792073E9582801783FFFFE7028A
:10A3100003DD617100451C183EC6B70780013EC8C9
:10A320001C183ECA8357440002CE02D002CC231E22
:10A33000F100834784002A8902D22301F1023C08FC
:10A340003ED402D697000000E78000FB835705004B
:10A350002316F10297500000E78020C52307A102D1
:10A360005C4003556400F18313F717008347F10243
:10A3700052055181F99BD98FA307F1029710010073
:10A38000E780407639CDAA840355050097A00000E8
:10A39000E78040BD83D704002AD26800231CF10067
:10A3A00083D72400231DF1001C4803D647008C43AB
:10A3B00097200000E780C0CD8347B400CA86177697
:10A3C0000100130666508117A305F4006C004810C5
:10A3D00097200100E780A0815D611783FFFF670080
:10A3E00043D22155D5BF1C45B1CF03C5A70089462F
:10A3F00013576500630BD7028D46630ED70285465F
:10A400006300D702130740063305E50203C7B70010
:10A41000418B15CB83C7B700BD8B3355F540828088
:10A420001375F5031307803EC5B709671375F50368
:10A4300013070771D1BF372709001375F5031307F9
:10A44000077CD9B7014582801783FFFFE70223C944
:10A4500003A98500630C09048347B900AE8493F710
:10A46000070E85C303459900930520030D8105055B
:10A47000B305B5028844610597300100E780A0AAC2
:10A4800035A02E8597000000E78020F62A8419CD9C
:10A4900097000000E780605C8325C900B307B540E2
:10A4A00063FA87002E94B305A440E9F51783FFFFF4
:10A4B000670023C585457DBF1783FFFFE70223C2E1
:10A4C0002A8403D50500011132C636C43AC22EC013
:10A4D00002CA02CC02CE97A00000E780A0A8824565
:10A4E0002ACA22852ECC97000000E780E0E00357BF
:10A4F0000500231EE10097500000E78000ABA24654
:10A5000032469247230FA10036874C08B286228537
:10A51000014697000000E780E0A605611783FFFF72
:10A52000670023BE1783FFFFE70263BB61711C183E
:10A530003EC6B70780013EC81C183ECA3C0800450D
:10A540003ED4AA8402CC02CE02D002D202D6970018
:10A550000000E78060DA8357050035592316F102C1
:10A5600097500000E78060A42307A10209C4835725
:10A57000440081EB21594A855D611783FFFF670025
:10A5800043B8035564005205518197100100E780DC
:10A5900060552A8965D18347B40093F7070E99C7A0
:10A5A0001305840197300100E780209A8357440007
:10A5B000231EF100834784002301F1025C40035510
:10A5C0000900D98313F7070883471102231CA10050
:10A5D00093F7F707D98FA300F10283572900231DB2
:10A5E000F1005C40F18313F717008347F102F99BF8
:10A5F000D98FA307F10297A00000E780A0962AD286
:10A6000035D9834794006800139757008347B400F7
:10A61000FD8BD98FA305F4001C4803D647008C435B
:10A6200097200000E780C0A6A687177701001307D0
:10A63000A729740005464C10268597000000E78086
:10A6400060942A890DD98347B400A685FD8BA305A4
:10A65000F40097000000E78060DF31BF1783FFFF41
:10A66000E702E3A7832485FE2A844111268597000B
:10A670000000E78080D7834734FF93F7070E8DCB28
:10A680002AC6268597000000E78060C809CD834769
:10A6900034FFB245FD8BA309F4FE91C522859730A6
:10A6A0000100E780408841011783FFFF670063A531
:10A6B0007DD98327C4FF2685829775F5834734FFAC
:10A6C00093F7070E91C7228597300100E780E08756
:10A6D000032584FE97000000E78000E5E9B71783B3
:10A6E000FFFFE702C39C9C4141112A8903C7070071
:10A6F00089472E84935667006380F6040D4663886D
:10A70000C6049307F0076304F7022E859720000024
:10A71000E78080A8AA848149C16B130C490097B7D0
:10A72000FF1F9387A7579C43984763E4E9044101BF
:10A730001783FFFF6700639B03D745008547E3F856
:10A74000E7FE2E8597200000E78060AAE1B703D7D7
:10A750004500E3FEE7FC2E8597200000E780C0A3BC
:10A76000AA84228597200000E78020A5C204C98C16
:10A770005DB7DC470355A900139A49003E9A931729
:10A780000501C187635DF00083570A006397A70244
:10A7900063E774038327CA00034D5A002DA0A16705
:10A7A0002167A98F1307F7EFE374F7FE639709009A
:10A7B00097000000E780209161FD85098DB7832710
:10A7C0008A00034D4A00835DA90003576900216A8E
:10A7D000138BC7003AC6814A33CA4D01631E5D011F
:10A7E00097B7FF1F9387074C9C43E1DBA2866286E5
:10A7F000814526858297D1B7A1679387F7EF930CA0
:10A800004BFF63F24703B2455A8597F0FFFFE7809D
:10A81000A0710DC103278B00104709CE104363823E
:10A82000C4023107D5BFEE85668597000000E7803A
:10A83000008F71F993861A0093FAF60F130B0B022F
:10A8400071BF835644005C43E3E9F6F622853AC6BD
:10A8500097100000E780407EA1679387D7042A8A7B
:10A86000035D4400324763E897008347D90093E7CC
:10A8700007F8A306F9001C4766852286E2858297C1
:10A88000C1670844FD17337AFA00529508C02312B5
:10A89000A40125B797B7FF1F938747409843814787
:10A8A00015C31447814763FFD500939745004C4774
:10A8B000BE9519C903C7550081476375E600DC459D
:10A8C0001606B2973E85828003C745008147E37B29
:10A8D000E6FE16069C45F5B71773FFFFE702837E79
:10A8E000AA892E8A814497BAFF1F938A2A3B83A79D
:10A8F0000A00984763E6E4001773FFFF6700C37F11
:10A90000DC471394440001493E9413BB1400834771
:10A910004400634BF900014913BB14008347540002
:10A92000634FF9008504E1B7084493175900528733
:10A93000DA860146A2853E9582990509C9BF484439
:10A94000931759005287DA860546A2853E9582996B
:10A950000509E9B71773FFFFE7026378814517F52B
:10A96000FFFF1305054897B7FF1F239B073297008A
:10A970000000E780A0F61773FFFF6700837897B7A2
:10A98000FF1F9387A7319C4395C31773FFFFE7020F
:10A990000375814517F5FFFF1305A54497000000D7
:10A9A000E780C0F31773FFFF6700A37582801773FA
:10A9B000FFFFE702237137E404008327841241116B
:10A9C0002315E100AE893289368A3A8681460147ED
:10A9D000ED45AA8482972AC621C90356A100D285D3
:10A9E00097400100E78080258327C413CE85268504
:10A9F0008297058905C98327440D23142101014647
:10AA00002C00268582972A8401C9B7E7040083A712
:10AA1000C712ED4528008297228541011773FFFF79
:10AA20006700836D4944D5B76554FDB75C41FD1798
:10AA30005CC182801773FFFFE702636AB7E7040017
:10AA4000FC5F829795473305F50281450D811773A9
:10AA5000FFFF6700036B1773FFFFE7024368B7E769
:10AA60000400FC5F829795473305F5020D8117734B
:10AA7000FFFF670003691773FFFFE7024366B7E74D
:10AA8000040083A7870B0355050082971773FFFF08
:10AA9000670023671773FFFFE70263640355050030
:10AAA0003287AE861796FF1F0356A6A297B5FF1FE3
:10AAB0009385851F97000000E780A0EF1773FFFFC5
:10AAC000670023641773FFFFE7026361B7E70400C1
:10AAD00083A7C71782971773FFFF670083621773F7
:10AAE000FFFFE702C35FB7E7040083A7871397B5AB
:10AAF000FF1F9385651B829701451773FFFF670052
:10AB000043601773FFFFE702835DB7E7040083A785
:10AB1000C71F81451795FF1F0355A5978297177388
:10AB2000FFFF6700035E1773FFFFE702435BB7E7B2
:10AB3000040083A7871397B5FF1F9385E5178297B6
:10AB400001451773FFFF6700C35B1773FFFFE70241
:10AB50000359B7E7040083A7C71F81451795FF1F57
:10AB60000355259982971773FFFF67008359177361
:10AB7000FFFFE702C3562E8597800000E780A0B054
:10AB800097800000E780A0ED1773FFFF6700635711
:10AB90001773FFFFE702A35497800000E780A0F738
:10ABA0001773FFFF6700E3555C49E1175CC95CC59B
:10ABB00083572501A1072319F50083570501A10734
:10ABC0002318F5008280F1473305F50297B7FF1F80
:10ABD000938787109C433E9582808D476315F608C6
:10ABE00003D74600854763F0E7081773FFFFE702C6
:10ABF000034F368536842E8997100000E780C059B0
:10AC000029C98357440093140501C18063E3970465
:10AC1000228597100000E7802058FD14231294002D
:10AC20009307A0026300F5029307B0026307F502E1
:10AC300093079002631FF500228597000100E780CB
:10AC4000808601A80146CA85228597A00000E7807A
:10AC500020B11773FFFF6700C34A228597100000D9
:10AC6000E7808004FDB7828097B6FF1F93860607B2
:10AC70009C42014599CF9843D44217B6FF1F232F1A
:10AC8000E6046396D70097B6FF1F23ABE60413854F
:10AC9000C7FE82801773FFFFE7026344970000003E
:10ACA000E780A04B714433058502914597900000E1
:10ACB000E780E0E911E565551773FFFF670063441E
:10ACC00097B7FF1F23A8A70097000000E780E04880
:10ACD00033058502914597900000E78040E761DDEC
:10ACE00097B7FF1F23AAA7FE97000000E780E04662
:10ACF00097B7FF1F239AA7FC97000000E780E04565
:10AD000097B7FF1F2393A7FC97770100938707C18D
:10AD100017B7FF1F232EF7FA97070000938707E95D
:10AD200017B7FF1F2324F7FA014579B71773FFFF01
:10AD3000E702E33AAA8517B5FF1F1305E5F8971058
:10AD40000000E780805C1773FFFF6700833B177389
:10AD5000FFFFE702C33897000000E78060FD97100F
:10AD60000000E780005C97B7FF1F938727F79C439D
:10AD700091CF1387C7FE19CB83D5C7FF17B5FF1F28
:10AD8000130545F697200100E780E0191773FFFFD0
:10AD9000670023371773FFFFE70263349700000053
:10ADA000E780C0EC09CD834785002A8493F7070428
:10ADB00099EB0355E50097000000E78080F91773D1
:10ADC000FFFF670003348347C5009304450117B9AB
:10ADD000FF1F1309A9F085E3832709005CC997B712
:10ADE000FF1F23AD97EE83274900F1FB97B7FF1FA5
:10ADF00023A897EEE9B7FD172306F50061059780B4
:10AE00000000E78080D78307840063CB0704834773
:10AE1000840093E707F82304F400B7E704009C5F7D
:10AE200082974205A94741813375F5028347840023
:10AE300093F707FCC98F2304F4008347D4003E95A1
:10AE40001C402318A40089CF984319CB8347C40022
:10AE50005040814585073305F5024205418102973F
:10AE6000832709005CC897B7FF1F23A997E68327AC
:10AE7000490089E797B7FF1F23A497E68347C400DB
:10AE80009DDF8355040117B5FF1F1305A5E5972026
:10AE90000100E780400925B71773FFFFE70223246D
:10AEA00097B7FF1F938747099C4701448583858B8C
:10AEB00085E3AE84B2853A8697100000E780404C67
:10AEC0002A8419C597100000E7808042829408CC3C
:10AED00022851773FFFF6700C3221773FFFFE70286
:10AEE000631E41112E8932C6AA8997000000E780AF
:10AEF000C031324713060502CA86970500009385C4
:10AF0000C5CC17B5FF1F130525DC97000000E780AF
:10AF1000E0F82A8425C99304C50097000000E78063
:10AF2000E0411946AA85268597100000E780401663
:10AF30008545268597100000E780201217750100CF
:10AF40001305859B4E9583450500268597100000C7
:10AF5000E780E0165C4831468145A1075CC85CC4C7
:10AF600083572401E1172319F40083570401E117E3
:10AF70002318F4001C4C3E859770FFFFE7802019D2
:10AF8000A3042501228541011773FFFF6700C31643
:10AF90001773FFFFE702A3144111AA842EC632C41F
:10AFA00097100000E7802037004DB24522468347C6
:10AFB00084000CC050C093F7F70393E70704230401
:10AFC000F40023180400268597100000E780403223
:10AFD00083479400A9462317A40013D73700050719
:10AFE0003307D7029D8B85072306F400A306E400F0
:10AFF00083C70401D8488507230FF7FE17B7FF1F43
:10B000001307C7CD5843232A04009307440129E3BB
:10B0100017B7FF1F2326F7CC17B7FF1F2320F7CC46
:10B0200017B4FF1F130404CC228597200100E7808A
:10B03000C0E11C44858B5D8D19E5814522859720F3
:10B040000100E78040EE41011773FFFF6700630BCB
:10B050001CC317B7FF1F2325F7C8D9B71773FFFF06
:10B06000E702E30797050000938565B70145970060
:10B070000000E78000B001451773FFFF6700630819
:10B080001773FFFFE702A30597000000E78080B079
:10B090001773FFFF6700E3068347C500A5E3177337
:10B0A000FFFFE702C3032A840355E5009700000071
:10B0B000E78000C821C18347840093F7F7FB23048E
:10B0C000F4001C4091C7DC4381C74C400145829786
:10B0D00097000000E78080B917B5FF1F130585C0F2
:10B0E00097200100E78060E60355E4009700000028
:10B0F000E78020C61773FFFF6700A30082801773E5
:10B10000FFFFE702C3FD97B7FF1F938727BD970592
:10B110000000938565C817B5FF1F1305A5BC23A0C4
:10B12000070023A2070097200100E780A0CF177334
:10B13000FFFF670003FD1C4D91CFDC4381CF1773E8
:10B14000FFFFE702C3F98345070082971773FFFFEC
:10B15000670023FB828097B7FF1F9387E7BA9C4362
:10B1600003C50700828097B7FF1F9387E7B99C4309
:10B1700003C51700828097B7FF1F9387E7B89C43EA
:10B1800003C52700828097B7FF1F9387E7B79C43CB
:10B1900003C54700828097B7FF1F9387E7B69C439C
:10B1A00003C53700828097B7FF1F9387E7B59C439D
:10B1B00003C55700828097B7FF1F9387E7B49C436E
:10B1C00003C56700828097B7FF1F9387E7B39C434F
:10B1D00003C57700828097B7FF1F9387E7B29C4330
:10B1E00003C58700828097B7FF1F9387E7B19C4311
:10B1F00003C59700828097B7FF1F9387E7B09C43F2
:10B2000003C5A700828097B7FF1F9387E7AF9C43D2
:10B2100003C5B70011E11D45828097B7FF1F9387D3
:10B22000A7AE9C4303C5C700828097B7FF1F9387D3
:10B23000A7AD9C4303C5D700828097B7FF1F9387B4
:10B24000A7AC9C4303C5E700828097B7FF1F938795
:10B25000A7AB9C4303D50701828097B7FF1F938755
:10B26000A7AA9C4303C52701828097B7FF1F938736
:10B27000A7A99C4303D54701828097B7FF1F9387F7
:10B28000A7A89C4303D56701828097B7FF1F9387C8
:10B29000A7A79C4303D58701828097B7FF1F938799
:10B2A000A7A69C4303C5A701828097B7FF1F93877A
:10B2B000A7A59C4303C5B701828097B7FF1F93875B
:10B2C000A7A49C4303C5C701828097B7FF1F93873C
:10B2D000A7A39C4303C5D701828097B7FF1F93871D
:10B2E000A7A29C438857828097B7FF1F9387C7A167
:10B2F0009C4303D5C702828097B7FF1F9387C7A0DF
:10B300009C4303D5E70219E11305800C828097B7AF
:10B31000FF1F9387679F9C4303C50703828097B7EE
:10B32000FF1F9387679E9C43C85B828097B7FF1F70
:10B330009387079D8843828097B7FF1F9387879CD9
:10B340008843828019E17D558280F5DE984265DF71
:10B35000FDD917B7FF1F130727BE1847AA877155D6
:10B36000058B631D072403C507001547E37DA7FC74
:10B3700003C737001305F0057D171377F70FE36454
:10B38000E5FC03C35700E30003FC83C86700E38CBC
:10B3900008FA03C77700494579171377F70FE36475
:10B3A000E5FA03C7A70011481305F7FF1375F50F5A
:10B3B000E36BA8F803CE97000D481305FEFF137545
:10B3C000F50FE362A8F803C8B70063090800651821
:10B3D0001378F80F1305600DE36705F703C5C70081
:10B3E000794879151375F50FE36FA8F403C8D700F2
:10B3F0000D457D181378F80FE36705F503D80701AD
:10B40000930E40175118420813580801E3ED0EF34C
:10B4100003C8E7007D181378F80FE36605F303C847
:10B4200027017D181378F80FE36F05F103C8870033
:10B43000C54E75181378F80FE3E70EF103D86701CE
:10B44000856E938EBEE06D18420813580801E3EC38
:10B450000EEF03D847016D18420813580801E3E4C2
:10B460000EEF03D887017918420813580801E36CDE
:10B4700005ED03C8A7017D181378F80FE36505ED06
:10B4800003C5B7011D487D151375F50FE36DA8EAD7
:10B4900003C5D701714879151375F50FE365A8EA5F
:10B4A00003D5E7011308E00F7D1542054181E36CE8
:10B4B000A8E803C50702494879151375F50FE36439
:10B4C000A8E8C85301C937C834005915130858BF34
:10B4D000E36BA8E603A8870237C53400130555BF00
:10B4E0005918E36205E717B5FF1F232DC58003C672
:10B4F000050117B5FF1F2329F5800545E375C5E450
:10B5000003D82501D04933760603E31E06E203C6BD
:10B510001501E30A06E217A6FF1F2323B67E83C5A3
:10B52000270001466387A50003C61700F1453306CF
:10B53000B60283C707039305C00272971A07130761
:10B54000C70516031A9796084697B387B702415561
:10B550003E973297420741836362E8061773FFFF05
:10B56000E702E3B7368597800000E78060699700BF
:10B570000100E780E0482A8497A00000E780405B54
:10B580002A9497F00000E78020272A9497900000E3
:10B59000E78060822A9497F0FFFFE780E06F2A94AB
:10B5A00097400000E78020942A9497700000E7807D
:10B5B000609D22951773FFFF6700A3B48280177305
:10B5C000FFFFE702C3B14111A307A10097A000004C
:10B5D000E78060C69305F100170500001305E5B587
:10B5E00097F0FFFFE780802F014541011773FFFFB0
:10B5F000670023B11773FFFFE702E3AB17B4FF1F28
:10B60000130484930328840079599368180097B42D
:10B61000FF1F23A714931378180063100802BA843D
:10B62000BE89368B328A2E89AA8A97F0FFFFE7807F
:10B63000E0A77D15269519E531594A851773FFFF57
:10B640006700E3AA97F0FFFFE78040A67D152695E7
:10B65000A167E353F5FE97B7FF1F9387A7C49843ED
:10B660003E8C814B01CB014597F00000E780E04420
:10B67000933B15004A85DA865686D285979000005E
:10B68000E780804E2A8911CD1C44F99B17B7FF1F14
:10B690002328F78A83270C00CDD3E3800BFA829707
:10B6A00069BF268597B7FF1F23AA078897F0FFFF7A
:10B6B000E780809C4146CE8517B5FF1F1305459155
:10B6C00097300100E780805797D00000E780009A0C
:10B6D0000325040B97D00000E780C09D054597D057
:10B6E0000000E780C0A4054597000000E78060EDFA
:10B6F000A9B797B7FF1F938727849C47858BEDC712
:10B700001773FFFFE702A39D17B5FF1F1305858A77
:10B7100097B7FF1F23A2078297B7FF1F23A00782B7
:10B7200097B7FF1F23AE078097200100E780E081D5
:10B7300097500000E780A0F697100100E780604D69
:10B7400097100100E780605397A7FF1F9387477DFD
:10B750009C4391C7054597800000E780002197A78B
:10B76000FF1F9387A7659C4399C741657D15977017
:10B770000000E78000A397F00000E780A03E97D08C
:10B780000000E780409097B7FF1F9387A78F9C43E7
:10B79000139717016356070097F00000E780C0ADCC
:10B7A00097B7FF1F23A6078297B7FF1F23A407821F
:10B7B00097B7FF1F23A2078297B7FF1F23A0078217
:10B7C00097000000E780008C97000000E780C072BF
:10B7D00097F0FFFFE780401897F00000E78000D760
:10B7E0001773FFFF6700E391828097A7FF1F93877E
:10B7F000A7748843828097A7FF1F9387E773C84386
:10B8000082801773FFFFE702838D97800000E78037
:10B81000607597800000E780C0771773FFFF6700AF
:10B82000438E1773FFFFE702E3892A84930414020F
:10B8300001112E85B289A685214636C63A899730F0
:10B840000100E780403D0DE9B24638082686CE85E6
:10B850001305940497500000E780604121462C08AE
:10B860004A8597300100E780003B133515000561DC
:10B870001773FFFF670043880145D5BF1773FFFFAC
:10B88000E702E3859305450617A5FF1F1305054845
:10B8900097100100E78020691773FFFF6700638638
:10B8A0001773FFFFE702A38341112EC697F0FFFF36
:10B8B000E780A01AB24588C141011773FFFF6700F6
:10B8C00043841763FFFFE702E37FAA842E849780F7
:10B8D0000000E780006CAA8985452285970000005A
:10B8E000E780E07D83C7E4011389940899E3138915
:10B8F0000403CE85228597000000E780407C214626
:10B9000093051902228597000000E780607897A7C9
:10B91000FF1F938767628C43228597100000E780A2
:10B92000C082214693858402228597000000E7802B
:10B9300020761763FFFF6700237C1763FFFFE70292
:10B940008377397197F00000E780E0B493054006F3
:10B9500061E997800000E78000606302051497A703
:10B96000FF1F83C7673C13B7170097A6FF1F238DE0
:10B97000E63A014499CFC16417A9FF1F1309C95BB7
:10B980009309400EFD1497000000E7800086634293
:10B99000A40A97F0FFFFE780400C4169B72909002E
:10B9A000096AFD7A2A8B81447D199389F97B130AF0
:10B9B0000A71938A8AC797000000E780008363D7E3
:10B9C000A4041304400EB387840217A7FF1F1307B4
:10B9D000A7560324070B3E948357C4016382270BA9
:10B9E00018403307EB4063EAE900834744008507CA
:10B9F000B3874703D6976365F70801468145094534
:10BA000097F0FFFFE780A04DAA8B29E59740000043
:10BA1000E780808385476317F506896593850571FF
:10BA200017A5FF1F1305852E97100100E780A04F73
:10BA300095A0B30734030327090BBA9703D7C701AF
:10BA40006308970003C75700A38207002382E7001B
:10BA5000050415BF9305C500228597000000E78007
:10BA600080E65E85228697650100938525EA97F03A
:10BA7000FFFFE78020525E8597100000E780608A14
:10BA8000850415BF97A7FF1F9387074B9C478D839E
:10BA9000858BC1F721611763FFFF6700436501468E
:10BAA0008545094502D002D202D402D697F0FFFFA5
:10BAB000E780E042AA8479DD97F00000E780E09C0F
:10BAC0001389C4002A8481454A8597000000E780D5
:10BAD000005F0C4041464A8597000000E780405BCC
:10BAE000832944006385090C4E8502D802DA02DC02
:10BAF00002DE97300100E780E0382ACE14100546B8
:10BB00002C0808184ECC97500000E780E00A137507
:10BB1000F50F51ED8355840093E525004A85970084
:10BB20000000E780E05E11460C104A859700000097
:10BB3000E78000560146976501009385A5DD2685BF
:10BB400097F0FFFFE7800045268597000000E7801B
:10BB5000407D5C40A1D3014685450D4597F0FFFF30
:10BB6000E780E037AA841DD548401389C400973088
:10BB70000100E78020312AC64A8597000000E7804F
:10BB8000404C3246636FC5004C404A859700000028
:10BB9000E780005001468145268597F0FFFFE7804A
:10BBA000603F268597000000E780A077E5B58355C4
:10BBB0008400ADB71763FFFFE702635297A7FF1F2B
:10BBC000938787379C471DC193E7870017A5FF1F01
:10BBD0001305C51317A7FF1F2324F736971001007D
:10BBE000E78040321763FFFF6700A351DD9B17A773
:10BBF000FF1F2327F73497300000E780E0647DF1D2
:10BC000017A5FF1F1305851097100100E780E0338B
:10BC1000D1BF1763FFFFE702034A4169AA892E8A51
:10BC2000B28A368BBA8B814417ACFF1F130CCC3011
:10BC3000930C400E7D1997F0FFFFE780005B63C413
:10BC4000A40001443DA03384940383270C0B3E944D
:10BC50008357C401638627055A87D6865286CE85C8
:10BC60001305040397000000E780E0BB01C92380AF
:10BC70000B0022851763FFFF670063478347F401CA
:10BC800085C35A87D6865286CE85130594089700B9
:10BC90000000E78040B909C585472380FB00D1BF7C
:10BCA000850451BF835745006380071E1763FFFF5C
:10BCB000E702434101112A8497000000E780C04D4C
:10BCC00009C985476309F50605611763FFFF67002A
:10BCD000A34297E00000E780007C7DF58357440095
:10BCE0004947ED9BE392E7FEC1452285970000009E
:10BCF000E7804033AA84228597000000E780204F28
:10BD00000357440002CE91472A89631AF70022851F
:10BD100097000000E780A0513C082ACC3ECE97E077
:10BD20000000E78080765C55C5D374084A86A685F6
:10BD30000545829751BF03574400D147E3F6E7F822
:10BD4000032A0400C169014997AAFF1F938ACA1EEA
:10BD5000130B400EFD1997F0FFFFE7800049634F7A
:10BD6000A90E2285032A040097000000E780C04244
:10BD7000A1452A89228597000000E780A02AAA848D
:10BD8000228597000000E780804A14402A86AA890D
:10BD900078082685CA8597000000E780C0E7AA8456
:10BDA00005D503C7F40189476315F7008347C1012F
:10BDB00081DF5546D2851385640097300100E78006
:10BDC000E0E7014597800000E780C01901C583D7EF
:10BDD000C401A5E797A7FF1F938707169C479355B4
:10BDE0001900858913D73700058B01CF8983858B8F
:10BDF0006399B70001452EC697000000E780C0DBBD
:10BE0000B2454E8597800000E780601F0346C10160
:10BE10002A8493751900268597900000E780E03901
:10BE200035C1268597800000E780E018268511C07F
:10BE3000014597800000E780004C97300000E780C4
:10BE4000A0408547E312F5E883C754001307F00FBD
:10BE5000E38CE7E68507A382F400BDB5B30469036C
:10BE600083A70A0BBE9483D7C401638B3701554661
:10BE7000D2851385640097300100E780C0D955DD75
:10BE80000509D1BD5DD86DB782801763FFFFE7025A
:10BE9000632397800000E780000C05C1C164014462
:10BEA00017A9FF1F130949099309400EFD1497F0C4
:10BEB000FFFFE7808033634EA40017A5FF1F130523
:10BEC000E5E497100100E780E0031763FFFF6700D8
:10BED000A322330534038327090B3E958357C501FD
:10BEE000638897002312050097800000E780A00C6C
:10BEF000050475BF97A7FF1F938707049C478D8391
:10BF0000858B8DE31763FFFFE702631D17A5FF1FF6
:10BF10001305C5DF97100100E78020031763FFFFBB
:10BF20006700231E82801763FFFFE702431B97050C
:10BF300000009385C5A017A5FF1F130525DD9710E9
:10BF40000100E78020EE1763FFFF6700831B176384
:10BF5000FFFFE702C3188841B7E70400BC5B050593
:10BF600042054181829709C585472300F5000505F3
:10BF70001763FFFF6700E31883C7F5FF2E8585076A
:10BF8000A38FF5FE828083C7F5FFFD1793F7F70FA8
:10BF9000A38FF5FE99EF1763FFFFE7024314B7E79E
:10BFA0000400BC571385F5FF82971763FFFF6700F6
:10BFB000431582801C41035745008D8FBA951CC1E3
:10BFC0002312B5003E85828093D78500A2051441D7
:10BFD000DD8D835745001387E6FF18C189072312BB
:10BFE000F50013D685004111238FB6FEA38FC6FE40
:10BFF0004101828018419307F7FF1CC18357450018
:10C0000085072312F500A30FB7FE828083574500F2
:10C010008D8F2312F5001C41BE950CC12E858280A8
:10C02000AA8703D7470008410D8FAA952392E700FE
:10C030008CC38280184108453305A740828083570E
:10C040004500035765001D8F1C4108453385A740F7
:10C050003305A74082801763FFFFE70243084111C1
:10C060002EC62A8497000000E780A0FDB2456373C6
:10C07000B50001A0835744000840BE952312B400C8
:10C080003E9541011763FFFF6700A3071763FFFF9A
:10C09000E702E30441112E84B28532C69700000006
:10C0A000E780A0FB3246A28597300100E78000B907
:10C0B00041011763FFFF6700C3041763FFFFE70237
:10C0C00003022E84854597000000E78000F92300D5
:10C0D00085001763FFFF6700C3021763FFFFE702D6
:10C0E000030041112317B100894597000000E78044
:10C0F000C0F68347E1002300F5008347F100A30069
:10C10000F50041011763FFFF6700A3FF1763FFFFFF
:10C11000E702E3FC93D78500A2054111DD8D2317CB
:10C12000B100894597000000E78020F38347E100D4
:10C130002300F5008347F100A300F50041011763D8
:10C14000FFFF670003FC1763FFFFE70243F9139744
:10C15000850193D78501C166938606F0D98F13D7E1
:10C160008500758FD98FA2053707FF00F98D411122
:10C17000DD8D2EC6914597000000E78000EE6C0033
:10C18000114697300100E78060AB41011763FFFF64
:10C19000670023F71763FFFFE70263F41C4185453F
:10C1A00003C4070097000000E78080E6228517633C
:10C1B000FFFF670003F51763FFFFE70243F21C412F
:10C1C0004111894503C7070083C717002307E10012
:10C1D000A307F10097000000E78080E30355E1002A
:10C1E00041011763FFFF6700C3F11763FFFFE70219
:10C1F00003EF1C414111894503C7070083C717009E
:10C200002307E100A307F10097000000E78040E06A
:10C210008357E100410113D58700A2075D8D4205D8
:10C2200041811763FFFF6700C3ED1763FFFFE7025C
:10C2300003EB0C4141112A8411466800973001003C
:10C24000E780C09F9145228597000000E78040DC91
:10C25000B247C166938606F01397870113D587010D
:10C26000598D13D78700758F598DA2073707FF00A7
:10C27000F98F5D8D41011763FFFF670083E81C455F
:10C28000BE950CC18280AE87944391E6584101EF80
:10C290000CC15CC1828003C7570013671700A382DB
:10C2A000E700B687D5B70CC3EDB7AA87084119CD0B
:10C2B0001841D44398C36313D500D8C32A870346D3
:10C2C00057009376160081E623200700828094436E
:10C2D00081CA8C4203A847008CC363930601CCC378
:10C2E000799A14C3A302C7003687D1BF1C45DC4727
:10C2F0001D8DB777DBB6938777DB09853305F502AC
:10C30000420541818280F147B385F50248452E956B
:10C3100082808347450085072302F50082801763EA
:10C32000FFFFE702C3DB2A8409E41763FFFF67000E
:10C3300043DD83474400F5DBFD1793F7F70F230236
:10C34000F400E5F71C4403D7270005072391E70015
:10C35000DC4399C3228582974C4889CD834754009A
:10C36000898B99E71C4422859C479C439C47829774
:10C37000232A04000040232004007DB71763FFFF39
:10C38000E702E3D58357250041112EC681EB014416
:10C39000228541011763FFFF6700A3D603570500FD
:10C3A0008147F146E305F7FEB385D702404585078F
:10C3B0002E948345440008C4F5F5B247AA8481E76A
:10C3C000232A040009A81C456C0022859C439C4339
:10C3D000829748C84DDD85472312F400B2472320D9
:10C3E0000400231804002319F4005C485CC483D7BC
:10C3F0002400FD172391F40061BF1763FFFFE702DC
:10C4000003CE97A7FF1F93876792884323260500D3
:10C4100023240500410597100100E78000B317634E
:10C42000FFFF670003CE1763FFFFE70243CB17A4AC
:10C43000FF1F1304A48F1C40411199CF9C47230078
:10C44000B5002AC65CC197000000E78040FB1C4095
:10C45000DC4399C33245829741011763FFFF6700B0
:10C4600043CA0347450029E3584DAA877D551DCF90
:10C470001763FFFFE702A3C61CC3DC4797A6FF1F95
:10C4800023A6E68AF156130507012390D7009705E6
:10C4900000009385050297100100E780A0980145F0
:10C4A0001763FFFF6700E3C57D55828082801763B5
:10C4B000FFFFE702C3C20111614681452800976072
:10C4C000FFFFE780C0C497A7FF1F938727869C4381
:10C4D00028009305F00FDC473EC697000000E78078
:10C4E000C0F405611763FFFF6700A3C197A7FF1F93
:10C4F0009387C7839C43D847A1679387C702631E6E
:10C50000F70A397106DE22DC26DA80004AD84ED6D8
:10C5100052D456D23285B28497000000E780C0C75B
:10C52000AA89268597000000E78020C92318A4FC6B
:10C53000268597000000E78040C82319A4FC2685C3
:10C5400097000000E78060C783D744000A8A231A57
:10C55000A4FC858393F7F70F230EF4FC8607BD0731
:10C5600093F7073F3301F1408A8A01498347C4FDAD
:10C570006367F902CE85130584FC232C54FD9700D4
:10C580000000E78080EA5281130104FCF2506254FB
:10C59000D2544259B259225A925A21618280268538
:10C5A00097000000E78060C193171900D69705092E
:10C5B0002390A7001379F90F55BF82809797FF1F2B
:10C5C0009387C7769C43D847A1679387A702631ACE
:10C5D000F70A397106DE22DC26DA80004AD84ED608
:10C5E00052D456D23285B28497000000E780C0BA98
:10C5F000AA89268597000000E78020BCFD572318F4
:10C60000A4FC26852319F4FC97000000E780E0BA1B
:10C6100083D744000A8A231AA4FC858393F7F70F73
:10C62000230EF4FC8607BD0793F7073F3301F14063
:10C630008A8A01498347C4FD6367F902CE851305E1
:10C6400084FC232C54FD97000000E78000DE52811B
:10C65000130104FCF2506254D2544259B259225A86
:10C66000925A21618280268597000000E780E0B41D
:10C6700093171900D69705092390A7001379F90F8E
:10C6800055BF82809797FF1F9387476A9C43D8477F
:10C69000A16789076310F70A397106DE22DC26DA02
:10C6A00080004AD84ED652D456D23285328997006D
:10C6B0000000E78060AEAA894A8597000000E78005
:10C6C000C0AF835749000A8A2318A4FC858393F7D7
:10C6D000F70F230CF4FC8607BD0793F7073F3301E0
:10C6E000F1408A8A8144834784FD63E7F402CE8562
:10C6F000130584FC232A54FD97000000E780E0D254
:10C700005281130104FCF2506254D2544259B2597E
:10C71000225A925A216182804A8597000000E78060
:10C72000C0A993971400D69785042390A70093F48B
:10C73000F40F55BF82809797FF1F9387275F9C4315
:10C74000D847A1679387E704631EF70A397106DEAD
:10C7500022DC26DA80004AD84ED652D456D2328510
:10C76000B28497000000E78020A3AA89268597005D
:10C770000000E78080A42318A4FC26859700000011
:10C78000E780A0A3231AA4FC268597000000E78079
:10C79000C0A283D744000A8A2319A4FC858393F797
:10C7A000F70F230EF4FC8607BD0793F7073F33010D
:10C7B000F1408A8A01498347C4FD6367F902CE8547
:10C7C000130584FC232C54FD97000000E780E0C58E
:10C7D0005281130104FCF2506254D2544259B259AE
:10C7E000225A925A21618280268597000000E780B4
:10C7F000C09C93171900D69705092390A7001379B9
:10C80000F90F55BF82809797FF1F938727529C434C
:10C81000D847A1679387C704631AF70A397106DE00
:10C8200022DC26DA80004AD84ED652D456D232853F
:10C83000B28497000000E7802096AA892685970099
:10C840000000E7808097FD572318A4FC2685231A53
:10C85000F4FC97000000E780409683D744000A8AE2
:10C860002319A4FC858393F7F70F230EF4FC8607A6
:10C87000BD0793F7073F3301F1408A8A0149834797
:10C88000C4FD6367F902CE85130584FC232C54FD97
:10C8900097000000E78060B95281130104FCF25058
:10C8A0006254D2544259B259225A925A216182801A
:10C8B000268597000000E780409093171900D697CF
:10C8C00005092390A7001379F90F55BF8280979728
:10C8D000FF1F9387A7459C43D847A167DD076317D0
:10C8E000F7041753FFFFE702837F797132853284A3
:10C8F00097000000E780408A2AC622859700000042
:10C90000E780A08B2311A102228597000000E78019
:10C91000A088B2452300A102280897000000E78004
:10C92000C0B045611753FFFF6700A37D82809797D2
:10C93000FF1F9387A73F9C43D847A167938787042E
:10C940006317F7041753FFFFE702637979713285A4
:10C95000328497000000E78020842AC62285970051
:10C960000000E78080852311A10222859700000046
:10C97000E7808082B2452300A102280897000000CA
:10C98000E780A0AA45611753FFFF67008377828085
:10C990009797FF1F938787399C43D847A167938751
:10C9A000A7046312F7021753FFFFE7024373011155
:10C9B0002800814597000000E78020A705611753F4
:10C9C000FFFF6700037482809797FF1F93870736E6
:10C9D0009C43D847A167938757026319F7021753FF
:10C9E000FFFFE702C36F0111328597F0FFFFE78079
:10C9F000A07A2308A1008145280097000000E78065
:10CA0000C0A205611753FFFF6700A36F828097974D
:10CA1000FF1F9387A7319C43D847A1679387E702FD
:10CA2000631BF7041753FFFFE702636B01113285A5
:10CA3000328497F0FFFFE7804078AA84228597F040
:10CA4000FFFFE7808077854709E9228597F0FFFFA0
:10CA5000E78080744205B337A00028008145231881
:10CA600091003ECA97000000E780209C05611753A3
:10CA7000FFFF6700036982809797FF1F9387072B4B
:10CA80009C43D84799476313F7081753FFFFE70202
:10CA9000036579713285328497F0FFFFE780C06FBC
:10CAA0002AC6228597F0FFFFE78020712310A1029C
:10CAB000228597F0FFFFE780206E2301A1022285E7
:10CAC00097F0FFFFE780406DA301A102228597F058
:10CAD000FFFFE780606C2302A102228597F0FFFF31
:10CAE000E780806B2313A102228597F0FFFFE78088
:10CAF000A06AB2452314A102280897000000E7802D
:10CB0000C09245611753FFFF6700A35F828097972C
:10CB1000FF1F9387A7219C43D847A1679387C7032B
:10CB20006313F7081753FFFFE702635B79713285E0
:10CB3000328497F0FFFFE78020662AC6228597F0AF
:10CB4000FFFFE78080672310A102228597F0FFFF97
:10CB5000E780A0662311A102228597F0FFFFE780FE
:10CB6000A0632302A102228597F0FFFFE780C06245
:10CB7000A302A102228597F0FFFFE780E061230373
:10CB8000A102228597F0FFFFE7800061B245A30371
:10CB9000A102280897000000E7802089456117530B
:10CBA000FFFF6700035682801753FFFFE7022353FE
:10CBB00001112A8497F0FFFFE780005EAA84228596
:10CBC00097F0FFFFE780605F228597F0FFFFE78027
:10CBD000C05E035744008D4763F7E700228597F056
:10CBE000FFFFE780805D228597F0FFFFE780E05C34
:10CBF0002800A68597000000E78020830561175371
:10CC0000FFFF670003509797FF1F938727129C43EE
:10CC1000D847A167FD07631FF7001753FFFFE7021F
:10CC2000034C328597000000E78040F81753FFFF60
:10CC30006700234D82809797FF1F9387270F9C43A0
:10CC4000D847A167E5076315F7081753FFFFE70209
:10CC5000034979713285328497F0FFFFE780C05332
:10CC60002AC6228597F0FFFFE7802055228597F09E
:10CC7000FFFFE78080542310A102228597F0FFFF79
:10CC8000E780A053520551812311A102228523027E
:10CC9000010297F0FFFFE7802050A302A102228546
:10CCA00097F0FFFFE780404F2303A102228597F012
:10CCB000FFFFE780604EB245A303A102280897F06A
:10CCC000FFFFE780807645611753FFFF67006343EE
:10CCD00082809797FF1F938767059C43D847A1677A
:10CCE0009387E703631FF7001753FFFFE702233F14
:10CCF000328597000000E78060EB1753FFFF670065
:10CD0000434082809797FF1F938747029C43D847F1
:10CD1000A16793874704631EF7021753FFFFE702DB
:10CD2000033C79713285328497F0FFFFE780C0467B
:10CD30002AC6228597F0FFFFE7802048B2452808E1
:10CD400097F0FFFFE780606E45611753FFFF6700B4
:10CD5000433B82809797FF1F938747FD9C43D847AB
:10CD6000A167938787026310F7041753FFFFE70259
:10CD7000033779713285328497F0FFFFE780C04135
:10CD80002AC6228597F0FFFFE7800041B2452300C5
:10CD9000A102280897F0FFFFE7802069456117533B
:10CDA000FFFF6700033682801753FFFFE70223333C
:10CDB000011197F0FFFFE780203EAA85280097F039
:10CDC000FFFFE780806605611753FFFF670063334D
:10CDD0009797FF1F938787F59C43D847A167D10793
:10CDE000631FF7001753FFFFE702632F3285970099
:10CDF0000000E780A0FB1753FFFF670083308280AD
:10CE00009797FF1F938787F29C43D847A167C50771
:10CE1000631FF7001753FFFFE702632C328597006B
:10CE20000000E780A0F81753FFFF6700832D828082
:10CE30009797FF1F938787EF9C43D847A167B90750
:10CE4000631FF7001753FFFFE7026329328597003E
:10CE50000000E780A0F51753FFFF6700832A828058
:10CE60009797FF1F938787EC9C43D847A167AD072F
:10CE7000631FF7001753FFFFE70263263285970011
:10CE80000000E780A0F21753FFFF6700832782802E
:10CE90009797FF1F938787E99C43D8478947631873
:10CEA000F7021753FFFFE70283230111328532C8CF
:10CEB00097F0FFFFE780402EAA85280097F0FFFF3C
:10CEC000E780A05605611753FFFF67008323828028
:10CED0009797FF1F938787E59C43D847A1678D07E6
:10CEE0006311F7041753FFFFE702631F0111328537
:10CEF000328497F0FFFFE780202A13066100AA849E
:10CF00004C00228597300000E780C0232800A685CA
:10CF100097F0FFFFE780605105611753FFFF67003F
:10CF2000431E82809797FF1F938787E09C4381CFA2
:10CF3000DC4391CB1753FFFFE702631A8297175325
:10CF4000FFFF6700031C82801753FFFFE7022319CE
:10CF500079713C08AE843ED2A165B7070A002A84E5
:10CF60003ED448103C08DD053ED636C432C63AC22F
:10CF700097D0FFFFE780202F12474810BA8597F01F
:10CF8000FFFFE780C01332464810B28597F0FFFFDD
:10CF9000E780E014A2464810B68597F0FFFFE780CF
:10CFA0000012501001478146A685228597D0FFFFC9
:10CFB000E780C05045611753FFFF67008314175384
:10CFC000FFFFE702C31101117C000329C501AE84F4
:10CFD0003ECAA165B70707002A843ECC48087C00FA
:10CFE000C5053ECE97D0FFFFE780E0278345D900F7
:10CFF000480897F0FFFFE780800C50080147814602
:10D00000A685228597D0FFFFE780404B0561175327
:10D01000FFFF6700030F1753FFFFE702430C83C7AF
:10D02000950093F7F707A384F50097000000E780C9
:10D0300040F91753FFFF6700C30C1753FFFFE702C8
:10D04000030A79713C08AE843ED2A165B707090096
:10D050002A843ED448103C08938545043ED632C607
:10D0600036C497D0FFFFE7800020A2464810B6855F
:10D0700097F0FFFFE780A00432464810B28597F092
:10D08000FFFFE780C005501001478146A685228535
:10D0900097D0FFFFE780804245611753FFFF67008D
:10D0A00043061753FFFFE702830383C7950041112F
:10D0B0002A8493F7F707A384F50032852EC697F0EC
:10D0C000FFFFE780800F85672AC46370F5029770C1
:10D0D0000000E78020E92246B24509ED114781466C
:10D0E000228597000000E78060E641011753FFFFAB
:10D0F0006700230101478346F501DDB71753FFFFA2
:10D10000E70243FC01113C003ECAB7070A003ECCCF
:10D110003C003ECE83C79500AA89328593F7F70776
:10D12000A384F5002E8497F0FFFFE7800009856750
:10D13000637DF504A165AA8493858504480897D08A
:10D14000FFFFE7804012268597700000E78080E1AE
:10D150002A8929E19145480897F0FFFFE78020F6EA
:10D16000A685480897F0FFFFE78060F7CA85480862
:10D1700097F0FFFFE780A0F4014781465008A285A1
:10D180004E8597D0FFFFE780603305611753FFFF9F
:10D19000670083F68145480897F0FFFFE78020F29B
:10D1A0000349090275BF1753FFFFE702A3F1797125
:10D1B0001C103ECAB7070F003ECC404D1C10AA847D
:10D1C000AE894808994532C636893ECE97D0FFFFD2
:10D1D000E780600932464808B28597F0FFFFE78094
:10D1E00000EE630C0902A545480897F0FFFFE780B1
:10D1F000C0E62546CA8597200100E78020A4500894
:10D2000001478146CE85268597D0FFFFE780002B1A
:10D2100045611753FFFF670023EE8355C40248089A
:10D2200097F0FFFFE780A0EB0355E402814505C5B9
:10D23000854785456301F502C167FD179305F00F2A
:10D24000630BF5007D1597700000E780208E930535
:10D25000150093F5F50F480897F0FFFFE78020E6EB
:10D2600083450403480897F0FFFFE78040E58345C6
:10D270001403480897F0FFFFE78060E48355240318
:10D28000480897F0FFFFE78080E58355440348088E
:10D2900097F0FFFFE780A0E49DB71753FFFFE70279
:10D2A00003E483C795008146014693F7F707A384FB
:10D2B000F50097000000E78040EF1753FFFF67007D
:10D2C00043E41753FFFFE70283E179713E841C10AA
:10D2D0003ECA2E89B7070F00A1653ECCFD051C1084
:10D2E000AA84480842C03AC23ECE36C432C697D05D
:10D2F000FFFFE78040F732464808B28597F0FFFF0E
:10D30000E780E0DBA2464808B68597F0FFFFE7809C
:10D3100000DD12474808BA8597F0FFFFE78020DC60
:10D320000248630C08029145480897F0FFFFE78028
:10D33000C0D21146A28597200100E78020905008B6
:10D3400001478146CA85268597D0FFFFE7800017F1
:10D3500045611753FFFF6700C3DA8945480897F016
:10D36000FFFFE78080CF834704002300F500834759
:10D370001400A300F500E1B71753FFFFE70283D4C1
:10D3800083C7950001112A8A93F7F707A384F50054
:10D390003285AE8432C697F0FFFFE78000E2324666
:10D3A0002A89328597F0FFFFE78000DF8567637386
:10D3B000F902AA894A8597700000E780A0BA2A84FA
:10D3C00019ED114781464A86A685528597000000CF
:10D3D000E780C0B705611753FFFF6700E3D193876C
:10D3E000E9FF93F7F70F0547E366F7FE8347F5017B
:10D3F00095EB8947E380F9FE8346F40152850147A6
:10D400004A86A68597000000E78040B4A167D90747
:10D4100048083ECC230A010002CE97000000E780B6
:10D42000A0B04DBF639EE7008947639EF900930754
:10D430001020231FF50097700000E780C0B76DBF74
:10D440000947E39BE7FA8D47E398F9FA228597703D
:10D450000000E78080DF9797FF1F938767AC9C43AE
:10D4600099E79797FF1F938767959C4399C703D5C3
:10D47000040097800000E780A0CE231F04002285CF
:10D480005DBF1753FFFFE70283C501113C003ECA91
:10D49000B7070B003ECC3C003ECE83C795002A89DF
:10D4A000328593F7F707A384F500AE8497F0FFFF6A
:10D4B000E780A0D093170501C187635AF006A165E4
:10D4C0002A849385E502480897D0FFFFE780A0D91A
:10D4D000A285480897F0FFFFE78060C09797FF1F7D
:10D4E0009387C78D9C43A9EB01449375F40F4808BB
:10D4F00097F0FFFFE780A0BC9355844093F5F50FAC
:10D50000480897F0FFFFE78080BB9355044193F5EF
:10D51000F50F480897F0FFFFE78060BA01478146A2
:10D520005008A6854A8597D0FFFFE78020F905615E
:10D530001753FFFF6700E3BC416585460546A2859A
:10D540007D1597500000E78060BD59DD51059700BB
:10D550000100E780808F130440063344850271B7D1
:10D560001753FFFFE702A3B70111B70706003EC636
:10D5700083C7950021642A8993F7F707A384F500F0
:10D58000AE8428009305A4040AC40AC897D0FFFFFC
:10D59000E78060CD300001478146A6854A8597D057
:10D5A000FFFFE780A0F197E0FFFFE780C0141304BE
:10D5B0009404480822CC230A010002CE9700000000
:10D5C000E780809605611753FFFF670083B3175309
:10D5D000FFFFE70223AFC1642A8901449799FF1F27
:10D5E00093898995130A8002FD1497E0FFFFE78075
:10D5F000C0C06347A40001451753FFFF6700C3AFD6
:10D60000B307440303A7C90ABA9703D70700630601
:10D61000970083D72700638427010504F9B70545E0
:10D62000E1BF1753FFFFE702E3A92A8A2E8999C1B8
:10D6300023A0050081498144978AFF1F938A8A6F3E
:10D64000614B97E0FFFFE78080C163C7A4004E8570
:10D650001753FFFF670043AA3384640383A70A00BC
:10D660003E948357040099E763040900232089004E
:10D670008504C1BF4146D2851305440097100100BF
:10D68000E780605975F5A289E5B71753FFFFE702F8
:10D6900063A339717C083ED4B7070A003ED67C08E4
:10D6A0003ED883C795002A8A328593F7F707A3846B
:10D6B000F5002E8932C697F0FFFFE78000B085673E
:10D6C0006373F5083246AA84328597F0FFFFE7803E
:10D6D000A0AC8547AA8963E8A706A1659385850460
:10D6E000281097D0FFFFE78000B8268597700000CC
:10D6F000E78040872A8429ED9145281097F0FFFFA5
:10D70000E780E09BA685281097F0FFFFE780209D2B
:10D71000CE85281097F0FFFFE780609A0147814689
:10D720003010CA85528597D0FFFFE78020D9A167C6
:10D730009387770448183EDC230A010202DE97F043
:10D74000FFFFE780607E21611753FFFF6700C39AE8
:10D750008145281097F0FFFFE7806096A685281086
:10D7600097F0FFFFE780A0979797FF1F938747B336
:10D770009C4381CB22856389090097D00000E78014
:10D7800040248345040271B797D00000E780C0228F
:10D79000CDBF1753FFFFE702E39283C79500411106
:10D7A000AA8993F7F707A384F5003285AE84328AFD
:10D7B00097F0FFFFE78060A08567637FF5022A8905
:10D7C00097600000E780007A2A84914631C583473C
:10D7D000F50105476387E70291C70D476366F704C4
:10D7E000AD461DA89305050303250A004146971081
:10D7F0000100E78040420DE941011753FFFF670038
:10D80000A38F9305950803250A0041469710010050
:10D81000E7806040814669F54A86A6854E85970077
:10D820000000E780C081C9BF83250A001305940862
:10D8300097700000E780A02919C1C146F1BF978702
:10D84000FF1F9387E76D9C4399E79787FF1F938797
:10D85000E7569C4399C7228597800000E780208A7D
:10D8600069FD8547A30FF400228597B00000E7808B
:10D870006084228597600000E780E0734E858146D2
:10D880004A86A68597F0FFFFE780607BA1679387B4
:10D89000570448003EC42302010002C697F0FFFF70
:10D8A000E780806891BF1753FFFFE702C38083C7FB
:10D8B00095004111AA8993F7F707A384F5003285F3
:10D8C0002E89B28A97F0FFFFE780208F8567637407
:10D8D000F50EAA8497600000E780C0682A840DEDE9
:10D8E000416B014A978BFF1F938B0B65130C400E06
:10D8F0007D1B19A833048A0383A70B0B3E9483571F
:10D90000C40163836705050A97E0FFFFE780E08DA8
:10D91000E342AAFE95460DA08357C5016396970280
:10D920009305050303A50A00414697100100E7800F
:10D93000802E994611E181462686CA854E8597F04C
:10D94000FFFFE780C06F85A883A50A0013050403C5
:10D9500097700000E780A017C14679FD2285231E3D
:10D96000940097A00000E780E07422859760000093
:10D97000E78060649797FF1F938787929C43A9C3B2
:10D9800023000402228597D00000E78040F04E85F6
:10D9900081462686CA8597F0FFFFE780406AA16727
:10D9A0009387070448003EC42302010002C697F093
:10D9B000FFFFE780605741011743FFFF67002373B4
:10D9C00089472300F402E1B7397106DE22DC4AD828
:10D9D000800052D456D25AD026DA4ED65ECE2E8A47
:10D9E00032892A8B97D0FFFFE780207D06057105DD
:10D9F00041998A8A3301A140232224FC231404FC88
:10DA000097D0FFFFE780607B83479A0006053505C6
:10DA100093F7F7072315A4FCA304FA004A852326ED
:10DA200024FC97E0FFFFE780407993170501C18749
:10DA30006340F0025681130104FCF2506254D25448
:10DA40004259B259225A925A025BF24B21618280AA
:10DA5000AA844A8597E0FFFFE7802076AA894A8555
:10DA600097E0FFFFE7806075A1659385C5022A896D
:10DA7000130544FC97C0FFFFE780E07E268597C032
:10DA8000FFFFE7802073854511C94A86CE8597C080
:10DA9000FFFFE780A06CAA8B21E98945130544FCB0
:10DAA00097E0FFFFE780A061A685130544FC97E09F
:10DAB000FFFFE780C062CE85130544FC97E0FFFFBF
:10DAC000E780E061CA85130544FC97E0FFFFE7802B
:10DAD000006101478146130644FCD2855A8597D0E0
:10DAE000FFFFE780A09DB9B78145130544FC97E08F
:10DAF000FFFFE780C05CA685130544FC97E0FFFFAD
:10DB0000E780E05DCE85130544FC97E0FFFFE780EA
:10DB1000005DCA85130544FC97E0FFFFE780205CA9
:10DB2000814497D0FFFFE7804069E3D4A4FA83A73C
:10DB30000B0113971400BA9783D5070099C51305F5
:10DB400044FC97E0FFFFE78080598504D9BF7971D5
:10DB500006D622D44AD000184ECE52CC56CA26D26F
:10DB60005AC8AE893289AA8A97D0FFFFE780E0645D
:10DB70000605690541990A8A3301A140232A24FC3C
:10DB8000231C04FC97D0FFFFE780206383C7990024
:10DB900006052D0593F7F707231DA4FCA384F900C0
:10DBA0004A85232E24FC97E0FFFFE780006193174E
:10DBB0000501C187634FF0005281130104FDB2508B
:10DBC000225492540259F249624AD24A424B456168
:10DBD0008280AA844A8597E0FFFFE780005EA16506
:10DBE0009385A5022A89130544FD97C0FFFFE780AE
:10DBF0008067268597C0FFFFE780C05B854509C920
:10DC0000CA8597C0FFFFE78060582A8B29E18945C4
:10DC1000130544FD97E0FFFFE780604AA6851305E2
:10DC200044FD97E0FFFFE780804BCA85130544FD64
:10DC300097E0FFFFE780A04A01478146130644FDB5
:10DC4000CE85568597D0FFFFE7804087B5B78145E1
:10DC5000130544FD97E0FFFFE7806046A6851305A6
:10DC600044FD97E0FFFFE7808047CA85130544FD28
:10DC700097E0FFFFE780A046814497D0FFFFE78051
:10DC8000C053E3DBA4FA83270B0113971400BA9760
:10DC900083D5070099C5130544FD97E0FFFFE78092
:10DCA00000448504D9BF1743FFFFE702434383477E
:10DCB0004500404DD5EFFD575DC4834694000947AC
:10DCC0006363D70A0346B400854663EEC60883063D
:10DCD000E40063CA06085C45F9562390D70097878D
:10DCE000FF1F83C7670599E3A304E4009787FF1F1D
:10DCF0009387C70C9C4381E78947A306F400978765
:10DD0000FF1F9387E7599C4381E789472306F40067
:10DD10009705000093854506AA841305040197F032
:10DD20000000E7802010FD57231AF40281471CDC15
:10DD300001489787FF1F23AD87FE9787FF1F9387B3
:10DD400067FF232E040304C0804397D0FFFFE780C2
:10DD5000005161463306C502814522859740FFFF89
:10DD6000E780E03A81473E851743FFFF670063394C
:10DD7000FD57D5BF1743FFFFE70263362A840355DB
:10DD8000450297600000E780E01D19E5231E0400AE
:10DD90001743FFFF6700E3368357E401F5DB930584
:10DDA00004FF174501001305A5F097E00000E78088
:10DDB000E014F9BF1743FFFFE70263322E89A16524
:10DDC00041119385E5032A8436C432C6BE843AC223
:10DDD00097C0FFFFE780204912472285BA8597E068
:10DDE000FFFFE780C02D32462285B28597E0FFFF16
:10DDF000E780E02EA2462285B68597E0FFFFE78008
:10DE0000002E630309029145228597E0FFFFE7801A
:10DE1000C0241146A68597100100E78020E2410149
:10DE20001743FFFF6700E32D8945228597E0FFFF39
:10DE3000E780A02283C704002300F50083C71400F5
:10DE4000A300F500E9BF1743FFFFE702432983C79B
:10DE50009500444D054793F7F707A384F5001C424E
:10DE6000411183C707006367F7062E842A89B1C072
:10DE700003C7D400630FF7021787FF1F130707F4C8
:10DE8000184305C3A386F40097A00000E780404A2A
:10DE900083C7D40099E741657D1597400000E7806E
:10DEA000403083D72403918B89C797E00000E78037
:10DEB000C0134A85A28597F0FFFFE7808010A16715
:10DEC000C10748003EC42302010002C697F0FFFFCD
:10DED000E780800541011743FFFF67008322174356
:10DEE000FFFFE702C31F03D745008D47AA844111F6
:10DEF0002E8432892E8563E3E70297E0FFFFE780F7
:10DF0000C02BAA8523000900268597C0FFFFE78064
:10DF1000E02741011743FFFF6700A31E97E0FFFFC3
:10DF2000E780A0292AC6228597E0FFFFE780E02846
:10DF3000B24585472A862300F900268597C0FFFF52
:10DF4000E780C021F9B7397106DE22DC26DA8000CD
:10DF50004ED652D456D24AD85AD05ECEAE89B2846A
:10DF6000AA8A97D0FFFFE780402406051305250203
:10DF700041990A8A3301A140232224FC231404FC82
:10DF800097D0FFFFE780602283C7990006054D0503
:10DF900093F7F7072315A4FCA384F900268523260D
:10DFA00024FC97E0FFFFE780402193170501C1871C
:10DFB0006340F0025281130104FCF2506254D254C7
:10DFC0004259B259225A925A025BF24B2161828025
:10DFD000AA8B03AB040097C0FFFFE780A01D51E5AB
:10DFE00083D7440001498544F11793B71700A30173
:10DFF000F4FC834734FCA165C9C79385E504130588
:10E0000044FC97C0FFFFE7800026A685130544FC6B
:10E0100097E0FFFFE780A00ADE85130544FC97E048
:10E02000FFFFE780C00B834734FC114691E30946AC
:10E03000DA85130544FC97E0FFFFE7806005814423
:10E04000630A0900416B7D1B97D0FFFFE780E01555
:10E0500063CCA40201478146130644FCCE85568555
:10E0600097C0FFFFE7808045B1B7A685130634FC53
:10E0700097000000E780E0E6933415002A898604C3
:10E080008DBF9385C504A5BF8327C90013971400CE
:10E09000BA9783D5070063886501130544FC97E0B0
:10E0A000FFFFE780C003850445B71743FFFFE70282
:10E0B000830079711C103EC4B7070F003EC61C10C8
:10E0C0003EC883C79500AA8A328593F7F707A384D1
:10E0D000F500AE89328497E0FFFFE780000E9317CA
:10E0E0000501C187635AF0062A8A228597E0FFFF5F
:10E0F000E780A00C2A895285032B040097C0FFFFFC
:10E10000E780400B39ED8357440081440544F11703
:10E1100093B71700A303F10083457100DA872287C4
:10E12000CA865286280097000000E780E0C80147B1
:10E1300081463000CE85568597C0FFFFE7800038C6
:10E14000A1679387D70348083ECC230A810026CED7
:10E1500097F0FFFFE78040DD45611743FFFF670051
:10E1600003F9A2851306710097000000E78060D7CD
:10E17000AA84094455D13544E30055FB4A8597F0FC
:10E18000FFFFE78000450D4441D9014497D0FFFFD0
:10E19000E780A001634DA400C16B0144FD1B97D033
:10E1A000FFFFE7808000634EA4001544B5B7DC4450
:10E1B00013171400BA9783D7070063832703050456
:10E1C000F1B7D84493171400BA9703D70700631B1D
:10E1D000770123902701268597A00000E78080DB48
:10E1E00001441DBF050465BF1743FFFFE70283ED30
:10E1F00083C7950041112A8A93F7F707A384F50096
:10E2000032852E89328497E0FFFFE78000FB931769
:10E210000501C1876353F006AA89228597E0FFFFB5
:10E22000E780A0F92311A1004E85832A040097C03E
:10E23000FFFFE78020F839E5835744008544014417
:10E24000F11793B71700A300F1000348110003571B
:10E250002100D6875285CE862686CA8597F0FFFF95
:10E26000E7806006A167F10748003EC423029100E1
:10E2700022C697F0FFFFE78020CB41011743FFFF45
:10E28000670083E7A2851306110097000000E7806E
:10E2900040C52A84894455D9835721001167854494
:10E2A000BA97C2071167C1831307F7EFE36FF7F857
:10E2B0009787FF1F9387C7C69C4381CB854513056E
:10E2C000210097500000E7802075835521002285AA
:10E2D000814497C0FFFFE78080E425D92310050023
:10E2E000228597A00000E78040CD85B71743FFFF48
:10E2F000E70263DC83C7950041112A8B93F7F70788
:10E30000A384F50032852E8A328497E0FFFFE780F0
:10E31000C0EA93170501C1876351F006AA8A2285D6
:10E3200097E0FFFFE78060E92A895685832B040088
:10E3300097C0FFFFE78000E831E583574400814440
:10E340000544F11793B71700A301F100034831000A
:10E35000DE875A854A87D6862286D28597F0FFFFC8
:10E36000E78060F6A167ED0748003EC42302810004
:10E3700026C697F0FFFFE78020BB41011743FFFF50
:10E380006700E3D6A2851306310097000000E780FE
:10E3900040B5AA8409445DD99167CA97C20711673D
:10E3A000C1831307F7EF0544E362F7FACA8597C004
:10E3B000FFFFE780C0D6014451F9814997D0FFFFA4
:10E3C000E780A0DF63DBA900984893971900BA970C
:10E3D00003D7070005EF2390270197D0FFFFE780C1
:10E3E000C0DD1544E384A9F6268597A00000E780E8
:10E3F000C0BC9787FF1F9387A7B29C430144B9D73E
:10E400004A8597500000E780C05889B785097DB7D5
:10E410001743FFFFE70203CB79713E847C083EC8B7
:10E420002E8AB7071400A1653ECAE5057C08AA89B3
:10E43000080836C4428932C6BA8AC6843ECC97C020
:10E44000FFFFE78040E2CA85080897E0FFFFE7800A
:10E4500000C732460808B28597E0FFFFE78020C872
:10E46000A246630A09049D45080897E0FFFFE7807C
:10E47000C0BE1D4681459740FFFFE78040C96389C4
:10E480000A089145080897E0FFFFE78000BD1146A4
:10E49000A68597000100E780607A10080147814651
:10E4A000D2854E8597C0FFFFE78040014561174345
:10E4B000FFFF670063C4B685080897E0FFFFE780A9
:10E4C00000C21C400808D8439355C701858912072C
:10E4D0005183B205D98D97E0FFFFE78040C01C4013
:10E4E000080883C5870097E0FFFFE78040BD1C4018
:10E4F000080883C5A70097E0FFFFE78040BC1C40E9
:10E50000080883C5970097E0FFFFE78040BB85BF01
:10E510008945080897E0FFFFE78020B483C704001F
:10E520002300F50083C71400A300F500BDB717430F
:10E53000FFFFE70223B983C795004111AA8993F72A
:10E54000F707A384F5003285AE84328497E0FFFF9D
:10E55000E780A0C693170501C187635DF0042A898F
:10E56000032A040097C0FFFFE780C0C419E983575E
:10E5700044000548F11793B71700A307F10081463F
:10E5800031A81306F100A28597000000E78060958E
:10E590001DC51C459DC783D6470001480347F100B0
:10E5A00093078500D2884A86A6854E85970000008D
:10E5B000E78040E641011743FFFF6700E3B30948E6
:10E5C0007DBF1D486DBF1743FFFFE702A3AF657115
:10E5D0005C083EC4B7077B013EC65C083EC883C7E3
:10E5E00095002A8A328593F7F707A384F500AE8950
:10E5F00097E0FFFFE78040BA8357E100E1C7894514
:10E60000280097C0FFFFE78000C68145280097E0FB
:10E61000FFFFE780C0AA97C0FFFFE780E0CB9787A6
:10E62000FF1F9387E7C79C431774FF1F0344C47001
:10E63000AA843334800099C3136424009777FF1FA2
:10E640009387C7779C4399C3136444009787FF1F40
:10E650009387078D9C4399C31364840083D504007A
:10E660002800014997E0FFFFE78060A783D52400D9
:10E67000280097E0FFFFE78080A683D544002800AC
:10E6800097E0FFFFE780A0A597D0FFFFE780E0AD10
:10E6900093150501C181280097E0FFFFE78020A4C2
:10E6A000A285280097E0FFFFE78060A39C44636099
:10E6B000F902014781463000CE85528597C0FFFFA1
:10E6C000E780C0DF59611743FFFF6700E3A2DC4426
:10E6D0001314490028003E9497E0FFFFE7806096FE
:10E6E000834744000347540089070607BA97860703
:10E6F000E36AF5FC835524002800814A97E0FFFF78
:10E70000E780E09D83454400280097E0FFFFE78015
:10E71000009B83455400280097E0FFFFE780209A84
:10E720008347440063C9FA00814A8347540063C1A8
:10E73000FA020509A5BF1C4413975A002800BA978E
:10E7400083D50700850A97E0FFFFE7804099C9BF9E
:10E75000032BC40093975A0028003E9B83552B003F
:10E76000850A97E0FFFFE780809783550B0028001C
:10E7700097E0FFFFE780A0964DBF1743FFFFE7023A
:10E7800003965C4993E717005CC997A00000E780F7
:10E7900020B61743FFFF6700C3961743FFFFE7024A
:10E7A00003942E84814597F0FFFFE780C0E705C5FD
:10E7B00083570500FD172310F50009C48357250072
:10E7C0002310F40097000000E78060FB0145174329
:10E7D000FFFF6700039331457DD823100400C5BFB8
:10E7E0001743FFFFE702038E83C7950041112A8A72
:10E7F00093F7F707A384F50032852E89328497E0DA
:10E80000FFFFE780809B93170501C1876356F006E1
:10E81000AA89C145228597E0FFFFE780A0802A8B67
:10E820004E85832A040097C0FFFFE780A09831E956
:10E8300083574400231101000544F11793B71700D3
:10E84000A300F10081440348110003572100D6873B
:10E850005285CE862286CA8597F0FFFFE780A0A664
:10E86000A1679387170248003EC42302810026C691
:10E8700097E0FFFFE780406B41011743FFFF670010
:10E88000A38713061100A28597F0FFFFE78060655C
:10E89000AA8409E523110100094475B793052100F5
:10E8A0005A8597000000E78080EF835721002A8473
:10E8B000D9DB9777FF1F9387A7669C4381CB85455C
:10E8C0001305210097500000E780001583552100B3
:10E8D0002685314497C0FFFFE78060842DD5231043
:10E8E0000500268597900000E780206D0144A1BFB8
:10E8F0001733FFFFE702A37E41112E896C00AA8423
:10E9000002C697F0FFFFE78000D20DC10357050054
:10E9100005072310E50097000000E78040E68147E7
:10E920003E8541011733FFFF6700A37D32479547BE
:10E9300065DBCA85268597300000E780400DC1471A
:10E94000E34005FE3244854741462310F4008357D7
:10E950000900A685130544002311F4009700010067
:10E96000E780C02D228545BF1733FFFFE70283757F
:10E9700083C795004111AA8A93F7F707A384F5008E
:10E980003285AE89328497E0FFFFE78000839317DA
:10E990000501C1876356F0062A8AC145228597D0B2
:10E9A000FFFFE7802068AA845285032B040097C0EC
:10E9B000FFFFE780208031E98357440023110100E5
:10E9C0008544F11793B71700A300F10001440348F1
:10E9D000110003572100DA875685D2862686CE8518
:10E9E00097F0FFFFE780208EA1679387070248001A
:10E9F0003EC42302910022C697E0FFFFE780C05289
:10EA000041011733FFFF6700236FA2851306110032
:10EA100097F0FFFFE780E04C2A8409E5231101000D
:10EA2000894475B726859305210097000000E7808B
:10EA300060ECAA8449FD83552100228597B0FFFF31
:10EA4000E780E06D49F5014997C0FFFFE780E07678
:10EA5000635DA900184893171900BA9703D70700F8
:10EA60000DEF035721002390E70097C0FFFFE780D9
:10EA7000C074630625039777FF1F9387674A9C43FB
:10EA800099C70355210097500000E78080F0228548
:10EA900097900000E78060521DBF050975B7954447
:10EAA0003DB705C19307F00F630FF500C547630C31
:10EAB000F5009307F5FF05453315F5004205418143
:10EAC00082800145828041657D158280B9E91733D6
:10EAD000FFFFE702C360034506033284970000008E
:10EAE000E78060FC9305803EB305B502C205C18195
:10EAF00081CD0357E402854763F8E700130504015D
:10EB000097E00000E78020428357E40241677D17C9
:10EB10006385E700FD172317F4021733FFFF670033
:10EB2000435E82801733FFFFE702E358004283C74A
:10EB30009500444D0349140093F7F707A384F500AB
:10EB400083470400220911673369F900A167B347BD
:10EB5000F90041112A8BAE8A63ECE70E834724004B
:10EB60001307C00EB91793F7F70F6373F710034736
:10EB70003400C14763EEE70E834744001307E00704
:10EB800093C707086371F70C8349840083477400B7
:10EB9000A209B3E9F900856763F7F90A034A64003B
:10EBA000834754004E85220A336AFA0097500000CA
:10EBB000E780403B61C123962403834B3400137AE2
:10EBC000FA00239A34032388740323994403938916
:10EBD0000401631C090023A60402239804024E8545
:10EBE00097E00000E78060363DA0034924004A8595
:10EBF00097000000E78020EB2397A402834744009E
:10EC00004E85A388F402E38D0BFCE30B09FC97E02F
:10EC10000000E780202F97900000E7800073814676
:10EC20000146D6855A8597E0FFFFE7800058A16727
:10EC3000938797033EC423020100480002C697E071
:10EC4000FFFFE780602E41011733FFFF6700234A73
:10EC50008544A2862686D6855A8597E0FFFFE78001
:10EC6000C054A167938797033EC423029100F1B774
:10EC7000BD44C5B79144F1BF1733FFFFE70283449A
:10EC800001111C08404D3EC2B7070F003EC41C08CE
:10EC90003EC62A89AE8997C0FFFFE780E0D9585C5D
:10ECA0001C5C6346B70E6394E50063E2A70E3385F0
:10ECB000A740B3B7A700B305B7401306803E81460F
:10ECC0009D8D97000100E78080B793140501C180F6
:10ECD000A1659385C503480097B0FFFFE780A05862
:10ECE0008145480097D0FFFFE780603D83550404CD
:10ECF000480097D0FFFFE780803E835524044800FA
:10ED000097D0FFFFE780A03D814589CCC167FD1703
:10ED10009305F00F6388F400268597500000E78084
:10ED2000E0E0AA85480097D0FFFFE780403903550F
:10ED30004404814501CDC167FD179305F00F6307BA
:10ED4000F50097500000E78060DEAA85480097D064
:10ED5000FFFFE780C03683456404480097D0FFFF7B
:10ED6000E780E03583457404480097D0FFFFE780D3
:10ED70000035500001478146CE854A8597B0FFFF98
:10ED8000E780C07305611733FFFF6700E3368144F6
:10ED900081B71733FFFFE702833483C7950093F7EA
:10EDA000F707A384F50097000000E78020ED1733F4
:10EDB000FFFF670003351733FFFFE702A33083C768
:10EDC00095004111404D93F7F707A384F5002A8A77
:10EDD0003285B284AE8997D0FFFFE780003E2A8B50
:10EDE000268597D0FFFFE780403D2A89268597D06A
:10EDF000FFFFE780603A93170B0163CA0702E177D0
:10EE0000CA97C207C183116763E3E702930709103A
:10EE1000C207C1831307B00F637BF7009317090183
:10EE2000C187AA8A634AF000C54763FE57014101C2
:10EE30001733FFFF6700432C97B0FFFFE7800028E0
:10EE4000E31725FFD5B763080B0263060902814467
:10EE500063890A02B7077F00231064052311240584
:10EE60007CC0568597000000E780E0C39304803E95
:10EE7000B304950239A0B7077F00232004047CC0A7
:10EE800081440355240497E00000E780A0A3A1C4B7
:10EE900097C0FFFFE78040BA269593D7F4413337F8
:10EEA0009500AE97BA9708DC5CDCCE85528597005A
:10EEB0000000E780A0DC99E023220404A167938787
:10EEC000B70348003EC42302010002C697E0FFFFDB
:10EED000E7808005A9BF814701481CDC232E04037D
:10EEE000E9B71733FFFFE702831F97C0FFFFE780F3
:10EEF0000037E1473305F502914597500000E78060
:10EF000000C5E55711C59777FF1F23A5A7E28147E5
:10EF10003E851733FFFF6700C31E85471777FF1F26
:10EF2000230CF7E082801733FFFFE702431B97773C
:10EF3000FF1F9387E7DF80433DC08357040463903E
:10EF4000A70683572404639CB7043689B28497C00C
:10EF5000FFFFE78060AE5C5C63C3B7046395B700F6
:10EF60001C5C63EEA7028347640463F3F400A68786
:10EF70002303F4048347740463F39700A687A30371
:10EF8000F4048357440441677D176385E7008507D0
:10EF90002312F4043C4481C7CA852685829717331F
:10EFA000FFFF670003169777FF1F938767D89C437F
:10EFB000014599C303C5870082801733FFFFE7022D
:10EFC00003120111B70707003EC683C79500584DCD
:10EFD0000AC493F7F7070AC8A384F5002A89AE8408
:10EFE00011CB1C4283C707002304F7009790000051
:10EFF000E7800034216493055402280097B0FFFF96
:10F00000E780602697000000E78020FAAA852800A4
:10F0100097D0FFFFE780A00A300001478146A68510
:10F020004A8597B0FFFFE78060491304440248080F
:10F0300022CC230A010002CE97E0FFFFE780C0EE5A
:10F0400005611733FFFF6700C30B1733FFFFE702AC
:10F05000030901117C003ECAB70707003ECC7C00C3
:10F060003ECE83C795002E84AA8493F7F707A38426
:10F07000F500A16593855502480897B0FFFFE7802A
:10F08000801E97000000E78040F2AA85480897D0CC
:10F09000FFFFE780C002500801478146A285268510
:10F0A00097B0FFFFE780804105611733FFFF6700DE
:10F0B00043059777FF1F9387A7C79C43094599C3CB
:10F0C00003C5970082809777FF1F938767C69C438D
:10F0D000094599C303C5D70082809777FF1F93879F
:10F0E00027C59C43014599C303C5A70082801733F8
:10F0F000FFFFE70223FD0111B70708003EC683C7E3
:10F100009500404D0AC493F7F7070AC8A384F50099
:10F110002A89AE8429C41442854703C7060063E0E8
:10F12000E70A83479400094681496380C702B30711
:10F13000F740A304E400B339F00083C716002305A9
:10F14000F40097900000E780A01E03572403058B6E
:10F1500019C76386090097D00000E78000E92164A1
:10F1600093058402280097B0FFFFE780C00F970047
:10F170000000E78040F4AA85280097D0FFFFE780D1
:10F1800000F497000000E78080F5AA85280097D05A
:10F19000FFFFE780C0F2014781463000A6854A851F
:10F1A00097B0FFFFE780803113047402480822CC37
:10F1B000230A010002CE97E0FFFFE780E0D6056159
:10F1C0001733FFFF670043F31733FFFFE70223F115
:10F1D00001117C003ECAB70708003ECC7C003ECE41
:10F1E00083C795002E84AA8493F7F707A384F500BC
:10F1F000A16593858502480897B0FFFFE780A006C8
:10F2000097000000E78020EBAA85480897D0FFFF11
:10F21000E780E0EA97000000E78060ECAA854808F4
:10F2200097D0FFFFE780A0E9500801478146A285FB
:10F23000268597B0FFFFE780602805611733FFFF41
:10F24000670023EC9777FF1F938787AE9C430145A8
:10F2500099C303C5B70082801733FFFFE70223E895
:10F260000111B70707003EC683C79500404D0AC489
:10F2700093F7F7070AC8A384F5002A89AE8405C866
:10F280001C42054783C707006368F7060347B400BD
:10F29000630FF700A305F40097900000E780400992
:10F2A0008347B400B9CF97D0FFFFE78040BE216409
:10F2B0009305B400280097B0FFFFE780C0FA9700DD
:10F2C0000000E78060F8AA85280097D0FFFFE7805C
:10F2D00000DF014781463000A6854A8597B0FFFFD1
:10F2E000E780C01D2904480822CC230A010002CE71
:10F2F00097E0FFFFE78040C305611733FFFF67001A
:10F3000043E097D0FFFFE78020BF55B71733FFFFDB
:10F31000E702E3DC01117C003ECAB70707003ECCE0
:10F320007C003ECE83C795002E84AA8493F7F7070E
:10F33000A384F500A165AD05480897B0FFFFE780FD
:10F3400080F297000000E78020F0AA85480897D057
:10F35000FFFFE780C0D6500801478146A285268579
:10F3600097B0FFFFE780801505611733FFFF670047
:10F3700043D99777FF1F9387A79B9C43094599C360
:10F3800003C5C70082801733FFFFE70243D5011191
:10F390007C00AE843ECAA165B70707002A843ECC34
:10F3A000D1057C0048083ECE97B0FFFFE780A0EB78
:10F3B00097000000E78020FCAA85480897D0FFFF4F
:10F3C000E780E0CF500801478146A685228597B0A7
:10F3D000FFFFE780A00E05611733FFFF670063D2D0
:10F3E0001733FFFFE702A3CF83C7950093F7F70713
:10F3F000A384F50097000000E78020F91733FFFF92
:10F40000670023D01733FFFFE702C3CB83C7950004
:10F410000329C501411193F7F707A384F5001C42A6
:10F4200083C90700854763E637079777FF1F9387F0
:10F4300027E79C432E84AA8485CF97000000E780AD
:10F4400080F389476306F502630409028347C90014
:10F45000638037032306390197900000E78040ED71
:10F4600083572903898B89C797D00000E780E0B7CD
:10F470002685A28597000000E78020F1A167CD07CF
:10F4800048003EC42302010002C697E0FFFFE78068
:10F49000A0A941011733FFFF670003C69777FF1F3D
:10F4A000938707899C431D4599C303C5E700828064
:10F4B0001733FFFFE702A3C20111B70707003EC6DB
:10F4C00083C79500584D0AC493F7F7070AC8A38469
:10F4D000F5002A89AE8415C71C4283C7070093969E
:10F4E0008701E18663C4060685466381D7068346A5
:10F4F000E7006388F6002307F70097900000E78095
:10F5000020E321649305E400280097B0FFFFE78023
:10F5100080D597000000E780A0F8AA85280097D042
:10F52000FFFFE780C0B9014781463000A6854A85C4
:10F5300097B0FFFFE78080F83504480822CC230A03
:10F54000010002CE97E0FFFFE780009E05611733C0
:10F55000FFFF670003BB1733FFFFE70243B801114A
:10F560007C003ECAB70707003ECC7C003ECE83C776
:10F5700095002E84AA8493F7F707A384F500A1656C
:10F58000B905480897B0FFFFE780E0CD970000007D
:10F59000E78000F1AA85480897D0FFFFE78020B2F6
:10F5A000500801478146A285268597B0FFFFE78076
:10F5B000E0F005611733FFFF6700A3B41733FFFFC7
:10F5C000E70243B0AA8401441769FF1F1309897633
:10F5D000E14997C0FFFFE78080C86344A40001456C
:10F5E00019A833053403832709003E958357250066
:10F5F0006397970011051733FFFF6700E3AF05041A
:10F60000C9BF032E8500630A0E121773FF1F130371
:10F61000239103230300631503002943639006121B
:10F6200003234E01631503001D436399071017332D
:10F63000FFFFE70243A8C689428A3E89BA8AB68498
:10F64000328BAE8B2A84B5E103554E0019E5014398
:10F650001A851733FFFF670083A9A167A98F116778
:10F6600063FBE70097000000E78080F5814597F095
:10F67000FFFFE780C0120844B70700E05841F98F48
:10F6800018455CC1B707001FF98F1CC55C4991C7BD
:10F69000610597E00000E780408BE38A09FA228544
:10F6A00097900000E78060C65DB7328597C0000084
:10F6B000E78040430D4349DD1C44116703D54700F3
:10F6C000A167A98F63FBE70097000000E78040EF88
:10F6D000814597F0FFFFE780800C03238400931699
:10F6E0004B01D1828347B300035663008588FD8BAD
:10F6F000A305F300FD777D8E558EFD76FD16B204D1
:10F70000F18E83274301C58E231273012313D30087
:10F710002304530123052301A3044301BDDF2285F4
:10F7200097B0FFFFE78060CCAA850844B5D161059A
:10F7300097D00000E780207F8DB71D431A85828017
:10F740001733FFFFE70203980569AA84AE89328A5E
:10F750000144FD5A7D1997C0FFFFE78000A563476C
:10F76000A40001451733FFFF67000399D84493179E
:10F770001400BA9703D70700631F3703239057017C
:10F7800063070A00268597900000E780A0809C44CC
:10F790009DC383D76700B3F72701639E3701D288E3
:10F7A00001488147014781460146814526859700EA
:10F7B0000000E78040E5050479BF1733FFFFE7024B
:10F7C000639079711C103EC4B7070F003EC61C1031
:10F7D0003EC883C79500AA8A328593F7F707A384AA
:10F7E000F5002E89328497D0FFFFE780009D9317A4
:10F7F0000501C187635AF006AA89228597D0FFFFC9
:10F80000E780A09B2A8A4E85032B040097B0FFFF58
:10F81000E780409A39ED8357440081440544F1174D
:10F8200093B71700A303F10083457100DA8722879D
:10F83000D2864E86280097E0FFFFE780E057014719
:10F8400081463000CA85568597B0FFFFE78000C724
:10F85000A1679387F70348083ECC230A810026CE90
:10F8600097D0FFFFE780406C45611733FFFF6700CB
:10F87000A388A2851306710097E0FFFFE78060660A
:10F88000AA84094455D1528597E0FFFFE78060D4F0
:10F890000D4459D90546D285268597000000E7809A
:10F8A00060EA2A8451B71733FFFFE7024383835589
:10F8B00007000346270041112A842E8532C62EC434
:10F8C00097E0FFFFE780E0D001C93246A2452285DC
:10F8D00097000000E78000E741011733FFFF670052
:10F8E00043821723FFFFE702037D83C79500411181
:10F8F000AA8A93F7F707A384F5003285AE8932848C
:10F9000097D0FFFFE780608B93170501C18763578E
:10F91000F00AC1452A8A228597C0FFFFE7808070E0
:10F920002A8D228597D0FFFFE78020892A892285AA
:10F9300097D0FFFFE7804086930705F893F7F70F0E
:10F940001307E007AA8B637BF706228597D0FFFF9A
:10F95000E78080842A8C228597D0FFFFE780C083D0
:10F96000AA8C5285032B040097B0FFFFE7808084A8
:10F9700039E983574400231101008144F11793B7FB
:10F980001700A300F100054403471100835621002E
:10F99000938784005685DA8822885286CE8597F030
:10F9A000FFFFE78020A7A167E90748003EC42302C4
:10F9B000810026C697D0FFFFE7800057410117233B
:10F9C000FFFF6700C37213061100A28597E0FFFFD7
:10F9D000E7802051AA8409E52311010009446DB78D
:10F9E000930521006A8597F0FFFFE780A0F02A8445
:10F9F00041FD835521009356C900131649018548DE
:10FA00006688E2875E87858A518226859700000096
:10FA1000E78060BF2A848DBF1723FFFFE702A36939
:10FA200083C7950041112A8B93F7F707A384F5004C
:10FA30003285AE89328497C0FFFFE7800078931744
:10FA40000501C1876352F00A2A8A228597C0FFFF09
:10FA5000E780A076AA8A228597C0FFFFE780E0753D
:10FA60002A89228597C0FFFFE7800073930705F876
:10FA700093F7F70F1307E0072A8C6377F7062285C1
:10FA800097C0FFFFE7804071AA8C228597C0FFFFD7
:10FA9000E78080702A8D5285832B040097A0FFFF9A
:10FAA000E780407139E58357440085440144F117EC
:10FAB00093B71700A301F1000347310093078400B7
:10FAC0005A85DE882688D6865286CE8597F0FFFF37
:10FAD000E78040948D4748003EC42302910022C62F
:10FAE00097D0FFFFE780404441011723FFFF6700E5
:10FAF0000360A2851306310097E0FFFFE780603EB8
:10FB00002A84894455D99356C9001316490185485A
:10FB10006A88E6876287858A5182D68597000000C9
:10FB2000E78060AEAA8449BF1723FFFFE70283592D
:10FB30002A8981440144617A916A176BFF1F130B74
:10FB40002B3E97B0FFFFE780406763C7A400228584
:10FB50001723FFFF6700435A832709009399140076
:10FB6000CE9703D5070033074501420741836364FD
:10FB7000570305C103270B0019C785453E859740EC
:10FB80000000E78060E9832709000504CE972390F1
:10FB9000070085047DB797000000E78060A28327F7
:10FBA00009000504CE972390070065D5814597F09D
:10FBB000FFFFE780C0BEF1BF1723FFFFE7028350BE
:10FBC00083C7950041112A8A93F7F707A384F500AC
:10FBD00032852E89328497C0FFFFE780005E93173D
:10FBE0000501C187635AF004AA89832A040097A0FB
:10FBF000FFFFE780205C31E58357440085440144E2
:10FC0000F11793B71700A301F10003483100D6871D
:10FC100052850147CE862686CA8597D0FFFFE780AA
:10FC2000806AA167F50748003EC42302910022C6FE
:10FC300097D0FFFFE780402F41011723FFFF6700A8
:10FC4000A34BA2851306310097E0FFFFE7806029F0
:10FC50002A8489445DD99767FF1F9387672C9C434B
:10FC600081CF044997B0FFFFE7802055AA852685FC
:10FC700097400000E78040DA130504019700000078
:10FC8000E780C0EA228597800000E7800033814446
:10FC9000ADBF1723FFFFE702034283C79500411161
:10FCA000AA8A93F7F707A384F5003285AE893284D8
:10FCB0002311010097C0FFFFE78020509317050133
:10FCC000C1876354F0062A8AC145228597C0FFFF89
:10FCD000E7804035AA8B5285032B040097A0FFFFD5
:10FCE000E780404D21E98357440085440144F117E2
:10FCF00093B71700A300F100034811000357210038
:10FD0000DA875685D2862686CE8597D0FFFFE78094
:10FD1000805BA1679387270248003EC423029100BD
:10FD200022C697D0FFFFE780202041011723FFFF65
:10FD30006700E33BA2851306110097E0FFFFE78011
:10FD4000401A2A8489444DD99767FF1F9387471D1E
:10FD500098433E8901CF044997B0FFFFE780E04513
:10FD6000AA85268597400000E78000CB1305040193
:10FD700097000000E78080DB97B0FFFFE780E0435B
:10FD800095443DD9930521005E8597F0FFFFE780FC
:10FD900060B6AA8435F11C480357210022852390C0
:10FDA000E70097800000E780402183270900A9D75A
:10FDB0000355210097400000E780A0BD35BF172301
:10FDC000FFFFE702432F83C795004111AA8A93F7EB
:10FDD000F707A384F5003285AE89328497C0FFFF10
:10FDE000E780A03D93170501C1876351F0062A8A79
:10FDF000228597C0FFFFE780403C2A895285032B6C
:10FE0000040097A0FFFFE780E03A31E58357440004
:10FE100085440144F11793B71700A301F10003488B
:10FE20003100DA8756854A87D2862686CE8597D0D6
:10FE3000FFFFE7804049A167F90748003EC423025D
:10FE4000910022C697D0FFFFE780000E41011723E3
:10FE5000FFFF6700C329A2851306310097E0FFFF6B
:10FE6000E78020082A8489445DD99167CA97C20730
:10FE70001167C1831307F7EF8544E362F7FA9767C9
:10FE8000FF1F9387E7099843BE8B01CF044997B0C2
:10FE9000FFFFE7808032AA85268597400000E78033
:10FEA000A0B71305040197000000E78020C897B0B1
:10FEB000FFFFE780803095443DD11C482285814476
:10FEC0002390270197800000E780200F83A70B0075
:10FED000B9D74A8597400000E780A0AB89B71723C0
:10FEE000FFFFE702C31F2A844105B2849700000088
:10FEF000E780C0C311C5228597800000E780E00B32
:10FF000081460146A685228597800000E780C04E85
:10FF10001C4C89C7DC4799C3228582971723FFFFB2
:10FF20006700231E9767FF1F938787E09C43014567
:10FF300099C31385070182809767FF1F938747DF67
:10FF4000884382801723FFFFE70263199317C600D7
:10FF5000DD8DC2054111C1812A8432C697C0FFFFE1
:10FF6000E780E0173246228511829375F60F97C01D
:10FF7000FFFFE780C01441011723FFFF67006318EC
:10FF80001723FFFFE702031479713C083ED2B7073D
:10FF90000C003ED43C083ED683C79500AE842A8927
:10FFA00093F7F707A384F500A165938535044810FE
:10FFB00097A0FFFFE780202BC165FD150144176A5C
:10FFC000FF1F130A6AF7930A400EAE892E8B2EC6C6
:10FFD00097B0FFFFE780602142059317040141813C
:10FFE000C183B24563E9A702C167FD176387F500C6
:10FFF000481097C0FFFFE780800E501001478146F0
:020000040001F9
:10000000A6854A8597A0FFFFE780404B45611723EF
:10001000FFFF6700630E3307540383270A0BBA9769
:1000200003D6C701630A3601638A35014810970079
:100030000000E78060F1DA85050451BFB285EDBFAD
:100040001723FFFFE702230779717C083EC8B70733
:1000500011003ECA7C083ECC83C79500AA89328530
:1000600093F7F707A384F5002E8997C0FFFFE78079
:10007000C01485676378F504A165AA84890508081A
:1000800097A0FFFFE780201E268597400000E780AD
:1000900060ED133415000A04A285080897C0FFFF1D
:1000A000E780E001A685080897C0FFFFE7802003EE
:1000B00025CC014781461008CA854E8597A0FFFFD1
:1000C000E780C03F45611723FFFF67004302B30786
:1000D00054030327CA0ABA9703D70700631C970083
:1000E00003D6270063806505080897000000E780B5
:1000F000A0E5DE8505042EC697B0FFFFE780E00F80
:100100004205931704014181C183B245E3E1A7FC95
:10011000C167FD17E38FF5F8080897C0FFFFE78078
:1001200000FC41BFB285F9B7C165FD150144176AEE
:10013000FF1F130A6AE0930A80022E8BAE8B65BF05
:100140001723FFFFE702A3F91841834717008346EF
:100150000700A207D58FD207D1832390F5008347EC
:100160002700034717008D45A207D98F91832310DD
:10017000F60097C0FFFFE780A0E91723FFFF6700A5
:1001800043F81723FFFFE702E3F3C1640144176953
:10019000FF1F130969DA93098002FD1497B0FFFF6E
:1001A000E780A0056347A40001451723FFFF670010
:1001B000A3F4330534038327C90A3E95835705000A
:1001C000E38597FE0504D9BF1723FFFFE70283EFFE
:1001D0002A8AAE89B284B68A97400000E78080D828
:1001E00019E591473E851723FFFF6700E3F02A8951
:1001F0004E8597C00000E780E08E2A84638E0A0453
:100200008D476DD103570500C547E31D47FD0347E3
:10021000F9018546AD47E317D7FC8347450081CFF9
:100220004146A6855D0597F00000E780C09E8147A6
:1002300055D9AD4745BF130965012302E500CA85BD
:10024000268597100000E780606231C1A547E38BE7
:100250000AF82302040079B705C183570500E39229
:1002600047F94146A685190597F00000E780A09A56
:1002700081472DD99947BDB74E8597000000E7808B
:1002800080F02A84954739DD130955004DBF41465A
:10029000A68523104401231134011305190097F09A
:1002A0000000E780A099228597800000E780A0EAFF
:1002B00081470DBF1723FFFFE70263E279717C00DE
:1002C0003ECCB7070A003ECE7C003ED083C79500E7
:1002D000B2842E8493F7F707A384F5001306A100D8
:1002E0002A892C00268597000000E780A0E5A165FB
:1002F00028088D0597A0FFFFE780E0F69040835522
:10030000A10003558100854697000000E78000ECBE
:10031000AA84AA85280897C0FFFFE78040DA035621
:10032000A10083558100280897000000E780C0C124
:10033000300801478146A2854A8597A0FFFFE780E4
:10034000E017854748103ED42302910202D697D089
:10035000FFFFE78060BD45611723FFFF670063DA99
:100360001723FFFFE702A3D779717C003ECCB707C4
:100370000A003ECE7C003ED083C79500B2842E8416
:1003800093F7F707A384F5001306A1002A892C0030
:10039000268597000000E780E0DAA16528088D0532
:1003A00097A0FFFFE78020EC90408355A100035504
:1003B0008100814697000000E78040E1AA84AA8579
:1003C000280897C0FFFFE78080CF0356A100835520
:1003D0008100280897000000E78000B73008014737
:1003E0008146A2854A8597A0FFFFE780200D48102F
:1003F0002302910202D402D697D0FFFFE780C0B259
:1004000045611723FFFF6700C3CF1723FFFFE702F4
:1004100003CD97000000E78060DB1723FFFF670034
:1004200043CE9767FF1F9387E79088438280172307
:10043000FFFFE702C3CA835725004111AE842A8417
:100440002307B10017F5FFFF130525466C0023169F
:10045000F10097A0FFFFE780604891C42285978054
:100460000000E780E0D6FD572310F40013062002B9
:100470008145130554009720FFFFE78040C94101E3
:100480001723FFFF6700E3C71723FFFFE70283C3BC
:1004900079717C003ECCB7070A003ECE7C003ED08E
:1004A00083C79500AA89AE8493F7F7073285A384A2
:1004B000F5001306A1002C0097000000E78080C81B
:1004C00003558100114497400000E780A0A915C59D
:1004D0000355A100014497B00000E780A06011CD52
:1004E000035705008357810045446318F70085458D
:1004F00097000000E780E0F301442169930539008B
:10050000280897A0FFFFE78000D6A285280897C09B
:10051000FFFFE780C0BA0356A10083558100280879
:1005200097000000E78040A2300801478146A68579
:100530004E8597A0FFFFE78060F848104AD4230259
:10054000810202D697D0FFFFE780009E4561172306
:10055000FFFF670063BA1723FFFFE702A3B69757B1
:10056000FF1F9387E77C2A8488432E8915C503578C
:1005700045038357C4016311F7022326050223189C
:100580000502410597D00000E780209C6306090022
:1005900097800000E78060DB81449769FF1F9389A3
:1005A000A999130A800297B0FFFFE78000C563C4D2
:1005B000A4049767FF1F938767809C4399C70355DF
:1005C000C40197200000E780C0BD630709002285B1
:1005D00097800000E780C0A01306400E8145228569
:1005E0009720FFFFE780A0B2FD57231EF4001723DA
:1005F000FFFF670063B03385440383A7C90A3E95B4
:10060000035705008357C4016317F700CA85970095
:100610000000E78000E2850479B71723FFFFE702B7
:1006200063AA83C795004111AA8993F7F707A384AA
:10063000F5003285AE8497C0FFFFE78000B885677C
:100640006378F5042A8997400000E780A09101446F
:1006500001CD83D704003144638827018545970085
:100660000000E78080EF01444E85A2864A86A68579
:1006700097D0FFFFE780A09CA167938717044800ED
:100680003EC42302810002C697D0FFFFE780C089E5
:1006900041011723FFFF670023A61723FFFFE7028F
:1006A00063A29757FF1F9387A768804329C401451A
:1006B00097C00000E780002181470148C1641CDC2D
:1006C000232E0403232004041769FF1F1309C9867E
:1006D00001449309400EFD1497B0FFFFE780E0B09E
:1006E000634FA400814517F5FFFF1305857F97A091
:1006F000FFFFE780A01E1723FFFF6700E39F33057E
:1007000034038327090B3E958357C5016387970000
:10071000854597000000E78040E4050475BF9357C6
:10072000050113D78700A380F50093170501C18346
:10073000A1832380E5002381F500A381A5008280A9
:100740001723FFFFE702A3992300050083C71500C5
:10075000A300F50083C725002301F50083C73500FA
:10076000A301F50083C745002302F50083C75500A8
:10077000A302F50083C7650093059500A303050058
:100780002303F50023040500328597000000E7806D
:1007900040F91723FFFF6700C3961723FFFFE70207
:1007A00063924111E9540DCD85CD93F9C5FF2E8497
:1007B0002A89AA84338AA900B7EA040063189A0236
:1007C0000D88854411CCB7E704009C5F82972AC648
:1007D00022866C003305390197E00000E78000466F
:1007E000268541011723FFFF6700039183A78A0332
:1007F0009104829793170501C183A183A38EF4FE10
:1008000093570501238FF4FEA183238EA4FEA38FAB
:10081000F4FE6DB763E6D5021723FFFFE702238CD2
:10082000B28741113686BE8536C697E00000E78064
:10083000E040B246410136851723FFFF6700638C15
:10084000814636858280838705001387F5003D0544
:10085000FD8793F77708834607007D158606B58FD9
:10086000A300F5006307B7007D17834717009D833A
:10087000DDB782801723FFFFE7026386B7E7040036
:1008800083A7070932872A863A8582971335150090
:100890001723FFFF6700E38615C181478DC117232A
:1008A000FFFFE702C383414697E00000E78000397D
:1008B00085473E851723FFFF6700A38481473E8558
:1008C00082801DCD1723FFFFE702638141468145EA
:1008D0002A849720FFFFE7808083414681451305E6
:1008E00004039720FFFFE78080820147C16723222E
:1008F000040438C87CC805451723FFFF67006380E0
:100900000145828081473DCDB5CD1713FFFFE7023A
:10091000037DB2842E891306800581452A849710B1
:10092000FFFFE780C07ECA8524C4268597000000AB
:10093000E780C0F64146814522859710FFFFE7809A
:10094000007D3044A285228597000000E780C0F238
:1009500093040401A285268597000000E780E0EE5D
:10096000A6851305040297000000E78000EE2285AB
:1009700097000000E78020F585473E851713FFFFAD
:10098000670023783E8582801713FFFFE702837399
:100990004111E9540DCD85CD93F9C5FF2E842A89E7
:1009A000AA84338AA900B7EA0400639844030D8837
:1009B000814411CCB7E704009C5F82972AC6228647
:1009C0006C003305390197E00000E7802027268579
:1009D00041011713FFFF6700237283A78A03910465
:1009E000829793170501C183A183A38EF4FE9357C9
:1009F0000501238FF4FEA183238EA4FEA38FF4FEB2
:100A00006DB765CD1713FFFFE702C36BB28411E624
:100A100005451713FFFF6700236E2A842E890145C1
:100A2000EDD93C487848B3E6E700E5D69386F7FF72
:100A3000B3B7F6007D17032A4404BA9734C87CC8BC
:100A400063050A06C14913050A03B3894941229582
:100A5000637D3601B2862E86A68597000000E7806A
:100A6000A0DB7C40BE9464C065B7CE862E86CE8562
:100A700097000000E78040DAC114D2944E992322F7
:100A80000404A2879306040103C7070003C60703F3
:100A90008507318FA38FE7FEE398F6FE3044A285E9
:100AA000228597000000E78020DD2699C1493306A2
:100AB000994063EC9900A9DCA686A685130504037A
:100AC00097000000E78040D579BF8147B306F40066
:100AD0003307F6000347070083C5060085072D8FFF
:100AE0002380E600E39437FF3044A28522859700F7
:100AF0000000E78060D8C1145DBF014582800DC150
:100B00001713FFFFE702A35D1306800581459710C9
:100B1000FFFFE780C05F05451713FFFF6700635EB7
:100B200001458280814749C5C1C51713FFFFE70210
:100B3000035BFC4141462E84AA846399C704138653
:100B40000501A2878146C14503C7070003C5070306
:100B50008507298F3305D600034505008506298FB3
:100B6000A38FE7FEE392B6FE3044A2852685970068
:100B70000000E78060D0228597000000E78060F8E1
:100B800085473E851713FFFF6700A35713850703AB
:100B90001D8E814522959710FFFFE78040577C40CE
:100BA000130700F813060402A2972388E70251BF37
:100BB0003E8582801713FFFFE70263526D712E841A
:100BC000B284AA8590102800368997000000E7803B
:100BD000A0D309EDD55725A050400C402800970020
:100BE0000000E78040E27DD5FD142104F5F42C00DF
:100BF0004A8597000000E78020F3814761DD3E854C
:100C000051611713FFFF6700C34F1713FFFFE70280
:100C1000034D41112EC432C62C000546970000003A
:100C2000E78080F941011713FFFF6700834D171319
:100C3000FFFFE702C34A01112A842EC602C802CA76
:100C400002CC02CE97E00000E780C023B2462A869D
:100C5000A285080897000000E78060FB1375F50F78
:100C600005611713FFFF6700C3491713FFFFE70272
:100C700003477971B2872A8421462308B1001305FE
:100C80001101BE853AC436C697E00000E78000FB3C
:100C9000B24693059101368597000000E78060A871
:100CA0002285141035460C0897000000E78020F6D6
:100CB0002A84224701E921460C103A8597E000007A
:100CC000E780C0F7228545611713FFFF6700634384
:100CD0001713FFFFE702A3407171AE84AA850A854E
:100CE000328497000000E78060BB11C90A86A685A0
:100CF000228597000000E78020B8814711E1C547B1
:100D00003E854D611713FFFF6700A33F1713FFFFD9
:100D1000E702E3391D712A8AB289BE8435468547C8
:100D2000130511012E8CB68A3A8BC28C468D23088E
:100D3000F10097E00000E78060F010100C08528589
:100D4000231F010097000000E780C0F82A843DEDD2
:100D5000A1476313FD089307900591E0E5473546E9
:100D6000E2851305110113990A012308F1001359B3
:100D7000090197E00000E78060EC13578900939722
:100D80008A00D98F90080C085285231FF100970024
:100D90000000E78020F42A8415E9A1E49387FA0093
:100DA00091831379F9003EC6631309004149668BAC
:100DB0008144C14B854DB247639F970C6A868C0076
:100DC00033855C0197E00000E78040E722852561DC
:100DD0001713FFFF6700633193079004C9F0A5471D
:100DE000BDBF834701050947C14B2308F100834775
:100DF0001105A58FA308F10093872400814463E1C6
:100E0000FB04014714083386E6008C08B386E4002F
:100E1000BA95DA9683C6060083C505000507AD8E30
:100E20002300D600E390E7FE4147639CE704900867
:100E30000C08528597000000E780C0E925D181A009
:100E4000B3069B00BA871008B305F60090083E96DB
:100E500003C506000346060085078506298E238004
:100E6000C500E39277FF998F90080C085285BE94D5
:100E700097000000E78000E68947014749D12A84AE
:100E8000B1B790083E96034606001408BE9623802C
:100E9000C600850759BFB247850463879714814709
:100EA0001808B306F70098083E973386F900034701
:100EB0000700034606008507318F2380E600E39193
:100EC00077FF90080C08528597000000E78080E0CB
:100ED0005DF53546E285130511012308B10197E060
:100EE0000000E780A0D51397040141839397840005
:100EF0002183D98F10180C085285231FF100970009
:100F00000000E78020DD25FD814710183387F900B8
:100F10003E960347070003460600B306FB0085071D
:100F2000318F2380E600E39277FF65A81808B306A7
:100F3000F70098083E973386F900034707000346F9
:100F400006008507318F2380E600E3E127FFCA878B
:100F5000639E770990080C08528597000000E7808F
:100F600060D711FD81479800B306F700900818106C
:100F70003E973E9603470700034606008507318FDC
:100F80002380E600E39177FF3546E28513051101E2
:100F90002308B10197E00000E78040CA13970401DD
:100FA0004183939784002183D98F10180C085285B0
:100FB000231FF10097000000E780C0D1E31105EC8A
:100FC000814710183387F9003E9603470700034610
:100FD0000600B306FB008507318F2380E600E3E2BD
:100FE00027FFC109410BC1BB814785B79408BE9655
:100FF00083C6060018083E972300D700850789BFDF
:10100000638006321713FFFFE702630A59712A84CF
:10101000BE89B28B85473546130511022E8B468C4F
:101020004289BA8A368A2300F10297E00000E780FD
:10103000E0C010180C102285231701029700000051
:10104000E78040C963180512A147631FFC06930798
:10105000900563930900E5473546DA8513051102CB
:1010600093140A012300F102C18097E00000E78099
:10107000E0BC93178A0013D78400D98F90080C1016
:1010800022852317F10297000000E780A0C47DE1CC
:10109000639209049307FA00BD88918391E0C144EB
:1010A000C207C183DE8C814A3EC6414DB24763E22E
:1010B000FA0E6286B3854B01881097E00000E78046
:1010C00080B54DC93D557DA093079004E39609F87E
:1010D000A54759B7834701050947C14C2300F102D1
:1010E00083471105B3C7F900A300F10293872900D4
:1010F000814963E1FC04814618103306D7008C084F
:101100003387D900B69556970347070083C5050076
:1011100085062D8F2300E600E390D7FE41476390BC
:10112000E70690080C10228597000000E78080BA3F
:1011300035D189A0B3863A01BA871010B305F600FD
:1011400090083E9603C506000346060085078506FF
:10115000298E2380C500E39297FF3387EC409008E7
:101160000C102285BA9997000000E780A0B6894745
:10117000014741D165611713FFFF670003F790082E
:101180003E96034606001410BE962380C6008507CF
:1011900079B7B247850A93990A01939D8A0093D93A
:1011A00009016391570F85473546DA85130511020A
:1011B0002300F10293D9890097E00000E78000A89E
:1011C000B3ED3D0190000C1022852317B103970069
:1011D0000000E78020B059FD8147A68963EA9706A1
:1011E00026860C084A8597E00000E78020A5814705
:1011F0001810B306F700100898083E973E9603476C
:101200000700034606008507318F2380E600E3E1EF
:1012100097FE639FA90590080C1022859700000097
:10122000E78040AB21F981479810B306F70090089A
:1012300018183E973E9603470700034606008507A9
:10124000318F2380E600E391A7FF4109C10CB9BDAE
:1012500018089000B306F7003E963387FC0003475A
:101260000700034606008507318F2380E600B5B7E7
:1012700098084E97034707001C10CE972380E7007D
:10128000850941BF85473546DA85130511022300DC
:10129000F10293D9890097E00000E780209AB3ED2E
:1012A0003D0190000C1022852317B1039700000028
:1012B000E78040A2E31005EC814718089000B306D0
:1012C000F7003E963387FC000347070003460600FD
:1012D0008507318F2380E600E391A7FF41460C0884
:1012E0004A8597E00000E780609581471810B306B3
:1012F000F700100898083E973E96034707000346FC
:1013000006008507318F2380E600E391A7FF900850
:101310000C10228597000000E780C09B1DD599BD69
:101320007D5582801713FFFFE70263DB01112A84DA
:101330002E8593055100328902C002C202C402C642
:101340009304740097F0FFFFE780A03D1D46A6853B
:101350001305910097E00000E780408E10088A8511
:101360004A8597000000E780E09619ED9307140086
:10137000180883C607000346070085070507B18ED6
:10138000A38FD7FEE397F4FE05611713FFFF6700F5
:1013900043D71713FFFFE702E3D22E848C4141119C
:1013A000AA89838715003289914463D30700A14439
:1013B0009757FF1F9387C7EE9C43A1C7C1CA8D47AC
:1013C0002310F10083C725004A852301F10083C75C
:1013D0003500A301F10083C745002302F10083C754
:1013E0005500A302F10083C7650093059100A30394
:1013F00001002303F1002304010097F0FFFFE780C1
:1014000040320C404A860A8597F0FFFFE780803320
:101410000328040083564400A6881D08814701471D
:10142000E51642868A854E8597000000E780408E4B
:101430002A8919E5A685228597B0FFFFE780E0C1DC
:101440004A8541011713FFFF670003CB4A860A85CF
:1014500097F0FFFFE780002F6DB71713FFFFE7023C
:1014600063C62E848C414111AA8983871500328975
:10147000914463D30700A1449757FF1F938747E226
:101480009C43A1C7C1C68D472310F10083C7250027
:101490004A852301F10083C73500A301F10083C70A
:1014A00045002302F10083C75500A302F10083C762
:1014B000650093059100A30301002303F1002304B9
:1014C000010097F0FFFFE780C0250C404A860A859F
:1014D00097F0FFFFE78000278356440003280400AD
:1014E0008A85858EC2061D08C1822312D400A68873
:1014F00081470147E51642864E8597000000E78048
:1015000060B041011713FFFF670003BF4A860A85D9
:1015100097F0FFFFE78000234DBF1713FFFFE7029F
:1015200003BCB335B000011185052A891315F601F6
:10153000336515012308B1009305110136843AC6BD
:1015400032C03EC442C297F0FFFFE780801DA24731
:101550001248425593D68700230BF1009305910161
:1015600093578800A30AD100A30BF100230C0101BB
:1015700097F0FFFFE780E01A324702460328040095
:10158000B337E000835644009207914411C2A1444E
:101590004A85A68842860C0897F0FFFFE7804077CF
:1015A0002A8919E5A685228597B0FFFFE780E0AA82
:1015B0004A8505611713FFFF6700A3B41713FFFFE8
:1015C000E70243B001113EC68647B335B00085053A
:1015D000AA891315F6015D8D2308B1009305110149
:1015E00036843A89B28442C446C297F0FFFFE7804E
:1015F000401322489248164593578800A30AF100E9
:101600009305910193D78800230B0101A30BF100EF
:10161000230C110197F0FFFFE780A0103247104024
:1016200083564400B337E00092070328090091482D
:1016300091C0A1480C084E8597000000E780809C6F
:10164000AA8401E9835544004A8597B0FFFFE780EB
:10165000C0A0268505611713FFFF6700E3A9AA95BF
:101660009307F00F17070100130707686317B5000A
:1016700013C5F7FF1375F50F828005058346F5FF47
:10168000B58FBA9783C70700D5B7035745001441F4
:101690009307F00F170601001306066536974207F9
:1016A0004183139506014181631BE500AD8FB2971D
:1016B00003C50700130515F3133515008280850651
:1016C00003C5F6FFA98FB29783C70700D9BF1713C9
:1016D000FFFFE702C3A0B28736842E86BA86AA85AA
:1016E0003E85BA8497F0FFFFE7806052634F0500A4
:1016F000228597D00000E780E0782A86A686A2851A
:10170000268597F0FFFFE78080501713FFFF6700E3
:10171000439F1713FFFFE702E39A5D712A8BAE8A9E
:10172000170501001305C5592C00B284368ABA8901
:101730003E8997F0FFFFE780C04F2A845DE13410B7
:101740004146DA85280097F0FFFFE780404C2A8465
:1017500049E98547A303F100A6C293077100240855
:10176000BEC4A68685470D462C18281002DC02DE72
:10177000D6C0BEC697F0FFFFE78000442A8435E15B
:1017800083477102A6860D4693F7F7072300FA00F8
:10179000C1473EDE2C188947281026DCA303F10040
:1017A00097F0FFFFE78040412A8405ED4146A6857A
:1017B0004E8597D00000E78060488D47A6860D468D
:1017C0002C182810A303F10097F0FFFFE780C03E1C
:1017D0002A8401E94146A6854A8597D00000E78022
:1017E000E045228561611713FFFF6700E39017133F
:1017F000FFFFE702C38E97F700009387E7A09843A7
:1018000083C7470079712A89AE8417050100130543
:10181000A54B0C083AC42306F10097F0FFFFE780C0
:1018200040412A8405ED14104146CA85080897F006
:10183000FFFFE780C03D2A8415E1140815462C00FF
:10184000081097F0FFFFE780803C2A8401E92146D9
:101850002C08268597D00000E780403E2285456110
:101860001713FFFF6700E3891713FFFFE7022387C2
:1018700097F70000938747999C477971AA842E8433
:10188000170501001305C5440C083EC697F0FFFF7D
:10189000E780203A0DE914104146A685080897F024
:1018A000FFFFE780C03605E1140811466C00081000
:1018B00097F0FFFFE780A03519E58347F10193F723
:1018C000F7032300F40045611713FFFF67006383EC
:1018D0001713FFFFE702A3803688A148814701471D
:1018E000E54697F0FFFFE780A0421713FFFF670070
:1018F00043811703FFFFE702837E3688A1488147B3
:101900000147E54697F0FFFFE780C06F1703FFFF31
:101910006700237F1703FFFFE702637C01112A841E
:101920002E850C0832C697F0FFFFE780803009ED66
:10193000324797060100938626381008C145228554
:1019400097000000E780E0D805611703FFFF6700FC
:10195000437B1703FFFFE70283784111C1472EC085
:1019600032C48A8509463EC23EC697F0FFFFE78033
:10197000A02441011703FFFF6700A3781703FFFFAF
:10198000E702E3754111AE8613061009AA850A85A0
:1019900002C002C202C402C697F0FFFFE780202700
:1019A00041011703FFFF6700C3751703FFFFE7023D
:1019B0000373328797060100938606322E869305BD
:1019C000000297000000E780C0D01703FFFF670008
:1019D00043731703FFFFE70283707971C1472ACC75
:1019E0002ED032D42C080D4628003ECE3ED23ED614
:1019F00002C402C602C802CA97F0FFFFE780C01BFC
:101A000045611703FFFF6700C36F1703FFFFE7027E
:101A1000036D0111AA842E84170501001305452CBE
:101A20008A8597F0FFFFE780C02015E5140841463E
:101A3000A6850A8597F0FFFFE780601D09ED8347C3
:101A4000E1010347F101A207D98FCA07C983617772
:101A5000D98F2310F40005611703FFFF6700636A45
:101A600015CD1703FFFFE70283679747FF1F938793
:101A7000E73090439745FF1F938585301745FF1F3B
:101A80001305C52B97D00000E78000C51745FF1F41
:101A90001305C52A1703FFFF6700A3661745FF1F3D
:101AA0001305C52982808DCD1703FFFFE70223634D
:101AB0009747FF1F9387872C944301112E840A8632
:101AC0009745FF1F9385C52B97D00000E78040C640
:101AD0000A850294014505611703FFFF67006362F1
:101AE0007D5582801703FFFFE702635F97D00000F8
:101AF000E78080D19747FF1F23A2A72817F5FFFF94
:101B00001305E5C997B00000E780C0741703FFFF15
:101B10006700235F1747FF1F1307872893171500D8
:101B200008433E95FD572310F50082801703FFFF01
:101B3000E702E35A2A84084009E51703FFFF67001C
:101B4000435C1C4158401CC06313E5005CC08347E4
:101B5000550023200500F99BA302F50097A0FFFF85
:101B6000E780207CC9BF1703FFFFE702A355974713
:101B7000FF1F9387E72498432A8411CB83473500BE
:101B800093F7070289C70355050089450297130596
:101B9000440197B00000E780403B835504000355A3
:101BA000E40097300000E780A00C485819C597A0C2
:101BB000FFFFE7800077232A0402130584039700C0
:101BC0000000E780E0F68144B1499790FFFFE7808D
:101BD000006D63CBA402834734002320040493F7F1
:101BE00027FCA301F40000489790FFFFE780206CDA
:101BF00013161500814522859700FFFFE7802051CD
:101C00001703FFFF6700434FB3873403032904031F
:101C100085043E994A8597000000E78060F123041F
:101C2000090065B78347350093F7070299E301453B
:101C300082808357E500E39CB7FEC167FD176316FA
:101C4000F60005458280054599A81703FFFFE702C6
:101C5000034993170601C187B2842A840149635955
:101C6000F002835705009DCB01456367F6000345ED
:101C700084003E953325A6001375F50F0DA01C4872
:101C800013171900BA9783D70700E38E97FA05094F
:101C90009790FFFFE780A061E343A9FE014517038A
:101CA000FFFF670003461703FFFFE702A341AE896A
:101CB000AA849790FFFFE78040552A8497D0FFFFC2
:101CC000E780A02EAA86014713068401970500002D
:101CD000938585E41745FF1F1305C50C9790FFFFFB
:101CE000E780C01B2A8925C98C441304C5002285BE
:101CF0009E0593F5050897A0FFFFE780403CCC4088
:101D000083877400E18163DD070493E5050822857C
:101D100097A0FFFFE780A03A0D46938544002285F7
:101D200097A0FFFFE780C03683D50400228597A0E7
:101D3000FFFFE780E03D83D52400228597A0FFFFC9
:101D4000E780003D03D6490083A50900228597A0BE
:101D5000FFFFE780E0334A851703FFFF6700C339C1
:101D600093F5F5076DB71703FFFFE702433701113E
:101D70002A84328532C697A0FFFFE780E02797804C
:101D8000FFFFE780A033835704001747FF1F1307A7
:101D9000A71A3246231BF100930700F8A30DF100A8
:101DA0001C471843231AA1008983858BB307F7408A
:101DB000B28548083ECE231C0100230D0100970088
:101DC0000000E78080EE05611703FFFF67006333C3
:101DD0001703FFFFE702032F004101453DC49304B1
:101DE000C40026853289AE8997A0FFFFE780C02412
:101DF00095452A8A2685035B040197A0FFFFE780AB
:101E00002021268597A0FFFFE780603E8D45AA8AA6
:101E1000268597A0FFFFE780A01F268597A0FFFFDC
:101E2000E780E03C5C48420A135A0A01D2975CC43E
:101E300023186401814763983A0146054D813306B2
:101E400025419337160013F5F70F1703FFFF6700BF
:101E5000A32A1703FFFFE702032689692A8BAE8BAB
:101E6000328AB68A81440144314CFD199790FFFFB4
:101E7000E780E04263CDA4009790FFFFE780204514
:101E8000018D33B5AA001703FFFF6700432633898E
:101E9000840383270B003E9963170A008347890058
:101EA00085043E94E1B703560A00DE854A8533F681
:101EB000C90097000000E780E0F16DD10545E1B76A
:101EC0001703FFFFE702A32101112A847C000355B9
:101ED000E5003ECAB70707003ECC7C003ECE972007
:101EE0000000E78020082A898545480897A0FFFF61
:101EF000E78020399945480897A0FFFFE780E01563
:101F0000AA844A8597200000E780A0082380A400C7
:101F10009747FF1F938747029C434166130606F0CD
:101F20009396870113D78701558F93D68700F18E3B
:101F3000558FA207B706FF00F58FD98F11462C00E9
:101F4000138514003EC497D00000E78020CF5008CE
:101F5000A38204008945228597000000E780E0E025
:101F600019C9AA851305840397A0FFFFE780E03114
:101F70003C4085073CC005611703FFFF67006318FD
:101F80001703FFFFE702A3159790FFFFE7802034B8
:101F90002A8405049790FFFFE78060323305A4028E
:101FA000F14791453305F50297200000E78020BAFC
:101FB00011E565551703FFFF6700A3149747FF1F3F
:101FC00023A8A7DE9790FFFFE78060302A840504EE
:101FD0009790FFFFE780A02E3305A40289450605F0
:101FE00097200000E780A0B669D59747FF1F23A977
:101FF000A7DA9790FFFFE780802D2A840504979049
:10200000FFFFE780C02B3304A4029747FF1F239BE9
:1020100087D89790FFFFE780802B2A849790FFFF57
:10202000E780E029930714003385A7029747FF1F35
:10203000239BA7D6970701009387478E1747FF1F5B
:102040002326F7D60145BDB71703FFFFE702830735
:10205000AA842E8901449749FF1F9389E9ED130A49
:1020600080069790FFFFE78080256347A400014525
:102070001703FFFF670043083305440383A70902E2
:102080004A86A6853E9597000000E780E0B919E1F1
:102090000504C1BF0545E9BF1703FFFFE702A30120
:1020A000AA8A2E8BB28B368C3A8A814401448149AC
:1020B000974CFF1F938C4CE8130D80069790FFFF01
:1020C000E780E01F63C9A40011E085494E8517032E
:1020D000FFFF6700C3013389A40383A70C025E8658
:1020E000D6853E994A8597000000E780E0B31DC180
:1020F0009790FFFFE780A01D0544636D4501D286E0
:102100006286DA851305090397000000E780A0D4F2
:1021100011C1854985045DB71703FFFFE70283FA04
:10212000C16441112A8901449749FF1F9389C9E07D
:10213000130A8006FD1436C632C42EC29790FFFFE4
:10214000E780E01792452246B2466348A400014565
:1021500041011703FFFF670023FA3305440383A7F8
:1021600009023E9509C683473500C18B9DC791C6BC
:102170008347350093F707028DC3630699008357A1
:10218000E500639C27010357050001CB63E7E500E9
:1021900083478500BA97E3CDF5FA050469BF1703B5
:1021A000FFFFE70223F2C1642A8901449749FF1F18
:1021B000938989D8130A8006FD149790FFFFE78062
:1021C00000106346A4001703FFFF6700E3F2330526
:1021D000440383A709023E958357E500638A97006D
:1021E000630499006396270197000000E780E09759
:1021F0000504E1B71703FFFFE70263EB89692A8A49
:10220000AE8A328BB68B8144174CFF1F130CCCD295
:10221000930C8006314DFD199790FFFFE780200A4F
:1022200063C6A4001703FFFF670023EC3389940300
:1022300083270C028355CA015A863E994A85970026
:102240000000E780609E31C1814D15A03384AD034D
:102250008327090303D60B00D68533F6C9003E94C5
:10226000228597000000E780E0B609E9850D979088
:10227000FFFFE780C002E3CBADFC01A822859700F9
:102280000000E780E08A23040400850471B7170387
:10229000FFFFE70243E24169AA8A014A174BFF1F89
:1022A000130B8BC97D19C14B054C9790FFFFE7803D
:1022B00000016346AA001703FFFF670043E3930989
:1022C0008006B3073A0383290B02BE9983D7E9003E
:1022D000638E270163842A01639A570103A489034B
:1022E00001E84E8597000000E780C0BD050A75BF74
:1022F00083570401639977099304C400268597A046
:10230000FFFFE78060D385452A8D2685835C040125
:1023100097A0FFFFE780C0CF268597A0FFFFE7804B
:10232000A0E762056185635905048D45268597A060
:10233000FFFFE780E0CD8945268597A0FFFFE78076
:1023400020CD8945268597A0FFFFE78060CC854595
:10235000268597A0FFFFE780E0CC8347050009476B
:1023600093F7F707639AE7009945268597A0FFFF43
:10237000E78040CBA30285014848337D2D01231817
:1023800094016A9548C40040A1BF1703FFFFE7020C
:1023900003D537E404008327041D82979747FF1F66
:1023A00083C787A61715FF1F1305051AA300F5009D
:1023B0008327441C82978327841C81461306F00FD1
:1023C0008145014582971703FFFF670083D31747B5
:1023D000FF1F1307679318439745FF1F83C5C5A2C7
:1023E0009747FF1F9387C7A083468703034697033A
:1023F0006397D5009747FF1F2388C7A0828083C5B6
:1024000087010347A7036317B6009747FF1F238D74
:10241000E79E828003C687016317C7009747FF1FA7
:102420002384D79E828083C68701130750026319D5
:10243000D700930760021747FF1F2307F79C82808E
:1024400083C68701130660026315D60093077002E6
:10245000DDB783C7870155BF9747FF1F938747990C
:10246000D44B0947638DE6081703FFFFE70223C734
:102470001749FF1F130909953E8483470900918B73
:102480009DCFB7E4040083A7041D829783A7441C53
:102490001745FF1F13058593829783A7841C8146E8
:1024A0001746FF1F0346869481450145829721C543
:1024B00083470900ED9B1747FF1F2305F7908347CC
:1024C000040093F7F70F85CB91471747FF1F232B86
:1024D000F79297000000E78080EB97000000E7800C
:1024E00040EFB7E70400BC4F414691451745FF1F39
:1024F0000345859082971703FFFF670083C08280A2
:102500001703FFFFE702A3BD8D4741116306F504E2
:10251000C5476308F50285476310F5029747FF1F1B
:102520002386A78EB7E70400BC4B93050010174520
:10253000FF1F0345658C829741011703FFFF67006A
:1025400043BC85471747FF1F2302F78CB7E70400FA
:10255000BC4B93050020E1BF9747FF1F9387478936
:10256000D44B1147638DE600B7E7040083A7071D2E
:102570008297B7E70400BC4B930500044DBF0549A3
:102580001747FF1F2320278983C7070032C62E84E1
:1025900093F7F70FD5D3B7E4040083A7041D7D1488
:1025A0001374F40F8297E37689FCB245994703C60A
:1025B0001500E3F0C7FCFC4409061745FF1F13058F
:1025C00025858297BC48930500081745FF1F0345E2
:1025D000A582829779BF1703FFFFE70243B0174731
:1025E000FF1F1307E7804047184B1C409746FF1F0B
:1025F00023A6F6806316E4001747FF1F2322F78007
:10260000130584FE9790FFFFE78040A9035564FF00
:102610009780FFFFE780C07197A0FFFFE78060D041
:102620001703FFFF6700E3AD1703FFFFE70223ABCC
:102630009737FF1F9387C77BD84BDC4789C7970025
:102640000000E78080F985471737FF1F232CF77AB2
:102650009737FF1F9387476B9C43930500021735FD
:10266000FF1F0345657983C787031737FF1F230DB6
:10267000F778B7E70400BC4B82971703FFFF6700AA
:1026800043A89737FF1F23A7A77682801703FFFF72
:10269000E70243A337E404007C4CA1451735FF1F34
:1026A0000345857582977C48A1451735FF1F034573
:1026B000A5749734FF1F9384A4738297DC4489EB3D
:1026C00097000000E78080D91703FFFF6700C3A2CF
:1026D00003D567FF9780FFFFE7808065AA896DD1EA
:1026E000D84891476310F7027C4C91451735FF1F7E
:1026F0000345857082977C4891451735FF1F034538
:10270000A56F829703A9490103D409018947B7E955
:1027100004001737FF1F2327F76E83A7091D210425
:102720004204829783C784011715FF1F1305C5E173
:1027300061191717FF1FA309F7E083A7491C418000
:1027400082979737FF1F2383076C83A7C91C814695
:1027500009469375F40F4A85829711E99737FF1F51
:1027600083C7077B89C79700FF1FE780A048B7E7AB
:102770000400BC4F2146A1451735FF1F0345C5671F
:10278000829799B71703FFFFE702639593F7052038
:1027900001112E8481CF97000000E78020E91345C6
:1027A000042005611703FFFF6700A39593F7051049
:1027B000A9CF9734FF1F9384A463DC4897000000DF
:1027C000E78020C11737FF1F13070754184383C73B
:1027D0008401034787036318F700DC4489C7970027
:1027E0000000E78080DF85471737FF1F232CF76045
:1027F000B7E70400BC4B930500021735FF1F0345E4
:10280000A55F82971345041069BF93F70508BDC7FC
:102810009737FF1F83C7D75FE91719469735FF1F03
:102820009385255F1305D10093F4F70F1739FF1F28
:102830000349095E97C00000E78040409397040178
:10284000C1831737FF1F1307275D231DF100231CCA
:10285000F1009737FF1F9387A7593ACE3ACAD8435A
:102860002306010009CBDC439315890154080D466A
:10287000E185680082971345040825B793F7250082
:10288000A5C39737FF1F9387A756D84B8947630681
:10289000F7029737FF1F83C7E75213F7270011EF9F
:1028A000918B99CFB7E70400BC4F1306000A894506
:1028B0001735FF1F03454554829713452400D5B5AE
:1028C0009737FF1F938747449C4383C78703173776
:1028D000FF1F230BF75297000000E78060DBF1BF7A
:1028E00093F7050281CB97000000E78060DA13457B
:1028F000040245BD93F7850081CB97000000E78077
:10290000E0D21345840071BD93F7150081CB970089
:102910000000E780A0B41345140061B593F74500AB
:1029200081CB97000000E78060B31345440095BD5C
:1029300093F7050495C39737FF1F83C7674B91CB68
:1029400097000000E780A0A491471737FF1F232BB3
:10295000F74A13450404B1B593F705010145E38235
:1029600007E49737FF1F9387A748D84B9147631019
:10297000F7049737FF1F9387E7449C4313D727003B
:102980008583D98F858B91E7B7E7040083A7071D5F
:102990008297B7E70400FC4F91451735FF1F0345A9
:1029A000A545829785471737FF1F232DF744134509
:1029B0000401C5BB9737FF1F238CA754828017F3F0
:1029C000FEFFE702C3719737FF1F23A9074297371E
:1029D000FF1F23A7074285471734FF1F1304C43284
:1029E0001737FF1F2320F7421C4083C78703173781
:1029F000FF1F230BF7409790FFFFE780809229C5C8
:102A00009717FF1F23A6A7B41C4017050000130546
:102A1000A5D783C787031737FF1F2307F73E17176D
:102A2000FF1FA303F7B29737FF1FA383073CB7E746
:102A3000040083A7070882979737FF1F238EA73AC2
:102A400017F3FEFF6700E36BB7C7898E938767EDC7
:102A50001717FF1F232EF7AE45BF1737FF1F03477A
:102A60002739795555E79737FF1F9387673803C78D
:102A7000170005079736FF1FA38CE63603C717001C
:102A80008D463377D7029736FF1FA383E63683C67A
:102A900017001737FF1F13072727184393F6F60F62
:102AA000A9EE834787031737FF1F230FF7348547A6
:102AB0001737FF1F230EF7329737FF1F9387873093
:102AC0009C430145998BA9E717F3FEFFE7022361B9
:102AD00037E404007C48C1451735FF1F0345C53165
:102AE00082973C4885451735FF1F0345E53082979F
:102AF000014517F3FEFF6700C36083C717008546D3
:102B00006395F6008347970379BF8347A70361BFA7
:102B100082809737FF1F83C7A72DA1CF17F3FEFF32
:102B2000E702E35B37E404009737FF1F2382072C9B
:102B30007C4885451735FF1F0345052C82977C4C43
:102B400091451735FF1F0345252B82977C489145FA
:102B50001735FF1F0345452A82973C48C145173565
:102B6000FF1F034565298297014517F3FEFF6700A4
:102B700043597955828017F3FEFFE70243562A84B2
:102B8000035565FF9780FFFFE780801A9737FF1F87
:102B900093870726D847BE841DEF9790FFFFE780F5
:102BA00080779C48232004009DEB9737FF1F23A9C3
:102BB00087249737FF1F23A38724B7E70400BC4B64
:102BC00089451735FF1F034525238297014517F3D4
:102BD000FEFF67000353630A8700184375BF80C375
:102BE0009737FF1F23AE8720C9BF7955CDB717F39D
:102BF000FEFFE702C34E9737FF1F9387A731884335
